:100000000C9486090C94B7090C94B7090C94B709A1
:100010000C94B7090C94B7090C94B7090C94B70960
:100020000C94B7090C94B7090C94B7090C94B70950
:100030000C94B7090C949F0F0C94B7090C94B70952
:100040000C94B7090C94B7090C94B7090C94B70930
:100050000C94B7090C94B7090C94B7090C94A10E31
:100060000C94B7090C94CA910C94A0910C94B70904
:100070000C94B7090C94B7090C94B7090C94B70900
:100080000C94B7090C94B7090C94B7090C94B709F0
:100090000C94B7090C94B7090C94B7090C94C210CE
:1000A0000C94B7090C94B7090C94B7090C94B709D0
:1000B0000C94B7090C94B7090C94B7090C94B709C0
:1000C0000C94B7090C94B7090C94B7090C94B709B0
:1000D0000C94B7090C94B7090C946A910C94409154
:1000E0000C94B7090C94061C0C94A57F0C94D37F38
:1000F0000C94870B0C94760B0C94D7260C94FF2B46
:100100000C941A0A0C9475260C94120A0C94F82775
:100110000C94797E0C94210A0C94B6250C94792BBE
:100120000C94AB290C94780B0C94310A0C9429385C
:100130000C94DB1D0C94A6240C94967F0C942B0A33
:100140000C941D0C0C94770B0C94CC2E0C94C20CBC
:100150000C94DE240C944C0A0C94CC0C0C94DD0C06
:100160000C94BE0C0C9452240C9472970C94FF25A2
:100170000C94B97F0C94F80C0C94032A0C94C77F50
:100180000C94C2770C941E0A0C9428240C9491822F
:100190000C94A71B0C945B260C94AE1D0C94D10CF4
:1001A0000C94A92B0C94830C0C94697F0C94E10C97
:1001B0000C94D5250C949D0C0C9496260C94AA1F97
:1001C0000C94B0950C940D240C940C0A0C94DD7FC7
:1001D0000C94CE0B0C94270A0C94A80C0C94BB1F07
:1001E0000C94AD230C94D90C0C949A0B0C9467834B
:1001F0000C9468280C94772E0C943F0A0C94EE26ED
:100200000C94870C0C94160A0C94C9290C94FD0BC1
:100210000C94350A0C94A10B0C94390A0C949D1B78
:100220000C94FB0C0C94B9090C94510A0C941A838D
:100230000C94430A0C94750B0C94F10C0C94342A16
:100240000C94A1270C94CE0C0C94470A0C944D0AE4
:100250000C946D0C0C9453280C94687F0C94D42B44
:100260000C941A280C94658E0C9497240C94180FF7
:100270004E414E494E495459494E46CDCCCC3D0A8B
:10028000D7233C17B7D13877CC2B329595E6241F6E
:10029000B14F0A000020410000C84200401C462027
:1002A000BCBE4CCA1B0E5AAEC59D7400407A10F3FA
:1002B0005A00A0724E18090010A5D4E80000E87694
:1002C00048170000E40B54020000CA9A3B000000EB
:1002D000E1F505000080969800000040420F000004
:1002E00000A08601000000102700000000E80300C5
:1002F0000000006400000000000A0000000000018F
:1003000000000000002C76D888DC674F0823DFC18E
:10031000DFAE59E1B1B796E5E3E453C63AE6519949
:100320007696E8E6C28426EB898C9B62ED407C6F72
:10033000FCEFBC9C9F40F2BAA56FA5F490055A2A29
:10034000F75C936B6CF9676DC11BFCE0E40D47FE35
:10035000F520E6B500D0ED902E030094357705002A
:1003600080841E080000204E0A000000C80C3333B1
:1003700033330F986E12831141EF8D2114893BE6C0
:100380005516CFFEE6DB18D1844B381BF77C1D9049
:100390001DA4BBE424203284725E228100C9F124B2
:1003A000ECA1E53D27436F6E74656E742D54797032
:1003B000653A20746578742F68746D6C0D0A0D0AA7
:1003C0003C68313E45504943204641494C3C2F68EA
:1003D000313E00485454502F312E302034303020DC
:1003E00042616420526571756573740D0A00416342
:1003F000636573732D436F6E74726F6C2D416C6CFB
:100400006F772D4F726967696E3A202A0D0A436F24
:100410006E74656E742D547970653A200053657260
:100420007665723A205765626475696E6F2F312E5A
:10043000370D0A00485454502F312E3020323030BE
:10044000204F4B0D0A00506F7374206661696C6514
:100450006400436F6E6E656374696F6E3A20636CFF
:100460006F73650D0A00436F6E6E656374696F6E1E
:100470003A20636C6F73650D0A436F6E74656E741A
:100480002D547970653A206170706C69636174698C
:100490006F6E2F782D7777772D666F726D2D757251
:1004A0006C656E636F646564002D2D2D2D2D2D57A9
:1004B00065624B6974466F726D426F756E646172EE
:1004C000796A673271564955533874654F41624EA7
:1004D000332D2D00436F6E74656E742D54797065E5
:1004E0003A206170706C69636174696F6E2F6F631D
:1004F0007465742D73747265616D00436F6E7465FD
:100500006E742D446973706F736974696F6E3A20ED
:10051000666F726D2D646174613B206E616D653D27
:100520002266696C65223B2066696C656E616D654B
:100530003D22002D2D2D2D2D2D5765624B697446C2
:100540006F726D426F756E646172796A673271564F
:100550004955533874654F41624E3300436F6E7492
:10056000656E742D4C656E6774683A2000436F6E3B
:1005700074656E742D547970653A206D756C74696C
:10058000706172742F666F726D2D646174613B20AF
:10059000626F756E646172793D2D2D2D2D576562E8
:1005A0004B6974466F726D426F756E646172796AE1
:1005B000673271564955533874654F41624E330066
:1005C000436F6E6E656374696F6E3A20636C6F7310
:1005D0006500504F53542055706C6F616420466124
:1005E000696C65643A2000234E6F2073656E736FEB
:1005F0007220666F722074656D7020262068756D9C
:10060000696469747921004E6F2053656E736F724F
:10061000210020666F722074656D70202620687539
:100620006D696469747921002353656E736F72205C
:100630004572726F72200053656E736F722045723F
:10064000726F7221002357726F6E672073656E732D
:100650006F7220666F722074656D70202620687539
:100660006D6964697479210057726F6E67205365F4
:100670006E736F7221004320483D00543D002020DE
:10068000202020202020202020202020202000208A
:10069000202020202020202020202020202020007A
:1006A000202020202020202020202020202020204A
:1006B000002020202020202020202020202020205A
:1006C000002020202020202020202020202020204A
:1006D0000054696D657374616D702075706C6F6125
:1006E00064206661696C65640053657474696E6743
:1006F00020636C6F636B2074696D65002365727293
:100700006F72202D200049502061646472657373FC
:100710003A2000496E76616C696420534D207374F1
:100720006570732070657220616E676C653D005363
:100730004D2073746570732070657220616E676CF4
:10074000653D003C703E54696D653A20003C2F6861
:10075000333E0A003C62723E4254206E616D653D3C
:10076000003C62723E506174683D003C68333E5309
:10077000797374656D3A2056657273696F6E3D00CA
:10078000506172616D657465727320726573657412
:1007900020646F6E6521002F6F652F736D6C696724
:1007A0006874706F2F73332F00234C616D70207647
:1007B0006F6C74616765207061726974793A2000AA
:1007C000235461626C6520616E676C652064697298
:1007D000656374696F6E3A20002343757272656EAB
:1007E0007420534D20697320230023534D3A5461E4
:1007F000626C652073746570732070657220616E21
:10080000676C653D0023534D3A506F6C6172697A95
:1008100065722073746570732070657220616E67F5
:100820006C653D002344485450494E3D00234448E4
:10083000543D00236E65743D424C4500236E657443
:100840003D5769466900236E65743D425400236636
:10085000747020757365726E616D653A003A00239D
:10086000486F7374207365727665722049502061F9
:100870006E6420506F72743A002354696D65207362
:1008800065727665722049503A002352656C617931
:1008900020646576696365733A002352656C6179FB
:1008A00020737461747573206C6162656C733A2097
:1008B000002352656C6179207374617465733A002A
:1008C0002352656C61792070696E733A00234E6F14
:1008D0002E206F6620636F6E74726F6C2072656C71
:1008E0006179733D00234E6F2E206F662072656C18
:1008F0006179733D0046696E64696E672057694689
:1009000069204950004E45543D426C7565746F6FC7
:100910007468204C45004E45543D426C7565746FBB
:100920006F7468004E45543D576946690053442032
:100930006F70656E206661696C004E65772064613A
:10094000746120636F6C6C656374696F6E2073747F
:1009500061727465640053484F57533D00484947DE
:1009600048004C4F57004E4557002343757272653F
:100970006E742073657474696E67733A00534554DE
:100980000053797374656D207265736574206174AA
:1009900020005245534554005052494E5450415244
:1009A00000524541445344005341564553443D0091
:1009B00023445320546865726D6F6D6574657220B1
:1009C00063616C6962726174656420666F72202372
:1009D0000044535400496E76616C696420616E670F
:1009E0006C6520666F7220004D323D004E3D004D1B
:1009F000323D004E3D002073746570732070657247
:100A000020616E676C653D005350413D005453506A
:100A1000413D00505350413D005350413D00207333
:100A2000746570732070657220616E676C653D003F
:100A300046313030300046353030004631303030CD
:100A400000414E474D0054414E47430050414E47F0
:100A50004300414E4743005461626C654000506F53
:100A60006C6172697A65724000414E474D3D005499
:100A7000414E474D3D0050414E474D3D00414E4790
:100A80004D3D00414E47533D005233300054414EDE
:100A900047533D0050414E47533D00414E47533D63
:100AA000005200414E474C453D0054413D005041ED
:100AB0003D00413D00414E474C453D005461626C54
:100AC0006520536574203000235475726E74616222
:100AD0006C6520536574203000523330004633304B
:100AE00000506F6C6172697A6572205365742030B2
:100AF0000023506F6C6172697A65722053657420AF
:100B00003000505A45524F3D00540050005A455253
:100B10004F005461626C652053657420300023548B
:100B200075726E7461626C6520536574203000507C
:100B30006F6C6172697A657220536574203000238E
:100B4000506F6C6172697A65722053657420300051
:100B500053455400505A45524F3D005A45524F009C
:100B600053504545443D005053504545443D005485
:100B700053504545443D0053504545443D004D3D8F
:100B8000004D4F544F523D004D3D004D4F544F527C
:100B90003D00534D3D00535445503D004453544E89
:100BA0003D005256484947483D0052564C4F573D2C
:100BB000004C4F5746414E54494D453D004849472A
:100BC000484D4F544F523D004C4F574D4F544F528C
:100BD0003D004849474854454D503D004C4F5754FF
:100BE000454D503D0054454D50433D007361766581
:100BF00053443D004E45543D0057694669204950D5
:100C00003A0049504144440041542B0050494E3D64
:100C10000042543D004C43443D00534554434C4F27
:100C2000434B00234C6F67676572204E616D653AD8
:100C300020004C4F474745520056455253494F4EAE
:100C4000002344657669636520737461747573204D
:100C50006661696C656420746F2075706C6F616487
:100C6000210023446576696365207374617475732C
:100C70002075706C6F616465642100555354415454
:100C80005553005265626F6F74696E672E2E2E0089
:100C90005245424F4F540053657276657220506F33
:100CA000727420757064617465640053504F5254BF
:100CB0003D0049502075706461746564005349506B
:100CC0003D002354696D6520536572766572204935
:100CD00050207570646174656400545349503D0040
:100CE00052454C41593F0052454C41592000435216
:100CF000454C41590044485450494E3D00524E41E4
:100D00004D453D004E523D005052494E54004E5507
:100D10004E4348554B3D004155544F535441525456
:100D20003D0074696D6520696E74657276616C3D15
:100D30000054494D453D0054494D455354414D5093
:100D40003D0054494D455354414D500053484F5771
:100D50004950005445535452454C4159004348456D
:100D6000434B433D00434845434B543D004453549B
:100D70003D004C5041524954593D0046414E3D00C2
:100D80004F56454E3D004448543D0050573D005598
:100D90005345523D00504154483D007C3C3E5E2B43
:100DA0003D3F2F5B5D3B2C2A225C0000002000238E
:100DB00000260029002C002F003200000100000353
:100DC000010601090100000A0B02090C0D0E0807BB
:100DD000030401000000000000000000000000000B
:100DE0000000000000000000000000000000000003
:100DF00000121110000000000000000000000000C0
:100E000000000000000000000000003C703E4C614B
:100E10006D7020616E64204D6F746F722044726932
:100E20007665727320537461747573EFBC9A3C2FAE
:100E3000703E003C21646F63747970652068746D46
:100E40006C3E3C68746D6C3E3C686561643E3C6D14
:100E500065746120636861727365743D22757466A0
:100E60002D38223E3C7469746C653E4F6E6C696E21
:100E700065206578706572696D656E74202D2050EF
:100E80006F6C6172697A6174696F6E206566666500
:100E9000637473206F66206C696768743C2F746993
:100EA000746C653E3C2F686561643E3C626F64799A
:100EB0003E3C68313E4F6E6C696E652065787065AA
:100EC00072696D656E74202D20506F6C6172697A45
:100ED0006174696F6E2065666665637473206F6602
:100EE000206C696768743C2F68313E003C68343E72
:100EF000436F7079726967687428432932303230E1
:100F00002D323032322E50726F662E205945554E9A
:100F10004720596175205975656E3C2F68343E3CF9
:100F20002F626F64793E3C2F68746D6C3E003C68A4
:100F3000313E43616E6E6F74206765742073656E19
:100F4000736F722072656164696E6773213C2F68EC
:100F5000313E002377656273657276657220626543
:100F600067696E730053657474696E672049500039
:100F700053657474696E67204465766963652049BA
:100F800050202E2E2E00506F6C6172697A6572208F
:100F900053657420300023506F6C6172697A6572FA
:100FA0002053657474696E6720302E2E2E005465B0
:100FB0007374204C616D70732F46616E730065729F
:100FC000726F72206F70656E696E672066696C65FE
:100FD0003A20004C616D70204D6F746F7200235485
:100FE000696D652020202020204461746520202028
:100FF00020205365636F6E647320506F6C6172695B
:101000007A6572205461626C652054286F432920F0
:1010100048282529202000696E69742E20646F6E8F
:10102000652E00534420696E69742E206661696CD8
:1010300065642100696E69742E206661696C65645F
:1010400021005245424F4F540053657474696E67D6
:101050002049502063616D004C4F474745520023A3
:1010600023204F452057656C636F6D652023230057
:10107000496E697469616C697A696E6720534420AE
:10108000636172642E2E2E0053797374656D207324
:1010900074617274696E672E2E2E00202D2075707B
:1010A0006C6F616420627920504F535420666169EF
:1010B0006C65642100202D2075706C6F6164206266
:1010C0007920504F5354204F4B210053797374654E
:1010D0006D207265737461727465642100205379A8
:1010E0007374656D20726573746172746564210038
:1010F000234E6574776F726B206D61696E746169E0
:101100006E656420617420002323436F6D6D616EF2
:101110006440000A004465766963652073746174F5
:101120007573206174200000002200250028002B28
:10113000002E003100340002010000050108010BFF
:101140000100002100240027002A002D0030003378
:101150000001010000040107010A01010210202022
:1011600008081020401020408002010201080402FB
:101170000101020408102040808040201008040271
:1011800001800402018040201008040201080402CA
:1011900001010204081020408001020408102040D0
:1011A0008005050505070508080808020202020A6D
:1011B0000A080804040404010101010101010103FA
:1011C00003030303030303040707070C0C0C0C0CB5
:1011D0000C0C0C0202020206060606060606060BA8
:1011E0000B0B0B0B0B0B0B417070656E64206D6568
:1011F00061732E200053696E676C65206D656173A5
:101200002E200053617665206D65617375726520CF
:10121000746F3A0020202020202020202020202031
:101220002020202000000001000100101002000119
:10123000000100B0000000160000002800000010AF
:10124000000000200000000100010000000000007C
:10125000000000000000000000000000000000008E
:1012600000000000000000FF000000FFFF0000FF82
:10127000FF0000FFFF0000CFBF0000C7BF0000C39A
:10128000BF0000C1BF0000C0BF000000000000C0E0
:10129000BF0000C1BF0000C3BF0000C7BF0000CF38
:1012A000BF0000FFFF0000FFFF0000000000000083
:1012B000000000000000000000000000000000002E
:1012C000000000000000000000000000000000001E
:1012D000000000000000000000000000000000000E
:1012E0000000000000000000000000557365722D32
:1012F0006167656E743A202A0D0A446973616C6CEB
:101300006F773A202F0D0A007297B09511241FBEF7
:10131000CFEFD1E2DEBFCDBF00E00CBF18E0A0E010
:10132000B2E0EAE3F4E701E00BBF02C007900D92E0
:10133000A438B107D9F724E1A4E8B8E001C01D92B0
:10134000A031B207E1F719E0C5E8D9E000E006C036
:1013500021970109802FFE010E9424B7C438D107CC
:1013600080E00807A9F70E942F9A0C940BBA0C94FE
:1013700000008DED9FE7892B49F080E090E0892BFC
:1013800029F00E94DD7F81110E94000080E090E042
:10139000892B49F080E090E0892B29F00E94000021
:1013A00081110E94000080E090E0892B49F080E0EC
:1013B00090E0892B29F00E94000081110E9400001A
:1013C00083ED9FE7892B49F080E090E0892B29F09D
:1013D0000E94D37F81110C940000089581508231C6
:1013E00008F05AC0E82FF0E08827E650F64F8F4FFC
:1013F0000C9424B71A0A1E0A0C0A120A160A4C0A7E
:10140000210A270A2B0A310A350A390A3F0A430AF8
:101410004C0A470A4D0A510A809180008F778093C9
:1014200080000895809180008F7DF9CF80918000A9
:10143000877FF5CF84B58F7784BD089584B58F7D80
:10144000FBCF8091B0008F778093B000089580919A
:10145000B0008F7DF9CF809190008F7780939000BE
:101460000895809190008F7DF9CF80919000877FC3
:10147000F5CF8091A0008F778093A0000895809190
:10148000A0008F7DF9CF8091A000877FF5CF80915C
:1014900020018F77809320010895809120018F7D16
:1014A000F9CF80912001877FF5CF4F925F926F92A5
:1014B0007F928F929F92AF92BF92CF92DF92EF92E4
:1014C000FF920F931F93CF93DF934B015C018091A9
:1014D000980B9091990BA0919A0BB0919B0B88154A
:1014E0009905AA05BB0509F4C6C08CE3C82ED12C0A
:1014F000E12CF12CC501A70196010E948EB56093E5
:101500009C0BCA01B901A70196010E948EB5609398
:101510009D0BC501B40120E13EE040E050E00E9497
:101520008EB5CA01B90128E130E040E050E00E94E8
:101530008EB560939E0BC501B40120E831E541E012
:1015400050E00E948EB569017A01CA01B9016C5F51
:101550007F4F8F4F9F4F27E030E040E050E00E94E8
:101560008EB56F5F60939F0B412C512C320140E090
:1015700004E610E0C0E9D1E0242F30E02E54384FCB
:10158000F901E370FF273097F9F4C901B8010E940F
:1015900010B7892B31F4C901BE010E9410B7892B05
:1015A00099F48EE691E0A0E0B0E0480E591E6A1E64
:1015B0007B1ED301C201AA27BB27C816D906EA069B
:1015C000FB0638F04F5FD8CF8DE691E0A0E0B0E0A9
:1015D000ECCF4093A20BC90164E670E00E9410B703
:1015E000EC01C90160E971E00E9410B7309721F465
:1015F0002097D9F40097C9F04DE651E060E070E023
:10160000441A550A660A770AC418D508E608F70886
:10161000A5E2B3E020E0213069F43097E9F52097A6
:1016200011F40097C9F54DE106C04EE651E060E0C7
:1016300070E0E6CF4C9150E070E060E031E0320FB6
:10164000C416D506E606F70640F0C41AD50AE60A1F
:10165000F70A1196232F3C30F1F62F5F2093A10B50
:10166000C394C092A00B8092980B9092990BA09279
:101670009A0BB0929B0BDF91CF911F910F91FF902E
:10168000EF90DF90CF90BF90AF909F908F907F9022
:101690006F905F904F9008954CE1CDCF2091A40AB8
:1016A000260F3327331F21323105ECF420916D0EC4
:1016B000FC0190E080E0243069F082E00895A09180
:1016C000A40A2191AC014C57554FA40FB52FB11D61
:1016D0002C930196861798F38091A40A680F609363
:1016E000A40A80E0089581E008950895089508957A
:1016F000E091270C8091260CE81730F4F0E0ED59CA
:10170000F54F808190E008958FEF9FEF08959091BD
:10171000270C8091260C2FEF3FEF981748F4E92F04
:10172000F0E0ED59F54F208130E09F5F9093270C5A
:10173000C90108958091260C9091270C891B990B63
:101740000895CF92DF92EF92FF920F931F93CF9362
:10175000DF937C01CB018A012091730E222389F053
:10176000EB016B01C40ED51ECC15DD0569F0699146
:10177000D701ED91FC910190F081E02DC701199501
:10178000F3CF642F0E944E0BC801DF91CF911F91C0
:101790000F91FF90EF90DF90CF900895CF93DF935C
:1017A0001F92CDB7DEB769832091730E2223F9F023
:1017B0002091960E203258F021E030E0FC01338376
:1017C000228390E080E00F90DF91CF910895809187
:1017D000740EE82FF0E0EB58F14F998190838F5F02
:1017E0008093740E8093960E81E090E0ECCF61E0E0
:1017F000CE0101960E944E0BF7CFDC015996ED9178
:10180000FC913097B9F083899489A589B68942857E
:10181000538564857585841B950BA60BB70B8115C5
:1018200020E89207A105B10538F08FEF9FE7A0E00F
:10183000B0E0089590E080E00895CF93DF931F9289
:10184000CDB7DEB76983DC01ED91FC910280F381B5
:10185000E02D41E050E0BE016F5F7F4F19950F9082
:10186000DF91CF910895FC0120812EBD9B01215075
:10187000310941F051810DB407FEFDCF4EB55EBD7B
:101880004193F5CF61507109860F971F0DB407FE84
:10189000FDCF2EB5FC0120830895E0912C0CF09132
:1018A0002D0C908180912B0C809589238083089545
:1018B0008EBD00000DB407FEFDCF8EB5089590E0FB
:1018C00020912E0C233339F40C96982F990F990FF1
:1018D000990F80E008954896F8CFCF93DF931F9239
:1018E000CDB7DEB76983DC01ED91FC910280F38115
:1018F000E02D41E050E0BE016F5F7F4F19950F90E2
:10190000DF91CF910895FC01818D928D0895CF9341
:10191000DF931F92CDB7DEB76983DC01ED91FC91B7
:101920000280F381E02D41E050E0BE016F5F7F4F08
:1019300019950F90DF91CF910895FC019485FB01DB
:101940008485981303C081E0983008F080E0089502
:10195000CF93DF931F92CDB7DEB76983DC01ED91A2
:10196000FC910280F381E02D41E050E0BE016F5F09
:101970007F4F19950F90DF91CF910895FC017687E5
:1019800065870895DC01ED91FC91068CF78DE02DC3
:10199000199591E089270895862F089581E086277B
:1019A000089521E0FC018485883008F020E0822F32
:1019B0000895FC01848595850895FC0184899589A5
:1019C000089520E334E0FC0131832083FB0140894A
:1019D000518962897389FC014283538364837583CF
:1019E0000895DC01ED91FC91048CF58DE02D1994A6
:1019F00090E080E00895CF92DF92EF92FF920F93F4
:101A00001F93CF93DF93CDB7DEB7AF970FB6F894A0
:101A1000DEBF0FBECDBF7C016A0100E314E01A8374
:101A200009831C861B8688EE93E0A0E0B0E08D87DA
:101A30009E87AF87B88B8AEB93E09A878987188F48
:101A40000F8B198E1A8E1B8E1C8E88E089A31BA704
:101A50000AA71CA61DA61EA61FA68091291090915C
:101A60002A10A0912B10B0912C108EA39FA3A8A791
:101A7000B9A78B839C83AD83BE8318861F82AE017A
:101A8000465D5F4FCE0101960E942587813091050A
:101A9000B1F4D701ED91FC910488F589E02D1DA3E7
:101AA0000CA38CA59DA5AEA5BFA58EA39FA3A8A79B
:101AB000B9A7A601BE016C5D7F4FC7011995AF960E
:101AC0000FB6F894DEBF0FBECDBFDF91CF911F914F
:101AD0000F91FF90EF90DF90CF900895FC01A48DBF
:101AE000A80FB92FB11DA35ABF4F2C91848D90E040
:101AF00001968F739927848FA689B7892C93A08923
:101B0000B1898C91837080648C93938D848D9813AC
:101B100006C00288F389E02D80818F7D808308953F
:101B2000CF93DF93282F30E0F901EB53F24F8491EC
:101B3000F901E55AFE4ED491F901EF55FE4EC491DC
:101B4000CC23A1F081110E94EE09EC2FF0E0EE0F02
:101B5000FF1FE555F24FA591B491EC91ED2381E083
:101B600090E009F480E0DF91CF91089580E090E06B
:101B7000FACF1F93CF93DF93282F30E0F901EB5377
:101B8000F24F8491F901E55AFE4ED491F901EF55D7
:101B9000FE4EC491CC23A9F0162F81110E94EE09AC
:101BA000EC2FF0E0EE0FFF1FE95DFE4EA591B49122
:101BB0008FB7F894EC91111108C0D095DE23DC9317
:101BC0008FBFDF91CF911F910895DE2BF8CFCF9378
:101BD000DF9390E0FC01E55AFE4E24918F559E4E16
:101BE000FC0184918823D1F090E0880F991FFC01BB
:101BF000EF5BFE4EA591B491FC01E95DFE4EC591EF
:101C0000D49161110EC09FB7F8948C91E22FE095AA
:101C10008E238C932881E223E8839FBFDF91CF91AD
:101C200008958FB7F894EC91E22BEC938FBFF6CF29
:101C30003FB7F8948091B60B9091B70BA091B80B79
:101C4000B091B90B26B5A89B05C02F3F19F001969E
:101C5000A11DB11D3FBFBA2FA92F982F8827BC0106
:101C6000CD01620F711D811D911D42E0660F771F2E
:101C7000881F991F4A95D1F708958F929F92AF922E
:101C8000BF92CF92DF92EF92FF926B017C010E9494
:101C9000180E4B015C01C114D104E104F104B9F048
:101CA0000E94180E681979098A099B09683E7340D9
:101CB0008105910580F321E0C21AD108E108F108FD
:101CC00088EE880E83E0981EA11CB11CE4CFFF9023
:101CD000EF90DF90CF90BF90AF909F908F9008953E
:101CE0002FB7F8946091B20B7091B30B8091B40B45
:101CF0009091B50B2FBF08956093AD0B7093AE0B11
:101D00008093AF0B9093B00B645D7E4F8F4F9F4FCE
:101D10006093A90B7093AA0B8093AB0B9093AC0BC1
:101D200082E090E09093A80B8093A70B0E94700E26
:101D30006093A30B7093A40B8093A50B9093A60BB9
:101D400008951F920F920FB60F9211242F933F9375
:101D50008F939F93AF93BF938091B20B9091B30BEE
:101D6000A091B40BB091B50B3091B10B23E0230FD0
:101D70002D3758F50196A11DB11D2093B10B80930D
:101D8000B20B9093B30BA093B40BB093B50B8091AF
:101D9000B60B9091B70BA091B80BB091B90B01960F
:101DA000A11DB11D8093B60B9093B70BA093B80BF8
:101DB000B093B90BBF91AF919F918F913F912F91AC
:101DC0000F900FBE0F901F90189526E8230F0296D4
:101DD000A11DB11DD2CFFC01248131E03093730EDF
:101DE0002093950E1092740E1092960E8385682B98
:101DF00082ED9FE00E94CE0B81E00C948A830F93CA
:101E00001F93CF938C01C62F0E94EB0E6C2F646042
:101E1000C8010E94EB0E6C2F6B7FC8010E94EB0E75
:101E200083EC90E00197F1F7CF911F910F91089506
:101E30000F931F93CF938C01C62F607F61600E9428
:101E4000FF0E80E1C89FB00111246160C8010E94AB
:101E5000FF0E81E090E0CF911F910F910895CF92F6
:101E6000DF92EF92FF920F931F930E94700E8B01EF
:101E70009C01C090A30BD090A40BE090A50BF09018
:101E8000A60B6091AD0B7091AE0B8091AF0B909152
:101E9000B00B0C191D092E093F09083E13402105FE
:101EA0003105E0F0DC01CB010196A11DB11D80934D
:101EB000AD0B9093AE0BA093AF0BB093B00BB701EB
:101EC000A60148515C4F6F4F7F4F4093A30B509337
:101ED000A40B6093A50B7093A60BC7CF1F910F9116
:101EE000FF90EF90DF90CF9008950E942F0F0E94F7
:101EF000550A8091A20B90E08E54984F08950E944D
:101F00002F0F0E94550A8091A10B90E008950E9426
:101F10002F0F0E94550A8091A00B90E008950E9417
:101F20002F0F0E94550A80919D0B90E008950E940A
:101F30002F0F0E94550A80919E0B90E008951F92EA
:101F40000F920FB60F9211240BB60F922F933F935F
:101F50004F935F936F937F938F939F93AF93BF93B1
:101F6000EF93FF938091C80A0E94900D2091CB0AB5
:101F70003091CC0A2F5F3F4F3093CC0A2093CB0A8D
:101F80009091CA0A953618F096E09093C70A9091FE
:101F9000C70A943009F46EC0F8F4923031F19330EE
:101FA00009F44CC09091C90A992319F0811171C0AC
:101FB0002F9AFF91EF91BF91AF919F918F917F9158
:101FC0006F915F914F913F912F910F900BBE0F90AA
:101FD0000FBE0F901F901895953009F457C096309A
:101FE00009F791E09093970B4FC08111DBCF2091BF
:101FF000CB0A3091CC0A2436310528F41092CC0A51
:102000001092CB0ACFCF1092970B1092CA0AE09190
:10201000CA0A91E09E0F9093CA0AF0E02091CB0A81
:102020003091CC0AEE0FFF1FE353F54F318320832D
:102030001092CC0A1092CB0A93E019C0813009F0BB
:10204000B1CFE091CA0A91E09E0F9093CA0AF0E0E6
:102050002091CB0A3091CC0AEE0FFF1FE353F54FCE
:10206000318320831092CC0A1092CB0A94E0909393
:10207000C70A98CF882359F22091CB0A3091CC0A15
:102080002536310508F48ECF95E0F1CF81118ACF46
:10209000B5CF2F988ECF10926D0E81E080936C0E8D
:1020A0001092470E61E084E10E94B90D61E085E184
:1020B0000E94B90DE9EBF0E080818E7F8083808102
:1020C0008D7F808388E48093B80085E48093BC0092
:1020D0000895CF93DF9391E09093830A8823B9F01A
:1020E000C091B800D091BA008091BC008A7B8093E7
:1020F000BC0060E084E10E94B90D60E085E10E94CF
:10210000B90D0E944B10D093BA00C093B800DF9174
:10211000CF91089585ED8093BC0080916F0E9091D2
:10212000700EA091710EB091720E0796A11DB11D97
:1021300023E0B695A795979587952A95D1F7209195
:10214000BC0024FD03C010926D0E089540916F0EE7
:102150005091700E6091710E7091720E452B462B4E
:10216000472B69F30097A105B10541F025E32A95B6
:10217000F1F700000197A109B109E1CF80916E0E3E
:102180000C9469101F920F920FB60F9211240BB688
:102190000F922F933F934F935F936F937F938F9300
:1021A0009F93AF93BF93EF93FF938091B900887F84
:1021B000803609F44DC008F040C0883209F4A9C047
:1021C00028F5803109F49DC0C8F4882309F4FBC0C8
:1021D000883009F496C0FF91EF91BF91AF919F9124
:1021E0008F917F916F915F914F913F912F910F90C0
:1021F0000BBE0F900FBE0F901F901895883109F4F9
:1022000088C0803241F780936B0E14C0803409F48B
:102210009DC040F48033B9F38833E9F680936B0EA8
:1022200085ECB0C0803509F485C0883509F496C0C6
:10223000883489F60E948A10CECF883909F48CC080
:1022400038F5883729F050F4883611F0803719F6C0
:1022500083E080936D0E1092C60A57C0883809F447
:102260007BC0803919F0803809F0B5CF8091C60A5B
:10227000803208F071C0E091C60A81E08E0F809331
:10228000C60A8091BB00F0E0EA55F54F80833DC05F
:10229000803B39F0E0F4803A09F479C0883A09F0DB
:1022A0009ACF84E080936D0E1092A50A1092A40A32
:1022B000E091240CF091250C19958091A40A8111CC
:1022C0000FC081E08093A40A1092840A09C0803C68
:1022D00009F4A6CF883C09F4A3CF883B09F07BCF53
:1022E000E091A50A81E08E0F8093A50AF0E0EC57FB
:1022F000F54F80818093BB009091A50A8091A40A3C
:1023000029C08091480E8093BB0085EC8093BC006F
:1023100062CF90916A0E8091690E981758F5E091FE
:102320006A0E81E08E0F80936A0EF0E0E75BF14F5A
:102330008081E9CFE0916A0E81E08E0F80936A0E72
:102340008091BB00F0E0E75BF14F808390916A0ED3
:102350008091690E9817C8F285E8D8CFE0916A0E8F
:1023600081E08E0F80936A0E8091BB00F0E0E75B06
:10237000F14F808380916C0E81115CCF81E080935E
:10238000470E84EA8093BC0010926D0E24CF85EC3A
:102390008093BC0010926D0E8091C60A803230F49A
:1023A000E091C60AF0E0EA55F54F10826091C60A46
:1023B00070E0E091220CF091230C86EA9AE01995E6
:1023C0001092C60A08CF10926B0E34CF8F929F9254
:1023D000AF92BF92CF92DF92EF92FF920F931F9333
:1023E000CF93DF938C01862F0B30110509F09FC02E
:1023F0009091DA12992309F0F89462E10E94D48551
:10240000EC018091DA12882309F07894209701F189
:1024100080E090ECA9E7B4EC8093CD129093CE12BB
:10242000A093CF12B093D0128093D1129093D21276
:10243000A093D312B093D412CE3F8FEFD80709F4F4
:10244000A9C0CF3FDC0709F462C0CCEFDFEF30C199
:10245000C091D512E090D6126E2D70E090E080E031
:102460000E944BB42DEC3CEC4CEC5DE30E94AAB412
:102470004B015C016C2F70E090E080E00E944BB457
:102480009B01AC01C501B4010E94F2B56093CD126D
:102490007093CE128093CF129093D012D091D71216
:1024A000F090D8126D2F6F7770E090E080E00E947E
:1024B0004BB44B015C016F2D70E090E080E00E9416
:1024C0004BB42DEC3CEC4CEC5DE30E94AAB49B01B8
:1024D000AC01C501B4010E94F2B5D7FD26C06093DE
:1024E000D1127093D2128093D3129093D412CE0D46
:1024F000CD0FCF0D81E090E02091D912C21302C020
:1025000090E080E0892B09F493C0CFEFDFEFCE019C
:10251000DF91CF911F910F91FF90EF90DF90CF90BF
:10252000BF90AF909F908F9008959058D8CFCFEFE5
:10253000DFEF0631110509F0BBC09091DA12992343
:1025400009F0F89461E00E94D485EC018091DA12E0
:10255000882309F07894209701F180E090ECA9E7B6
:10256000B4EC8093CD129093CE12A093CF12B0937F
:10257000D0128093D1129093D212A093D312B09321
:10258000D412CF3FDC0719F2209709F451C02296EC
:1025900009F05BCFCEEFDFEF8BC0C091D612D091A8
:1025A000D5126091D5127091D612762767277627BB
:1025B00090E080E00E9449B42DEC3CEC4CEC5DE3F3
:1025C0000E94AAB46093CD127093CE128093CF1262
:1025D0009093D012E090D812F090D7126F2D6F77B1
:1025E000762F6E2D90E080E00E9449B42DEC3CECFB
:1025F0004CEC5DE30E94AAB4F7FC18C06093D112C2
:102600007093D2128093D3129093D4128C2F8D0F8B
:102610008E0D8F0DC1E0D0E09091D912891302C0C8
:10262000D0E0C0E0D195C195D109ABCF9058E6CFAD
:10263000C090CD12D090CE12E090CF12F090D01278
:1026400020E030E048EC52E4C701B6010E9406B732
:10265000D0E0C0E0181614F4CBEFDFEF20E030E05C
:10266000A901C701B6010E9444B487FF02C0CAEFA6
:10267000DFEFC090D112D090D212E090D312F09040
:10268000D41220E030E048EC52ECC701B6010E94C1
:1026900044B487FF02C0C9EFDFEF20E030E040EF35
:1026A00052E4C701B6010E9406B718160CF483C0A5
:1026B0000C30110509F02BCF81E08093730E8CE56F
:1026C0008093950E1092740E1092960E60E082ED3B
:1026D0009FE00E94CE0B81E00E948A830E94180E28
:1026E0006B017C0180916D0E811168C081E0809347
:1026F0006D0E80936C0E9FEF90936B0E10926A0E8E
:1027000094E09093690E8093480E8091480E886BF8
:102710008093480E8091470E813009F028C11092B5
:10272000470E0E94180E6B017C018091480E809329
:10273000BB0080916F0E9091700EA091710EB091C0
:10274000720E892B8A2B8B2BA1F00E94180E009100
:102750006F0E1091700E2091710E3091720E6C19E7
:102760007D098E099F09061717072807390708F4FE
:1027700046C08091BC0083FDD8CF85EC8093BC001F
:102780000E94180E6B017C0180916D0E813009F45E
:10279000F0C080916A0E853008F00DC180916A0EFC
:1027A000A9E4BEE0E3E6FAE090E0981769F12D9124
:1027B00021939F5FFACFC8EFDFEF7ACF80916F0E42
:1027C0009091700EA091710EB091720E892B8A2B90
:1027D0008B2B09F487CF0E94180E00916F0E109179
:1027E000700E2091710E3091720E6C197D098E0958
:1027F0009F09061717072807390708F073CF80913C
:102800006E0E0E94691080E01092270C8093260CB7
:10281000082F10E0CEEFDFEF882309F478CECDEF5C
:10282000DFEF053011050CF472CEC6E4D9E082ED7D
:102830009FE00E94870B88872196CE01865499409D
:1028400080179107A4F3C0914E0900914F09602FA2
:1028500070E090E080E00E944BB42DEC3CEC4CEC3E
:102860005DE30E94AAB46B017C016C2F70E090E0E4
:1028700080E00E944BB49B01AC01C701B6010E94ED
:10288000F2B56B017C01C0924609D0924709E092F3
:102890004809F0924909D0915009109151096D2FC2
:1028A0006F7770E090E080E00E944BB44B015C01D8
:1028B000612F70E090E080E00E944BB42DEC3CEC86
:1028C0004CEC5DE30E94AAB49B01AC01C501B401CC
:1028D0000E94F2B5D7FD71C060934A0970934B090D
:1028E00080934C0990934D09C00FCD0FC10F80917B
:1028F0005209C8130ACE20E030E048EC52E4C70188
:10290000B6010E9406B7D0E0C0E0181614F4CBEF71
:10291000DFEF20E030E040EA50E4C701B6010E945A
:1029200044B487FF02C0CAEFDFEFC0904A09D090DD
:102930004B09E0904C09F0904D0920E030E040EF69
:1029400051ECC701B6010E9444B487FF02C0C9EF31
:10295000DFEF20E030E040EF52E4C701B6010E9413
:1029600006B718160CF0D3CDC8EFDFEFD0CD85EE4B
:1029700005CF80916F0E9091700EA091710EB09165
:10298000720E892B8A2B8B2B09F4FECE0E94180E17
:1029900000916F0E1091700E2091710E3091720E99
:1029A0006C197D098E099F09061717072807390733
:1029B00008F0EACE24CF85E0F3CE90588DCF61E0C9
:1029C000FC0184810C94B90DCF93DF93EC018FEF60
:1029D0008EBD2FEF8F819885AC014F5F5F4F588779
:1029E0004F838130924028F40DB407FEFDCF2EBDF9
:1029F000F1CF0DB407FEFDCFCE010E94DF141E8281
:102A0000DF91CF9108958EBD0DB407FEFDCF0895DF
:102A10008FEF0E9403158EB508958F929F92AF920B
:102A2000BF92FF920F931F93CF93DF93EC01F62E8B
:102A300049015A018E81882319F0CE010E94E414C5
:102A400060E08C810E94B90D8CE291E00E945F866B
:102A50008F2D80640E94031508E110E0D501C401A8
:102A6000002E04C0B695A795979587950A94D2F73E
:102A70000E94031508501109083F8FEF180771F7DE
:102A800085E9FF2021F088E0F8120DC087E80E9458
:102A9000031510E00E9408158A8787FF06C01F3FB4
:102AA00021F01F5FF7CF8FEFF2CFDF91CF911F9112
:102AB0000F91FF90BF90AF909F908F900895AF922D
:102AC000BF92CF92DF92EF92FF920F931F93CF931B
:102AD000DF93EC016901C801820F931F813092409E
:102AE00050F58E81882379F088819981AA81BB81F4
:102AF00084179507A607B70731F48F819885C81604
:102B0000D90608F042C0488359836A837B838B854A
:102B1000833039F089E0440F551F661F771F8A956F
:102B2000D1F79A01AB0161E1CE010E940D15882316
:102B300089F083E08D83CE010E94DF1480E0DF9175
:102B4000CF911F910F91FF90EF90DF90CF90BF90AA
:102B5000AF9008950E94700E5B010E9408158A874D
:102B60008F3F69F40E94700E6A197B096D327140C3
:102B7000A0F38FE08D83CE010E94DF14DCCF8E3F67
:102B8000B1F418861F8281E08E838FEF8EBD2FEF08
:102B90008F8198858C159D0560F40DB407FEFDCFDF
:102BA0002EBD8F819885019698878F83F1CF8DE018
:102BB000E1CFC8010197F7012FEFAF014E195F096F
:102BC0004817590738F40DB407FEFDCF3EB53193D1
:102BD0002EBDF3CF0DB407FEFDCF2EB5E80EF91EC6
:102BE000F70120838F819885080F191F18870F839D
:102BF0008985882319F00115124030F08E818823D1
:102C000019F0CE010E94E41481E099CF0F931F9335
:102C1000CF93DF93EC01890182E1411551056105F4
:102C2000710599F08B85833039F089E0440F551F89
:102C3000661F771F8A95D1F79A01AB0168E1CE0133
:102C40000E940D15882319F084E08D8338C08EEF23
:102C50008EBDF801C8019E5F0DB407FEFDCF208137
:102C60002EBD0DB407FEFDCF21812EBD3296E81793
:102C7000F90791F70DB407FEFDCF8FEF0E94031502
:102C80008FEF0E9403150E9408158A878F71853087
:102C900089F488E592E00E945F868823A9F020E00D
:102CA00030E0A9016DE0CE010E940D15882371F07E
:102CB00084E1CBCF81E18D83CE010E94DF14CE0170
:102CC0000E94DF1480E00AC085E1BFCF0E94081592
:102CD0008111EECFCE010E94DF1481E0DF91CF9110
:102CE0001F910F91089580915E0A8823A9F1409168
:102CF00048025091490260914A0270914B0223E4CC
:102D00003CE08091280C9091290C0E9406168111BC
:102D100002C080E0089540915F0A5091600A60917E
:102D2000610A7091620A411551056105710591F0C2
:102D300023E43CE08091280C9091290C0E94061617
:102D4000882339F310925F0A1092600A1092610A88
:102D50001092620A10925E0A81E008958F929F920B
:102D6000AF92BF92EF92FF920F931F93CF934B01BD
:102D70005C01C42F8091480290914902A0914A02BF
:102D8000B0914B0288159905AA05BB0549F10E942F
:102D9000731681110BC080E0CF911F910F91FF90AE
:102DA000EF90BF90AF909F908F90089583E4E82EAE
:102DB0008CE0F82E00E012E030E020E0B501A40144
:102DC0008091280C9091290C0E945F15882319F39B
:102DD0008092480290924902A0924A02B0924B021D
:102DE00040915E0A4C2B40935E0A81E0D5CF4F9212
:102DF0005F926F927F928F929F92AF92BF92CF928B
:102E0000DF92EF92FF920F931F93CF93DF93EC012A
:102E1000423051056105710590F480E0DF91CF915A
:102E20001F910F91FF90EF90DF90CF90BF90AF90E8
:102E30009F908F907F906F905F904F9008958985BD
:102E40009A85AB85BC850196A11DB11D8417950798
:102E5000A607B70710F3CB88DC88ED88FE888F893A
:102E6000803109F042C0BB27A72F962F852F48013C
:102E700059012A013B01C80ED91EEA1EFB1E809192
:102E8000480290914902A0914A02B0914B02C816A3
:102E9000D906EA06FB0699F58F898031C1F5B301A1
:102EA000A201552766277727440F551F4D5B534FC7
:102EB000FA019182808280915E0A816080935E0A2D
:102EC0008A89823080F08D819E81AF81B8858C0D9A
:102ED0009D1DAE1DBF1D80935F0A9093600AA09355
:102EE000610AB093620A81E099CFDB01CA01E7E091
:102EF000B695A79597958795EA95D1F7B8CF40E015
:102F0000C701B6010E94AE168111C6CF86CFB301AC
:102F1000A2014F77552766277727440F551F440F87
:102F2000551F4D5B534FFA0180829182A282B3827A
:102F3000C2CF8F929F92AF92BF92CF92DF92EF92C9
:102F4000FF920F931F93CF93DF93FC0181859285AE
:102F5000A385B4850196A11DB11D84179507A60709
:102F6000B70770F480E0DF91CF911F910F91FF9030
:102F7000EF90DF90CF90BF90AF909F908F9008958B
:102F800083889488A588B6888789803189F5BB278E
:102F9000A72F962F852FE9016A017B018F01BC01C4
:102FA000CD01680D791D8A1D9B1D8090480290906F
:102FB0004902A0904A02B0904B0286169706A806D6
:102FC000B90601F5F8018789803111F5DD24EE2479
:102FD000FF24F601EE0FFF1FED5BF34F808191811F
:102FE000B0E0A0E088839983AA83BB8381E0BBCF54
:102FF000DB01CA01C7E0B695A79597958795CA9555
:10300000D1F7C9CF40E00E94AE168111DBCFAACF25
:10301000E894C7F8DD24EE24FF24F601EE0FFF1F2D
:10302000EE0FFF1FED5BF34F80819181A281B38191
:10303000BF70D8CF4F925F926F927F92AF92BF9244
:10304000CF92DF92EF92FF920F931F93CF93DF9374
:1030500000D01F92CDB7DEB78C0149835A836B83B2
:103060007C835901C12CD12C7601412C82E0582E51
:10307000612C712C49815A816B817C819E012F5F6B
:103080003F4FC8010E949917882339F1F8018585BF
:10309000A301920104C0220F331F441F551F8A95BC
:1030A000D2F7DA01C901C80ED91EEA1EFB1E4981FA
:1030B0005A816B817C818789803111F188EF9FEF84
:1030C000AFEFBFE0481759076A077B0798F2F50191
:1030D000C082D182E282F38281E00F900F900F9044
:1030E0000F90DF91CF911F910F91FF90EF90DF90A4
:1030F000CF90BF90AF907F906F905F904F9008956A
:1031000088EF9FEFA0E0B0E0DDCFCF92DF92EF92AB
:10311000FF921F93CF93DF93EC0180E2689FF00151
:103120001124ED5BF34F9385917161F0842F8274CC
:1031300049F080E0DF91CF911F91FF90EF90DF90F9
:10314000CF900895142F6A8B809148029091490284
:10315000A0914A02B0914B028E879F87A88BB98BB2
:10316000C488D588F12CE12C7601DD24CC24CF8ACB
:10317000D88EE98EFA8E828D938DB0E0A0E0AC01FE
:10318000BD014C295D296E297F294F8B588F698F8E
:103190007A8F83858871B1F4848D958DA68DB78DD6
:1031A0008B8B9C8BAD8BBE8B81E08D831F701C83C2
:1031B0001E821F82188619861A861B861C861D860B
:1031C00081E0B8CF803109F0B4CF9E012D5E3F4F32
:1031D0008B8D9C8D0E941A18882309F4AACF84E055
:1031E000E4CF8F929F92AF92BF92CF92DF92EF92F5
:1031F000FF920F931F93CF93DF93EC018D81811189
:103200000EC080E0DF91CF911F910F91FF90EF9062
:10321000DF90CF90BF90AF909F908F9008950B89D3
:103220001C892D893E89041715072607370748F39F
:103230004A015B01823031F48A869B86AC86BD866A
:1032400081E0E0CF81149104A104B10449F41E820D
:103250001F82188619861A861B861C861D86F0CF4B
:103260000A851B852C853D85EB8DFC8D858590E041
:103270000996B901A8014150510961097109082E47
:1032800004C076956795579547950A94D2F77501CE
:103290006401E1E0CE1AD108E108F10804C0F69417
:1032A000E794D794C7948A95D2F7C416D506E60654
:1032B000F70620F0012B022B032B11F58F89988D37
:1032C000A98DBA8D8E839F83A887B9878E010A5FE7
:1032D0001F4FC114D104E104F10409F4ADCF4E81B4
:1032E0005F816885798598018B8D9C8D0E949917E7
:1032F00091E0C91AD108E108F1088111EACF81CF24
:10330000C41AD50AE60AF70AE1CF3F924F925F92BC
:103310006F927F928F929F92AF92BF92CF92DF92E5
:10332000EF92FF920F931F93CF93DF93CDB7DEB74A
:103330002C970FB6F894DEBF0FBECDBF5C01DC0149
:103340005B968D909C905C9716964D905D906D90DD
:103350007C901997411451046104710409F468C008
:10336000BFEF4B1A5B0A6B0A7B0A312CF401818593
:103370009285A385B4859C01AD012F5F3F4F4F4FD0
:103380005F4F29873A874B875C87730162011D82F3
:103390001E821F821886F40181859285A385B485DB
:1033A0002D813E814F815885281739074A075B07D1
:1033B00008F056C089859A85AB85BC858C159D051E
:1033C000AE05BF0550F482E0C82ED12CE12CF12CC3
:1033D00092E0492E512C612C712C9E012F5F3F4FA2
:1033E000B701A601C4010E9499178823C9F18981F8
:1033F0009A81AB81BC81892B8A2B8B2B09F1260109
:1034000037019FEF491A590A690A790A2D813E81CD
:103410004F8158852F5F3F4F4F4F5F4F2D833E8326
:103420004F8358873FEFC31AD30AE30AF30AB3CF97
:10343000F40140805180628073803324339496CFAE
:10344000C414D504E604F70409F70FEF1FEF2FEFBC
:103450003FE0B701A601C4010E94F716811119C00F
:1034600080E02C960FB6F894DEBF0FBECDBFDF9183
:10347000CF911F910F91FF90EF90DF90CF90BF9071
:10348000AF909F908F907F906F905F904F903F9004
:103490000895F50146815781608571854115510573
:1034A0006105710539F097018601C4010E94F71684
:1034B0008823B1F2D5011696CD92DD92ED92FC9261
:1034C0001997332051F0D701C6010196A11DB11DF6
:1034D000F40180839183A283B383F5018789908D62
:1034E000A18DB28D892B8A2B8B2B39F4C78AD08E74
:1034F000E18EF28E84818068848381E0B2CF2F9246
:103500003F924F925F926F927F928F929F92AF9273
:10351000BF92CF92DF92EF92FF920F931F93CF93C0
:10352000DF93EC015B012A018D81811115C08FEFC2
:103530009FEFDF91CF911F910F91FF90EF90DF9060
:10354000CF90BF90AF909F908F907F906F905F9043
:103550004F903F902F9008958C8180FFE8CF0B898A
:103560001C892D893E894A855B856C857D85C201D4
:10357000B0E0A0E068017901C41AD50AE60AF70AAA
:10358000C816D906EA06FB0618F42801441A550A9B
:1035900042011E0126E0220E311C8114910409F41F
:1035A000B3C04A855B856C857D856A0181E0D82240
:1035B0008B8D9C8D8A019B01E9E0369527951795A7
:1035C0000795EA95D1F7ED81E230E1F5FC01628DD6
:1035D000738D848D958D600F711F821F931F612CD9
:1035E00022E0722E6C187D088614970408F43401CA
:1035F0002C8126FD04C06114F2E07F0671F4009175
:1036000048021091490220914A0230914B0206175C
:1036100017072807390709F053C040E00E94AE168B
:10362000882309F484CFC6018D5B934FD5019C019B
:10363000260D371DFC012E173F0709F460C041918C
:103640004D93F9CFFC0174807A947022C114D10497
:1036500071F471100CC0452B462B472B39F58F891F
:10366000988DA98DBA8D8E839F83A887B987EB8D9E
:10367000FC8D6E817F8188859985625071098109F1
:103680009109258504C0660F771F881F991F2A9509
:10369000D2F70685178520893189600F711F821F37
:1036A000931F670D711D811D911D99CF4E815F8103
:1036B0006885798591010E9499178111D8CF37CFFC
:1036C000750183019601AB01BC018091280C90919A
:1036D000290C0E945F15882309F429CFA60CB71C7A
:1036E0008A859B85AC85BD85860D971DA11DB11D65
:1036F0008A879B87AC87BD87861897084ECF281B83
:10370000390BA20EB31EECCFC20113CFCF93DF93C0
:103710001F92CDB7DEB741E050E0BE016F5F7F4F33
:103720000E947F1A019731F4898190E00F90DF9118
:10373000CF9108958FEF9FEFF9CFFC01818D928D8E
:10374000009711F00C94861B8FEF9FEF08950F9355
:103750001F93CF93DF93EC01898D9A8D10E000E0E9
:10376000009799F00E94861B8C010F3F100769F0AB
:10377000898D9A8DFC0142855385648575854150FC
:103780005109610971090E94F118C801DF91CF91B7
:103790001F910F910895CF93DF93EC018D818823C2
:1037A00029F18C8187FF1EC0CE010E947A86FC0120
:1037B000892BE1F08D81823040F48B899C89AD8921
:1037C000BE89848F958FA68FB78F8F89988D938FA1
:1037D000828F8F89988DA98DBA8DB58BA48B8C81A2
:1037E0008F778C83DF91CF910C94731680E0DF91FB
:1037F000CF910895CF93DF93EC010E94CB1B8823D8
:1038000011F01D8281E0DF91CF910895FC01818D3F
:10381000928D009711F00C94CB1B08953F924F921C
:103820005F926F927F928F929F92AF92BF92CF9250
:10383000DF92EF92FF920F931F93CF93DF9300D00D
:1038400000D000D01F921F92CDB7DEB77C01DC0103
:1038500015968C91811115C0FE013196CE010C9602
:103860006F0130E23193E817F907E1F7DA0130E050
:1038700087E09D91B92E992329F19E3239F48A303F
:1038800011F480E0D9C038E08AE0F3CFEBE9FDE045
:103890004491442321F031969413FACFF2CF831749
:1038A00080F34FED490F4E3560F74FE9490F4A312C
:1038B00018F440EEB42EB90EF601E30FF11DB082FC
:1038C0003F5FD7CF89818032E1F2322E8B01FB013D
:1038D000838D948DD7015C969C938E935B97168213
:1038E0001782108611861286138614861586F801B3
:1038F00082859385A485B5854389548965897689B0
:1039000084179507A607B70708F04DC025E0B695C0
:10391000A795979587952A95D1F7F82FFF70AF2E29
:10392000D80115968C91823008F4ABCFC8010E9463
:10393000861B97FDA6CFF80182859385A485B58562
:103940004F96A11DB11D82879387A487B587F0E2AA
:10395000AF9EB00111246D5B734F6115710509F4C1
:1039600090CFDB018C91882341F0853E09F057C050
:10397000BB2029F0BB24B394BACFB1100EC0F7011D
:10398000A28A8091480290914902A0914A02B09186
:103990004B0286879787A08BB18BDB018C918111BD
:1039A000E9CFBB24B394832D8271823109F069CFB2
:1039B000BB2009F459C0C7010E947A86009709F418
:1039C00060CF20E2FC0111922A95E9F72BE0F60185
:1039D000DC0101900D922A95E1F721E238E2DC0149
:1039E00051963C932E93509740E058E01F965C937D
:1039F0004E931E9753963C932E93529759963C9311
:103A00002E93589757965C934E9356970E94731631
:103A1000882309F436CF432DF70162890AC04BE0B1
:103A200050E0C6010E945AB9892B09F060CF432D9E
:103A30006A2DC7010E9485182B960FB6F894DEBF39
:103A40000FBECDBFDF91CF911F910F91FF90EF90EF
:103A5000DF90CF90BF90AF909F908F907F906F90AE
:103A60005F904F903F900895F8018581823009F46E
:103A700008CFC8010E948519882309F402CFD80114
:103A80005B96ED91FC915C9716968D909D90AD9014
:103A9000BC901997B2E08B1A9108A108B1088585EE
:103AA00004C0880C991CAA1CBB1C8A95D2F7868579
:103AB0009785A089B189880E991EAA1EBB1E848194
:103AC00024013501480E511C611C711C841495049D
:103AD000A604B70401F1E1E04E1A5108610871082B
:103AE0000E947316882309F4CCCEE3E4FCE0119223
:103AF00083E49EE08E179F07D1F7409248025092D0
:103B0000490260924A0270924B0280915E0A816083
:103B100080935E0ADBCFD8015B96ED91FC91258501
:103B200080E092E0A0E0B0E004C0880F991FAA1FD7
:103B3000BB1F2A95D2F7F801438954896589768994
:103B4000840F951FA61FB71F838B948BA58BB68BF5
:103B5000D70152961C9283E49CE033CF1F93CF93FE
:103B6000DF93CDB7DEB76D970FB6F894DEBF0FBE0B
:103B7000CDBFAB011C821B8222E933E03A8329834B
:103B80001E8221E0BC01CE0101960E940E1C11E0B4
:103B900081110CC010E0812F6D960FB6F894DEBF36
:103BA0000FBECDBFDF91CF911F910895CE01019639
:103BB0000E94FA1BF0CFCF93DF93CDB7DEB76D979E
:103BC0000FB6F894DEBF0FBECDBF442391F1AB0119
:103BD000BC011C821B8282E993E09A8389831E8246
:103BE00022E0CE0101960E940E1C81110EC090E0D1
:103BF00081E0911101C080E06D960FB6F894DEBFB0
:103C00000FBECDBFDF91CF910895CE0101960E94E6
:103C10009386882361F3CE0101960E947A860097ED
:103C200031F325EEFC0120831E820E947316982F2B
:103C3000DFCF81E0E1CF2F923F924F925F926F9260
:103C40007F928F929F92AF92BF92CF92DF92EF922C
:103C5000FF920F931F93CF93DF9300D01F92CDB7A6
:103C6000DEB78C015B011A01DC0115968C9115976A
:103C7000813009F0C8C014968C9181FFC4C082FDC8
:103C8000AEC06101D8011A964D915D916D917C9104
:103C90001D97C114D10409F429C15B968D919C91A3
:103CA0005C97FC0174802FEF270D2A013B0139E05E
:103CB00076946794579447943A95D1F7722E74206E
:103CC0007A01F1E0FF22711020C0E114F104E9F45F
:103CD00016964D915D916D917C9119974115510505
:103CE0006105710509F098C057968D919D910D90D1
:103CF000BC91A02D0097A105B10509F0AFC0C80186
:103D00000E948519882309F47EC080E092E08E1914
:103D10009F0946018C159D0508F44C01D8015B965E
:103D20004D915C915C9716968D919D910D90BC91F3
:103D3000A02D0297A109B109FA01258504C0880FB9
:103D4000991FAA1FBB1F2A95D2F746855785608900
:103D50007189840F951FA61FB71F9C01AD01270D08
:103D6000311D411D511D29013A01811432E0930694
:103D700009F07AC08091480290914902A0914A02CC
:103D8000B0914B0284159505A605B70559F48FEF40
:103D90009FEFDC018093480290934902A0934A026E
:103DA000B0934B029501B301A2018091280C909130
:103DB000290C0E940616882331F19EEFB91AC81803
:103DC000D908F80182859385A485B585880D991D4C
:103DD000A11DB11D82879387A487B58753CFF801B2
:103DE000438954896589768982859385A485B585BB
:103DF000481759076A077B0709F443CFC8010E9497
:103E0000F11881113ECF81E090E0D80113969C9388
:103E10008E93129780E007C09E012F5F3F4F0E9454
:103E20009917811102C090E077C089819A81AB8196
:103E3000BC81F801238D348DF901278948EF5FEFAC
:103E400060E070E0203121F048EF5FEF6FEF7FE03E
:103E500084179507A607B70708F051CFF8018683A6
:103E60009783A087B18751CFE114F10491F5D80170
:103E70001A964D915D916D917C911D9753968D9100
:103E80009D910D90BC91A02D481759076A077B079B
:103E900000F10E947316882309F4B5CF40924802BE
:103EA0005092490260924A0270924B0280915E0ADF
:103EB000816080935E0A97012D5B334FD501C90164
:103EC000880D991DF9018E179F0759F04D91419367
:103ED000FACF41E0C301B2010E94AE168111EBCFCF
:103EE00092CF821B930BA80EB91E69CFF80183896C
:103EF0009489A589B68984179507A607B70738F46A
:103F00008481438B548B658B768B80688483F80126
:103F1000848183FD18C0C1010F900F900F900F9006
:103F2000DF91CF911F910F91FF90EF90DF90CF9095
:103F3000BF90AF909F908F907F906F905F904F90C9
:103F40003F902F900895C8010E94CB1B882309F44D
:103F50005ACFE1CFCF93DF931F92CDB7DEB76983FE
:103F600041E050E0BE016F5F7F4F0E941B1E0F902B
:103F7000DF91CF910895CF93DF93EC01E98DFA8D16
:103F8000309749F481E090E09B838A8390E080E061
:103F9000DF91CF91089513821282898D9A8D0E94AC
:103FA0001B1EE98DFA8D22813381232B59F7F0CF27
:103FB000FC01DB0112968D919C9113979383828370
:103FC00082E993E09183808314968C911497848383
:103FD00015968C911597858316964D915D916D91EF
:103FE0007C91199746835783608771871A964D9104
:103FF0005D916D917C911D9742875387648775878A
:104000001E964D915D916D917C9151974687578792
:10401000608B718B52968C915297828B53964D91F7
:104020005D916D917C915697438B548B658B768B0C
:1040300057964D915D916D917C915A97478B508F1A
:10404000618F728F5B968D919C91948F838F089571
:10405000DC015996ED91FC91309721F081E095813A
:10406000911101C080E00895CF93DF93EC01898D19
:104070009A8D009741F00E94FA1B898D9A8D0E94BB
:10408000E3B71A8E198EDF91CF910895EF92FF92C8
:104090000F931F93CF93DF93EC017B018A011B8267
:1040A0001A8288EE93E0A0E0B0E08C839D83AE831B
:1040B000BF8382E194E0998388838DE190E00E9440
:1040C00047B79A8F898F009779F02DE1F701DC01CE
:1040D00001900D922A95E1F74CE050E0B801CE0135
:1040E0000C960E94B2B9188EDF91CF911F910F915B
:1040F000FF90EF900895E0912C0CF0912D0C8081B1
:1041000090912B0C892B80830895AF92BF92CF9210
:10411000DF92EF92FF920F931F93CF93DF9300D024
:104120001F92CDB7DEB78C016B017A0180912E0C06
:104130008333E9F45B016801C40ED51EC016D106B5
:10414000A9F10E944D0C8FE00E94580C812F0E9413
:10415000580C802F0E94580C0F5F1F4F80E00E9468
:10416000580CF50181935F010E947B20E7CF8433D7
:1041700069F50E944D0C19830A838F2D8F778B83ED
:10418000EC8264E070E0CE0101960E94330CA7013E
:1041900070E060E0C6010E9482B9E114F10421F0F0
:1041A000B701C6010E94330C0E947B20C7010F900B
:1041B0000F900F900F90DF91CF911F910F91FF9073
:1041C000EF90DF90CF90BF90AF9008950E944D0C7C
:1041D0000F3F110509F030F419820A831B8263E056
:1041E00070E0D1CF17FD0BC019820A8333E016951A
:1041F00007953A95E1F7007E08600B83F0CFC80180
:1042000026E0969587952A95E1F7807E19830A83A3
:104210000115104C18F480618B83E1CF8861FCCFCD
:10422000CF93DF931F92CDB7DEB720912F0C30E0F4
:10423000322F2227260F371F90E0982F882741E042
:1042400050E0BE016F5F7F4F820F931F0E94852059
:1042500089810F90DF91CF910895AF92BF92CF9255
:10426000DF92EF92FF920F931F93CF93DF9300D0D3
:1042700000D01F921F92CDB7DEB78C017B016A017F
:1042800080912E0C8333E1F45801A40EB51EA016C4
:10429000B10609F46FC00E944D0C80EF0E94580CCB
:1042A000812F0E94580C802F0E94580C0F5F1F4FC7
:1042B000F70181917F010E94580C0E947B20E7CF7B
:1042C0005B01A40EB51E8433C1F40E944D0C19830A
:1042D0000A838D2D80688B83CC8264E070E0CE01F0
:1042E00001960E94330CAE14BF0409F441C0F701DB
:1042F00081917F010E94580CF6CF0E944D0C0F3F18
:10430000110509F028F419820A8384E08B830CC01C
:1043100017FD17C019820A8333E0169507953A9561
:10432000E1F7007E0C600B8386E0C816D104A0F58F
:10433000F701DE011496EA15FB0599F081918D9342
:10434000FACFC80126E0969587952A95E1F7807EF9
:1043500019830A830115104C10F48461D7CF8C6146
:10436000D5CFB6016D5F7F4FCE0101960E94330C11
:104370000E947B20C60128960FB6F894DEBF0FBEC0
:10438000CDBFDF91CF911F910F91FF90EF90DF9004
:10439000CF90BF90AF90089563E070E0CE0101969A
:1043A0000E94330CF70181917F010E94580CAE14DA
:1043B000BF04C1F7DDCFCF93DF931F92CDB7DEB738
:1043C00041E050E0BE016F5F7F4F90E080E00E94CF
:1043D000852089810F90DF91CF910895CF93DF934E
:1043E000C4E1D0E00E94DB21882361F061E070E04D
:1043F00080E090E00E943D0E2197A1F780E0DF91E0
:10440000CF91089581E0FBCFCF93DF931F92CDB77B
:10441000DEB7898341E050E0BE016F5F7F4F90E0DF
:1044200080E00E942D210F90DF91CF91089563E0ED
:1044300070E00C941021DA01E0912F0CF0E0FE2FD7
:10444000EE27E60FF71F90E0982F8827A901BD01FE
:104450008E0F9F1F0C942D21CF93DF931F921F92DD
:10446000CDB7DEB779836A8322E030E0AE014F5FDB
:104470005F4F60E170E00E941B220F900F90DF9170
:10448000CF910895CF93DF931F921F92CDB7DEB7E0
:1044900079836A8322E030E0AE014F5F5F4F64E0D2
:1044A00070E00E941B220F900F90DF91CF91089532
:1044B000CF93DF931F92CDB7DEB720912F0C30E062
:1044C000322F2227260F371F90E0982F8827498305
:1044D00041E050E0BE016F5F7F4F820F931F0E944B
:1044E0002D210F90DF91CF910895CF93C82F462FA4
:1044F00061E070E00E94582261E070E08C2F0E9421
:1045000010218111F9CFCF910895DA01E0912F0C9C
:10451000F0E0FE2FEE27E60FF71F90E0982F882798
:10452000A901BD018E0F9F1F0C9485206F927F9271
:104530009F92AF92BF92CF92DF92EF92FF920F9332
:104540001F93CF93DF931F921F92CDB7DEB7982EA4
:104550008B013A01690122E030E0AE014F5F5F4F0D
:1045600064E270E00E948522E980FA80FE24EF2454
:10457000FE24E00EF11E9701377040912E0C092D9C
:1045800010E0C801433309F04CC00896982F8827E3
:10459000990F990F990F820F931F473309F446C063
:1045A000A9014C0D5D1D4130584008F43FC060E04A
:1045B00078E05B01A21AB30AA501B3010E942D2184
:1045C000A6014A195B09B3016A0D7B1D80912E0C6F
:1045D000833349F5085F1F4F000F000F000F80E085
:1045E000902F0E942D21EC0CFD1CF982EA8222E022
:1045F00030E0AE014F5F5F4F64E270E0892D0E94B2
:104600001B220F900F90DF91CF911F910F91FF9080
:10461000EF90DF90CF90BF90AF909F907F906F9082
:1046200008954096B3CF005F1F4FD6CFA601B301C8
:10463000D8CFEF92FF921F93CF93DF931F921F92D9
:10464000CDB7DEB7182F22E030E0AE014F5F5F4FED
:1046500060E270E00E948522E980FA80FE24EF2467
:10466000FE2422E030E0AE014F5F5F4F60E270E079
:10467000812F0E94852289819A81982789279827EE
:10468000E816F90689F487E0189FF0011124E65234
:10469000F44FF582E482C7010F900F90DF91CF9124
:1046A0001F91FF90EF9008957C01DBCFFF920F9355
:1046B0001F93CF93DF931F921F92CDB7DEB7F82ED3
:1046C00022E030E0AE014F5F5F4F66E270E00E9493
:1046D000852209811A8110270127102722E030E066
:1046E000AE014F5F5F4F66E270E08F2D0E94852222
:1046F00089819A819827892798270817190749F4EB
:10470000C8010F900F90DF91CF911F910F91FF90F3
:1047100008958C01E3CF44E050E0BC018FE090E0CD
:104720000C942D2108951F93CF93DF93182F80E5CC
:1047300091E00E948783812F0E941923EC01812F31
:104740000E941722873121F08C3111F0D0E0C0E0B7
:10475000CE01DF91CF911F910895FC0184858830AF
:1047600010F40C94932390E080E00895CF92DF92B0
:10477000EF92FF921F93CF93DF93182F7B01EA01F3
:104780004130584010F0C0E0D8E080E591E00E9450
:104790008783812F0E9419236C01812F0E94172289
:1047A000873111F08C3121F5CC16DD0670F380E5F0
:1047B00091E00E9487839E01A70170E060E0812F55
:1047C0000E94962260E270E0812F0E94752262E0D2
:1047D00070E0812F0E94102184FD0DC0812F0E9466
:1047E00017228823B9F080E591E00E948783EFCFFC
:1047F000D0E0C0E0DCCF40E162E070E0812F0E94B9
:104800005822CE01DF91CF911F91FF90EF90DF9062
:10481000CF900895D0E0C0E0F4CF0F931F93CF93D3
:10482000DF938C01EA01FC018485883048F40E9402
:10483000B623892B39F481E090E0F80193838283D9
:10484000D0E0C0E0CE01DF91CF911F910F9108958C
:10485000CF92DF92EF92FF920F931F93CF93DF934C
:104860008B017A016C0129EBC20ED11CF60140814B
:10487000EC012A96442349F050E0BC0167567F4F73
:10488000CE010E940D24F6011082A701B801CE01CD
:10489000DF91CF911F910F91FF90EF90DF90CF901C
:1048A0000C940D24CF93DF93EC01C754DF4FE881C4
:1048B00021E02E0F2883E80FF92FF11DE756FF4F57
:1048C0006083203249F4BC0167567F4F40E250E0DC
:1048D0000A960E940D24188281E090E0DF91CF912A
:1048E00008951F93CF93DF931F92CDB7DEB7182F94
:1048F00080E591E00E948783812F0E945F0C27E072
:10490000129FF0011124E652F44F22813381377057
:1049100041E050E0BE016F5F7F4F820F931F0E9406
:10492000852089810F90DF91CF911F910895FC011F
:10493000808D883040F4218D328D232B21F00E9410
:10494000712490E008958FEF9FEF0895CF93DF9348
:10495000FC012485283028F08FEF9FEFDF91CF9165
:104960000895EC010190F081E02D0084F185E02DA7
:104970001995892B89F38C850E94712490E0EECFE4
:104980001F93CF93DF93182F87E0189FE001112426
:10499000C652D44F88819981009761F480E591E0F7
:1049A0000E948783812F0E9456232E81821B9109AA
:1049B00099838883DF91CF911F910895FC018485AD
:1049C000883010F40C94C02490E080E008954F9259
:1049D0005F927F928F929F92AF92BF92CF92DF921F
:1049E000EF92FF920F931F93CF93DF931F921F922B
:1049F000CDB7DEB7782E6B014A01A82EB12C27E087
:104A0000829FC0011124FC01E652F44F7F01008116
:104A1000118180E591E00E9487830815190554F4FF
:104A2000872D0E945623F70126818C01021B110954
:104A3000118300830115110519F5872D0E94172296
:104A4000843159F0882349F001E010E08C3111F4F1
:104A500010E000E0119501951109C8010F900F9029
:104A6000DF91CF911F910F91FF90EF90DF90CF904A
:104A7000BF90AF909F908F907F905F904F900895E0
:104A8000801691060CF4840187E08A9DF0018B9DCD
:104A9000F00D1124E652F44FE280F380C114D104EA
:104AA00051F12701F7E05F22872D0E945F0C840DF2
:104AB000951D20912E0C273309F453C09801240D25
:104AC000351D2130384008F44CC020E038E0490161
:104AD00084189508A401B6010E9485202601480C7F
:104AE000591C6801C818D908872D0E945F0CA601BF
:104AF000B2010E948520E00EF11E87E08A9DF00140
:104B00008B9DF00D1124E652F44FF382E282208156
:104B10003181201B310B318320838681800F912FBF
:104B2000911D8A3F910510F4232BF1F487E08A9DB3
:104B3000F0018B9DF00D1124E652F44F1682F9829C
:104B4000EA8222E030E0AE014F5F5F4F68E270E042
:104B5000872D0E941B2260E470E0872D0E94752241
:104B60007CCFA801B601C5CF868377CFCF93DF93E3
:104B7000FC01218D328D2115310529F48FEF9FEF36
:104B8000DF91CF910895EC01808D4217530708F013
:104B9000A9010E94E7241816190684F7298D3A8D79
:104BA000281B390B3A8F298FEBCF0F931F93CF938D
:104BB000DF931F92CDB7DEB7FC01218D328D232B01
:104BC00041F48FEF9FEF0F90DF91CF911F910F91E5
:104BD00008958C0141E050E0BE016F5F7F4FFC0102
:104BE000808D0E94E724181619065CF7F801818D64
:104BF000928D0197928F818F898190E0E4CF0F93FE
:104C00001F93CF93DF9300D000D01F921F92CDB798
:104C1000DEB78C01D80159964D915C915A97411598
:104C2000510551F0ED91FC91048CF58DE02D70E073
:104C300060E0C8011995EECFF801808D0E94C02474
:104C4000892BB1F148E050E0BE016F5F7F4FD80182
:104C500058968C910E94E72418161906F4F4D8018E
:104C6000509684E0FE01319601900D928A95E1F70D
:104C70008D8190E0982F88272E81820F911DF80159
:104C8000958B848B8F81282F30E0322F22278885C7
:104C9000820F932F911D928F818F28960FB6F894D3
:104CA000DEBF0FBECDBFDF91CF911F910F91089551
:104CB00090E080E0F2CFCF93DF931F92CDB7DEB7C5
:104CC00041E050E0BE016F5F7F4FFC0184850E9490
:104CD000E7241816190634F4898190E00F90DF91CB
:104CE000CF9108958FEF9FEFF9CFFC018485883035
:104CF00010F40C94E72490E080E00895CF93C82F3F
:104D000080E591E00E94878368E070E08C2FCF916E
:104D10000C947522CF93C82F80E591E00E94878381
:104D200060E170E08C2FCF910C947522CF92DF92CE
:104D3000EF92FF920F931F93CF93DF9300D000D099
:104D4000CDB7DEB78C016B017A01FC01808D883014
:104D500010F40E948A2680E394E09A838983F60106
:104D600082819381A481B5818B839C83AD83BE8333
:104D7000B701CE0101960E94158AF801808F883014
:104D8000A0F4F586E486128E118E81E026960FB689
:104D9000F894DEBF0FBECDBFDF91CF911F910F9171
:104DA000FF90EF90DF90CF90089580E0EFCFCF930A
:104DB000DF93EC01888D883020F40E948A2688E0F9
:104DC000888FDF91CF910895CF93C82F80E591E030
:104DD0000E9487838C2FCF910C941722EF92FF9221
:104DE0000F931F93CF93DF937C0180912E0CD4E01F
:104DF000833309F0D8E002E11CE0C0E0F801219122
:104E000031918F01F701848195812817390729F0A5
:104E1000CF5FDC13F3CF80E006C08C2F0E94E42626
:104E20008431B1F781E0DF91CF911F910F91FF9015
:104E3000EF9008959F92AF92BF92CF92DF92EF9240
:104E4000FF920F931F93CF93DF93EC017B0180912F
:104E50002E0C811121C01B821A8288EE93E0A0E003
:104E6000B0E08C839D83AE83BF8384EE93E099830F
:104E7000888388E08C8788EE93E09E878D87CE01BB
:104E8000DF91CF911F910F91FF90EF90DF90CF9026
:104E9000BF90AF909F90089534E0932E833311F02C
:104EA00028E0922E82E1C82E8CE0D82E10E098E007
:104EB000B92EA12CD6012D913D916D01F701848170
:104EC00095812817390791F4812F0E94E426082F35
:104ED000873111F08C3139F5812F0E94C024892B44
:104EE00059F50C3119F4812F0E947E261F5F911213
:104EF000E1CFA11008C0D701ED91FC910084F185AC
:104F0000E02DC70119951B821A8288EE93E0A0E07C
:104F1000B0E08C839D83AE83BF8384EE93E099835E
:104F20008883BC86A8CF843149F08111DFCFF60198
:104F3000329711821082DACFB12ED8CFAA24A3944F
:104F4000D5CF8F929F92AF92BF92CF92DF92EF9286
:104F5000FF920F931F93CF93DF93CDB7DEB72F97B9
:104F60000FB6F894DEBF0FBECDBF5C014B017A01D6
:104F700080912E0C8823C9F104E0833309F008E006
:104F8000B501CE0101960E941A2782E1C82E8CE05D
:104F9000D82E10E0F601219131916F01F501848145
:104FA00095812817390751F4812F0E94E426873113
:104FB00029F4A701B401812F0E94B6231F5F0113BA
:104FC000E9CFC7012F960FB6F894DEBF0FBECDBF55
:104FD000DF91CF911F910F91FF90EF90DF90CF90D5
:104FE000BF90AF909F908F900895F12CE12CE9CF66
:104FF000CF93DF93EC018C858830D0F40E94E426B7
:10500000843189F0882379F0883169F021E08C318E
:1050100059F4E881F9810084F185E02DCE011995DC
:1050200021E0892B09F420E0822FDF91CF910895B0
:1050300080E0FBCFCF92DF92EF92FF92CF93DF938E
:10504000EC018C85883068F40E947E260E94700EE8
:105050006B017C018C850E94E426811109C088E0E7
:105060008C87DF91CF91FF90EF90DF90CF900895E4
:1050700061E070E080E090E00E943D0E0E94700EC2
:10508000AB01BC014C195D096E097F098D859E85B8
:10509000B0E0A0E0481759076A077B07D8F28C8573
:1050A0000E948A26DCCFCF93DF93EC018C85883079
:1050B00060F40E94E426873111F08C3131F48C8544
:1050C0000E9493238115984088F3DF91CF91089532
:1050D000CF92DF92EF92FF920F931F93CF93DF93C4
:1050E000CDB7DEB7AF970FB6F894DEBF0FBECDBF1A
:1050F0008C016B017A0180E394E09A8389831B829F
:105100001C821D821E821C861B8648EE53E060E0D6
:1051100070E04D875E876F87788B2AEB33E03A87A4
:105120002987988F8F8B198E1A8E1B8E1C8E28E0E4
:1051300029A39BA78AA71CA61DA61EA61FA6D80149
:105140001C968C91883060F40E94E426882321F01C
:10515000F80184850E947E2688E0D8011C968C93F5
:105160008091291090912A10A0912B10B0912C10B1
:105170008EA39FA3A8A7B9A78B839C83AD83BE836F
:1051800018861F82AE01465D5F4FB601CE010196C3
:105190000E9425870097C1F0D801ED91FC9106840B
:1051A000F785E02D80E394E09DA38CA38CA59DA5BD
:1051B000AEA5BFA58EA39FA3A8A7B9A7A701BE01AF
:1051C0006C5D7F4FC8011995AF960FB6F894DEBF9E
:1051D0000FBECDBFDF91CF911F910F91FF90EF9048
:1051E000DF90CF9008958F929F92AF92BF92CF920F
:1051F000DF92EF92FF920F931F93CF93DF9300D034
:1052000000D000D01F92CDB7DEB790912E0C911137
:1052100015C018E0812F2A960FB6F894DEBF0FBE96
:10522000CDBFDF91CF911F910F91FF90EF90DF9055
:10523000CF90BF90AF909F908F90089528E0F22E6E
:10524000933311F494E0F92E6B01082F80E591E07F
:105250000E9487839E012F5F3F4F5901490110E053
:10526000812F0E941722F40181934F018823C1F0FE
:105270001F5FF112F5CFF12CF50191915F019D3186
:1052800049F0983139F09A51923020F0F3941F117F
:10529000F3CFBFCF60E170E08F2D0E9475221F2DEC
:1052A000E12EF12CF701EE0FFF1FEE5EF34F11829E
:1052B000108283EE93E00197F1F7402F70E060E0F9
:1052C000812F0E9458224FEF62E070E0812F0E94F0
:1052D0005822B601CD2889F48091900290919102D4
:1052E00001968115F0EC9F0798F1909391028093BD
:1052F00090026091900270919102812F0E9442224F
:1053000061E070E0812F0E94752227E02E9DC00190
:105310002F9D900D11249C012652344F7901F901E3
:105320001182108222E030E0AE01475F5F4F68E2F9
:1053300070E0812F0E94852289859A859827892788
:105340009827F7019383828316821582148262CF95
:1053500080E090ECCACF0F931F93CF93DF93EC01C3
:105360008B01888D883010F40E948A26B80182E073
:105370000E94F328888F883050F41D870C871A8E7E
:10538000198E81E0DF91CF911F910F91089580E0F8
:10539000F9CF9F92AF92BF92CF92DF92EF92FF929E
:1053A0000F931F93CF93DF938C015B01942EE52E17
:1053B000FC01C688D788F08C80E591E00E94878345
:1053C0008F2D0E941923C92DDE2D8C179D0708F4FF
:1053D000EC019E01A501B6018F2D0E949622F801D5
:1053E000868997898C0F9D1F978B868BCE01DF91C5
:1053F000CF911F910F91FF90EF90DF90CF90BF90D2
:10540000AF909F900895CF93FC01C08D80E591E00F
:105410000E94878360E270E08C2F0E94752262E018
:1054200070E08C2F0E94102184FD16C062E070E0B5
:105430008C2F0E94102183FF0AC048E162E070E0D7
:105440008C2F0E94582280E090E0CF91089580E553
:1054500091E00E948783E3CF40E162E070E08C2F0F
:105460000E94582281E0F0CFFF920F931F93CF93B9
:10547000DF93EB01FC01178A168A2A81211109C0EA
:105480002B81211106C02C81211103C02D812223E3
:1054900001F141155105E9F08A01FC01F08C80E52C
:1054A00091E00E948783AE014E5F5F4F24E030E0C1
:1054B0006CE070E08F2D0E941B22B8018F2D0E949E
:1054C0002C2281E090E0DF91CF911F910F91FF900E
:1054D000089580E0F7CF7F928F929F92AF92BF9214
:1054E000CF92DF92EF92FF920F931F93CF93DF93B0
:1054F000CDB7DEB7A6970FB6F894DEBF0FBECDBF0F
:105500008C01762E942E852E20E2A22ECE010196BD
:105510007C01DC01EA2D1D92EA95E9F76801F3E4CC
:10552000CF0ED11C80E394E09AA389A38FEF8BA3C5
:105530008CA38DA38EA343E450E0BE016F5D7F4F2B
:10554000C6010E94342A019609F4BFC081E0898314
:105550008A8386E0B82EBB821C82D80114966D9196
:105560007D918D919C9117970E942CB76D837E83BE
:105570008F83988789869A8680E890E09C878B87BE
:105580004CE150E0B701C6010E94C929FE013796DF
:105590008AE1DF011D928A95E9F74801B8E08B0E98
:1055A000911CF401D70101900D92BA94E1F740E10A
:1055B00050E0B701C6010E94C929F7011192AA94CF
:1055C000E9F796E0A92EB12C40E250E0B701C60100
:1055D0000E94C929F1E0AF1AB108B1F783E68983C7
:1055E00092E89A8393E59B838C8385E38D8381E0A6
:1055F0008E837F829DE3988797E099878A8786E0EC
:10560000F401DE011B9601900D928A95E1F78CE082
:10561000898B8A8B62E374E0CE0143960E949DB928
:10562000D8011B966C91CE0149960E94038AF8011D
:105630006485CE014B960E94038AD8011D966C9119
:10564000CE014D960E94038A4EE150E0B701C6019B
:105650000E94C929B3E07B121EC082E3898384E0E3
:105660008A83F80196859B8397859C8390899D8387
:1056700091899E8396E39F838887828D8987838D16
:105680008A87848D8B87858D8C874CE050E0B701AD
:10569000C6010E94C92987E3898386E08A8391E055
:1056A0009B8393E09C838D838FE08E838AE38F833B
:1056B0008BE388878FEF898749E050E0B701C60107
:1056C0000E94C929C6010E94032AA6960FB6F89423
:1056D000DEBF0FBECDBFDF91CF911F910F91FF9025
:1056E000EF90DF90CF90BF90AF909F908F907F9082
:1056F00008950F931F93CF938C01FC0164817581F2
:1057000081E20E94F328C82F8830F8F480E591E008
:105710000E9487838C2F0E941722833131F08C2FB7
:10572000CF911F910F910C947E2662E070E08C2F38
:105730000E947522F80184819581EC2FF0E0EE0F34
:10574000FF1FEE5EF34F91838083CF911F910F91E6
:1057500008950F931F93CF93DF931F921F92CDB79E
:10576000DEB7FC0124852830E0F48C0180E591E06F
:105770000E94878322E030E0AE014F5F5F4F60E11F
:1057800070E0F80184850E94852289819A8198279A
:10579000892798270F900F90DF91CF911F910F913C
:1057A000089590E080E0F6CF0F931F93CF93DF939F
:1057B0001F921F92CDB7DEB7FC0124852830E0F49C
:1057C0008C0180E591E00E94878322E030E0AE0109
:1057D0004F5F5F4F64E070E0F80184850E9485228E
:1057E00089819A819827892798270F900F90DF91B8
:1057F000CF911F910F91089590E080E0F6CFCF9266
:10580000DF92EF92FF921F93CF93DF93EC017B0126
:105810006A018C85883048F40E94E426882319F0B8
:105820008C850E947E2688E08C87F7018281938197
:10583000A481B5810097A105B10551F490E080E005
:10584000DF91CF911F91FF90EF90DF90CF9008955F
:105850008F3F9F4FAF4FBF4F89F370E060E081E211
:105860000E94F328182F8C87883040F780E591E05C
:105870000E948783A7014E5F5F4F24E030E06CE019
:1058800070E0812F0E941B22B601812F0E942C22E2
:1058900064E070E0812F0E9475220E94700E6B01FF
:1058A0007C018C850E94E426873111F18C3101F155
:1058B000882321F20E94700EAB01BC014C195D09D6
:1058C0006E097F098D859E85B0E0A0E0841795075D
:1058D000A607B70738F061E070E080E090E00E9432
:1058E0003D0EDFCF8C850E948A2688E08C87A6CF6C
:1058F00081E090E0A5CFCF93DF93EC0180E394E0CB
:10590000998388831A821B821C821D8280E591E024
:105910000E948783BE016E5F7F4F44E050E08FE0BE
:1059200090E00E948520CE01DF91CF9108959F9253
:10593000AF92BF92CF92DF92EF92FF920F931F939D
:10594000CF93DF935C017B018B01D0E0C0E0F801D5
:1059500091908F016501CC0EDD1EC6010E9468B5D5
:10596000981621F0692DC6010E9470B52196C533A5
:10597000F1E0DF0761F7C701DF91CF911F910F9130
:10598000FF90EF90DF90CF90BF90AF909F900895E1
:1059900081E08093EF028091F002882341F088E05B
:1059A00080935C1360E081E593E10C94EB0E089525
:1059B0008091F0028823F9F08091EF028823D9F0DA
:1059C00081E00E947A848BE39FE10197F1F760E028
:1059D00080E00E948B8461EC76E081E593E10E9497
:1059E000ED8E61E080E00E948B8461EB76E081E5E2
:1059F00093E10C94ED8E08950F931F93CF93DF9353
:105A00002091F002222309F45CC02091EF022223AE
:105A100009F457C0EA018C016F3F7F4FF1F461E058
:105A200080E00E948B84B80181E593E10E94CD8ED5
:105A300060EA76E081E593E10E94ED8E61E0F80195
:105A400084810E948B84BE01DD0F880B990BDF914E
:105A5000CF911F910F910C943D0E0E94700EAB01DF
:105A6000BC018091530990915409A0915509B091BE
:105A700056098C599F4FAF4FBF4F84179507A60704
:105A8000B707F8F461E080E00E948B84B80181E5FB
:105A900093E10E94CD8E6FE876E081E593E10E946C
:105AA000ED8E61E0F80184810E948B840E94700E6B
:105AB0006093530970935409809355099093560944
:105AC000C2CFDF91CF911F910F910895CF93DF93B4
:105AD000FB0122813381DC0113963C932E931297B4
:105AE000448155816681778114964D935D936D93C2
:105AF0007C931797408551856285738518964D93E1
:105B00005D936D937C931B971C96EF012C969C01E3
:105B1000275E3F4F49914D93A217B307D9F7218DC7
:105B2000328DFC01328F218FDF91CF910895DF926A
:105B3000EF92FF920F931F93CF93DF93D82EC9E379
:105B4000DCE07E0101E010E0F7018081F2E0EF0E81
:105B5000F11C61E00E94E70D90E080E0013011054A
:105B600031F48091CC12881F8827881F90E0880F1D
:105B7000991FFC01E15CF34F6081F701329780814E
:105B80000E94B90D64EF71E080E090E00E943D0E4C
:105B90000F5F1F4F04301105B9F6DD2009F454C022
:105BA000EE24E394F12C81E0E816F10409F046C0FC
:105BB0008091CC128095881F8827881F90E08E01E5
:105BC000880F991FFC01E15CF34F608188810E947E
:105BD000B90D68EE73E080E090E00E943D0E91E028
:105BE000E916F10471F58091CC12881F8827881F6F
:105BF00090E02296880F991FFC01E15CF34F6081D1
:105C0000F80180810E94B90D68EE73E080E090E0B9
:105C10000E943D0EFFEFEF1AFF0A84E0E816F10440
:105C200011F668EE73E080E090E0DF91CF911F9174
:105C30000F91FF90EF90DF900C943D0E81E090E08B
:105C4000BECF90E080E0D5CFDF91CF911F910F9133
:105C5000FF90EF90DF9008950F931F93CF93DF9302
:105C60008C01EB01FE0164912196662349F0D80175
:105C7000ED91FC910190F081E02DC8011995F2CFD2
:105C8000DF91CF911F910F910895EF92FF920F93A3
:105C90001F93CF93DF93EC017B018A0164E374E0EF
:105CA0000E942C2E6DE174E0CE010E942C2E6EEE2F
:105CB00073E0CE010E942C2EB701CE010E94C58E4A
:105CC0006DE278E0CE010E94C58E0115110521F02C
:105CD000B801CE010E94C58E6DE278E0CE01DF9161
:105CE000CF911F910F91FF90EF900C94C58ECF93A1
:105CF000DF93EC0163ED73E00E942C2E6DE174E004
:105D0000CE010E942C2E65EA73E0CE01DF91CF9187
:105D10000C942C2ECF93DF93EC01FB012481358171
:105D20000E94CD8DCE01DF91CF910895EF92FF9229
:105D30000F931F93CF93DF9300D000D0CDB7DEB782
:105D40008C017B016DE574E00E94B88D8AE0E81655
:105D5000F1042CF466E176E0C8010E94938CB7014F
:105D6000CE0101960E94058BBE016F5F7F4FC80177
:105D70000E949D8CCE0101960E94198DC801269625
:105D80000FB6F894DEBF0FBECDBFDF91CF911F914C
:105D90000F91FF90EF900895CF92DF92EF92FF92D4
:105DA0000F931F93CF93DF93CDB7DEB7C455D109BF
:105DB0000FB6F894DEBF0FBECDBF65965FAF4EAF96
:105DC00065972091BF0B3091C00B2F5F3F4F3093F1
:105DD000C00B2093BF0B2091D90B2111C1C08B01A7
:105DE0006C0181E08093D90B1092C00B1092BF0B15
:105DF0006DE574E0CE01895B9F4F0E94B88D6DE523
:105E000074E0CE01835B9F4F0E94B88D50E040E06C
:105E100069E374E0C6010E94452E0130110509F0C6
:105E20008EC06DE574E082E691E10E94FB8A6DE52B
:105E300074E08EE391E10E94FB8A6596EEADFFADC2
:105E400065978081882309F474C000E210E09E0108
:105E50002F5F3F4F40E250E0BE016F5D7F4FCE01AC
:105E60008D5A9F4F0E94FC84049739F3BE016F5DE9
:105E70007F4FCE018F5B9F4F0E94B88DBE016F5B3D
:105E80007F4FCE01895B9F4F0E94E08CCE018F5BDC
:105E90009F4F0E94198DBE016F5F7F4FCE018F5BB8
:105EA0009F4F0E94B88DBE016F5B7F4FCE01835B19
:105EB0009F4F0E94E08CCE018F5B9F4F0E94198DF7
:105EC0002D968EAD9FAD2D970297029730F462E527
:105ED00074E08EE391E10E94FB8ABE01695B7F4F13
:105EE00082E691E10E949D8C63968EAD9FAD639793
:105EF000892B09F4A2CF6DEA75E0CE018F5B9F4F2D
:105F00000E94B88DBE01635B7F4FCE018F5B9F4FB8
:105F10000E94338C6AEA75E00E941D8CBC0182E607
:105F200091E10E949D8CCE018F5B9F4F0E94198D45
:105F300084CF62E671E18EE391E10E949D8C109224
:105F4000D90BCE01835B9F4F0E94198DCE01895BD7
:105F50009F4F0E94198D0FB6F894DEBF0FBECDBFC4
:105F6000CC5ADF4F0FB6F894DEBF0FBECDBFDF9126
:105F7000CF911F910F91FF90EF90DF90CF900895F8
:105F80000F931F93CF93DF9300D000D0CDB7DEB730
:105F90002091BC0B2223A9F08C0165E776E0CE01AD
:105FA00001960E94B88DB801CE0101960E94338CF3
:105FB000BC0185E39FE00E94DB8ECE0101960E942A
:105FC000198D26960FB6F894DEBF0FBECDBFDF91B8
:105FD000CF911F910F9108950F931F93CF93DF934C
:105FE000CDB7DEB72C970FB6F894DEBF0FBECDBF8E
:105FF0008C010E94970FBC01C8010E94962E0E943E
:106000008F0FBC01CE0107960E94962E6FE376E0BB
:10601000CE0101960E94B88DBE01695F7F4FCE010F
:1060200001960E94338CBC01C8010E949D8CCE0158
:1060300001960E94198DCE0107960E94198D6AEA79
:1060400075E0C8010E94938C0E94870FBC01CE01AD
:1060500001960E94962EBE016F5F7F4FC8010E947D
:106060009D8CCE0101960E94198D69E574E0C801EE
:106070000E94938C0E947F0FBC01CE0101960E946A
:10608000962EBE016F5F7F4FC8010E949D8CCE018E
:1060900001960E94198D69E574E0C8010E94938CF5
:1060A0000E94750FBC01CE0101960E94962EBE0182
:1060B0006F5F7F4FC8010E949D8CCE0101960E94A8
:1060C000198DC8012C960FB6F894DEBF0FBECDBF58
:1060D000DF91CF911F910F9108950F931F93CF934D
:1060E000DF93CDB7DEB72C970FB6F894DEBF0FBEA7
:1060F000CDBF8C010E94970FBC01C8010E94962E53
:106100000E948F0FBC01CE0107960E94962E6FE36E
:1061100076E0CE0101960E94B88DBE01695F7F4F87
:10612000CE0101960E94338CBC01C8010E949D8C57
:10613000CE0101960E94198DCE0107960E94198DFD
:106140000E942F0F0E94550A60919C0B70E0CE01B7
:1061500007960E94962E6FE376E0CE0101960E948C
:10616000B88DBE01695F7F4FCE0101960E94338CCE
:10617000BC01C8010E949D8CCE0101960E94198D20
:10618000CE0107960E94198D6AEA75E0C8010E9447
:10619000938C0E94870FBC01CE0101960E94962E1F
:1061A000BE016F5F7F4FC8010E949D8CCE0101969A
:1061B0000E94198D69E574E0C8010E94938C0E94C9
:1061C0007F0FBC01CE0101960E94962EBE016F5F2B
:1061D0007F4FC8010E949D8CCE0101960E94198DAF
:1061E00069E574E0C8010E94938C0E94750FBC01A0
:1061F000CE0101960E94962EBE016F5F7F4FC801AF
:106200000E949D8CCE0101960E94198DC8012C968A
:106210000FB6F894DEBF0FBECDBFDF91CF911F91B7
:106220000F910895CF92DF92EF92FF920F931F93F9
:10623000CF93DF9300D000D0CDB7DEB77C01FB0158
:10624000848195818A01081B190B101611069CF098
:10625000C7010E949D8DC70126960FB6F894DEBF38
:106260000FBECDBFDF91CF911F910F91FF90EF90A7
:10627000DF90CF900895CE0101960E94AF8DCC247F
:10628000C394D12C6AEA75E0CE0101960E94938CEA
:10629000FFEFCF1ADF0A0C151D05A4F7BE016F5FD3
:1062A0007F4FC7010E949D8DCE0101960E94198DDE
:1062B000D2CF0F931F93CF93DF9300D000D0CDB7F1
:1062C000DEB78C0180914D0A882329F0B80188E956
:1062D0009EE00E94DB8E6EE170E080E090E00E9424
:1062E0003D0EB80185E39FE00E94DB8E80912A0C71
:1062F000882311F16AE070E080E090E00E943D0E9A
:10630000B801CE0101960E94AF8DBE016F5F7F4F35
:1063100085E393E10E94CD8E6EE278E085E393E120
:106320000E94C58ECE0101960E94198D64E170E035
:1063300080E090E00E943D0E26960FB6F894DEBFF6
:106340000FBECDBFDF91CF911F910F9108950F9395
:106350001F93CF93DF9300D000D0CDB7DEB7FC0101
:1063600024813581232B49F18C0180914D0A8823AA
:1063700029F0BF0188E99EE00E94CD8E6EE170E0B9
:1063800080E090E00E943D0EB80185E39FE00E940E
:10639000CD8E80912A0C882381F0B801CE01019620
:1063A0000E94AF8DBE016F5F7F4F85E393E10E9436
:1063B000CD8ECE0101960E94198D26960FB6F894C7
:1063C000DEBF0FBECDBFDF91CF911F910F9108951A
:1063D0002F923F924F925F926F927F928F929F92F5
:1063E000AF92BF92CF92DF92EF92FF920F931F93E3
:1063F000CF93DF93CDB7DEB7C258D1090FB6F8946B
:10640000DEBF0FBECDBF6C015B0188EE482E83E07E
:10641000582E612C712C02E114E09BE5892E912C01
:106420008C0E9D1E8CE0880E911C1B019FEF291A7B
:10643000390AD6015996ED90FC90F701858182309A
:1064400008F493C082859385A485B5858F719927BB
:10645000AA27BB27892B8A2B8B2B09F086C040E209
:1064600050E0BE016F5F7F4FC7010E947F1A8032EC
:1064700009F07BC08981882309F477C0853E79F3D0
:106480008E3269F38C8583FDEACF22961FAE1EAE55
:10649000229782E993E09FAF8EAF24961FAE249798
:1064A000BE016F5F7F4FE0E080E04EE2DB019D9137
:1064B000BD019032A1F0883049F426E730E02C0F7E
:1064C0003D1F2E0F311DD9014C93EF5F26E730E0C1
:1064D0002C0F3D1F2E0F311DD9019C93EF5F8F5F55
:1064E0008B3021F786E790E08C0F9D1F8E0F911D5A
:1064F000FC011082D60159966D917C9121E0AE018C
:106500004A585F4FCE01CE960E940E1C882369F137
:10651000BE01625C7F4FCE0181960E94D81FAE0102
:106520004A585F4FBE016F5D7F4FCE01855A9F4F26
:106530000E944620CE01855A9F4F0E942820882322
:1065400009F4ACC0F12CFA141B042CF569E0CE015F
:1065500001960E94848DCE0101960E94A731CE0142
:1065600001960E94198DF394EECF6F961FAE1EAE6A
:106570006F97A3964CAE5DAE6EAE7FAEA3976D9651
:106580001FAF0EAF6D97E6961FAE1EAEE697A896AC
:106590001FAEA897CFCFB401CE0101960E94B88D4F
:1065A000CE0101960E94A731CE0101960E94198D5D
:1065B000E696EEADFFADE697309709F447C08581CA
:1065C000823008F443C066E874E0CE0101960E9470
:1065D000B88DCE0101960E945931CE0101960E94DC
:1065E000198D6F968EAD9FAD6F979C838B83A3960D
:1065F0008CAD9DADAEADBFADA3978D839E83AF83B4
:10660000B887A7968CAD9DADAEADBFADA797898776
:106610009A87AB87BC871A8309838DE0F401DE017A
:106620001D9601900D928A95E1F7E6968EAD9FAD8D
:10663000E6979B8F8A8FB101CE0101960E94E831C7
:10664000CE01855A9F4F0E943420F3CE6BE574E053
:10665000CE0101960E94B88DCE0101960E94A7310D
:10666000CE0101960E94198DE696EEADFFADE6973C
:1066700040E050E0BA01309721F0438954896589A0
:106680007689CE0101960E94318BCE0101960E943F
:106690005931CE0101960E94198DD2CFCE57DF4FCE
:1066A0000FB6F894DEBF0FBECDBFDF91CF911F9123
:1066B0000F91FF90EF90DF90CF90BF90AF909F90A1
:1066C0008F907F906F905F904F903F902F900895A4
:1066D000DF92EF92FF920F931F93CF93DF93CDB78B
:1066E000DEB762970FB6F894DEBF0FBECDBF8C0148
:1066F000109257096DE574E0CE010D960E94B88D99
:10670000FF24F39485E39FE00E94C77F20915709FF
:10671000181619067CF521112DC085E39FE00E9413
:10672000A57F8A3009F07EC089899A89892B09F46E
:1067300081C0F09257096EE574E0CE0101960E9487
:10674000B88DBE01635F7F4FCE0101960E94338CEE
:10675000BC01CE0107960E94AF8DCE0107960E9424
:10676000C02FCE0107960E94198DCE0101960E947E
:10677000198D60C0F12CE12CDD24D394222309F47F
:1067800060C089899A89019709F045C06DE175E07B
:10679000CE0107960E94B88DBE01695F7F4FCE0182
:1067A0000D960E94028CF12C811115C06EE674E0EA
:1067B000CE0101960E94B88DBE016F5F7F4FCE0162
:1067C0000D960E94028CFF24F3948111F12CCE01CE
:1067D00001960E94198DCE0107960E94198DFF2007
:1067E000A1F050E040E0BE01635F7F4FCE01019613
:1067F0000E948A2EBE016F5F7F4F85E091E10E946B
:10680000E08CCE0101960E94198D64E170E080E079
:1068100090E00E943D0EBE01635F7F4FC8010E9461
:106820009D8D8EC08D3009F47FCF682FCE010D96DF
:106830000E94708C6AE070E080E090E00E943D0E63
:1068400061CF88E99EE00E94C77F1816190614F5EB
:1068500088E99EE00E94A57F8A30A9F08D3099F0EA
:106860009091570991110FC0682FCE010D960E948B
:10687000708C8FEFE81AF80A65E070E080E090E035
:106880000E943D0EDECF89899A89892BA9F3D09287
:106890005709F2CF64E170E080E090E00E943D0E85
:1068A000EF2809F43FC089899A89892BD9F1809111
:1068B000BC0B882389F165E776E0CE0101960E9442
:1068C000B88DBE016F5F7F4FCE010D960E94028C86
:1068D000F82ECE0101960E94198DF1101DC067E6B9
:1068E00074E0CE0101960E94B88DCE0101960E94FF
:1068F000A731CE0101960E94198DBE01635F7F4FC3
:10690000CE0101960E94AF8DCE0101960E945931B1
:10691000CE0101960E94198D64E170E080E090E064
:106920000E943D0E89899A892091570921112BCF08
:10693000009709F028CF6DE574E0C8010E94B88D7A
:10694000CE010D960E94198DC80162960FB6F8947B
:10695000DEBF0FBECDBFDF91CF911F910F91FF9092
:10696000EF90DF9008950F931F93CF93DF93CDB7F0
:10697000DEB72C970FB6F894DEBF0FBECDBF2C89C3
:106980003D89FE017496A7E3BCE090E080E032967A
:106990002817390734F0408151814D935D9301965A
:1069A000F6CFCE5BDE4F88819981C254D140281743
:1069B00039070CF044C2DC01AA0FBB1FA95CB34F1E
:1069C000880F991FFC01EB5CF34F80819181019648
:1069D0008D939C938C8D9D8D9093400C80933F0C58
:1069E0008E8D9F8D9093420C8093410CAD968FAD10
:1069F000AD97BE0164597F4F8F3209F029C2CE0195
:106A000007960E94B88D60E774E0CE0101960E945F
:106A1000B88DBE01695F7F4FCE0101960E94338C15
:106A2000BC0189EF92E10E94C98CCE0101960E94BF
:106A3000198DCE0107960E94198D69EF72E1CE0182
:106A400001960E94AF8DCE0101960E945931CE0170
:106A500001960E94198D66E874E0CE0101960E94AD
:106A6000B88DBE016F5F7F4F89EF92E10E94E28B8C
:106A7000182FCE0101960E94198D4091FD12509160
:106A8000FE12112309F4EBC1BA016250710989EFBA
:106A900092E10E94D18B682FCE0101960E94848DD5
:106AA000BE016F5F7F4F8BED92E10E94E08CCE01C3
:106AB00001960E94198D68EC71E1CE0107960E9443
:106AC000B88D68E874E0CE0101960E94B88DBE01D1
:106AD000695F7F4FCE0101960E94338CBC0183EF2A
:106AE00092E10E94C98CCE0101960E94198DCE01BF
:106AF00007960E94198D24968FAD24971F928F932D
:106B000023968FAD23971F928F9322968FAD229756
:106B10001F928F9321968FAD21971F928F938EE8AE
:106B200094E09F938F938EE49AE09F938F930E94BB
:106B3000DBB9CE52DF4F88819981C25DD0409093FE
:106B4000470280934602BE016C527F4FCE010196F0
:106B50000E94B88DBE016F5F7F4FCE0107960E94E5
:106B6000AF8DCE0107960E94848CBC018DEE92E120
:106B70000E94C98CCE0107960E94198DCE01019604
:106B80000E94198DBE0161527F4FCE0101960E9475
:106B9000B88DBE016F5F7F4F87EE92E10E94E08C5F
:106BA000CE0101960E94198D4091EB125091EC128A
:106BB0004250510967EE72E1CE0101960E948A2E81
:106BC000CE0101960E94698B6C5960939702CE01A9
:106BD00001960E94198DCC5EDE4F688179818A8191
:106BE0009B81C451D1400E944BB40FB6F894DEBFD4
:106BF0000FBECDBF9B01AC010E940BB7882389F06B
:106C00008CE390E0A0E0B0E0CC5EDE4F8883998317
:106C1000AA83BB83C451D140CD5EDE4F1882C351DD
:106C2000D140CD5EDE4F8881C351D140882399F099
:106C3000CC5EDE4F88819981AA81BB81C451D1404D
:106C40008093720290937302A0937402B0937502C2
:106C500081E08093340CC85EDE4F688179818A813F
:106C60009B81C851D1409B01AC010E940BB7882386
:106C700061F080E090E0A0E7B2E4C85EDE4F888378
:106C80009983AA83BB83C851D140C45EDE4F68811B
:106C90007981CC51D140072E000C880B990B0E94B2
:106CA0004BB49B01AC010E940BB7882341F082E0FA
:106CB00090E0C45EDE4F99838883CC51D140CE5B97
:106CC000DE4F68817981C254D140072E000C880BB9
:106CD000990B0E944BB49B01AC010E940BB7882317
:106CE00041F083E090E0CE5BDE4F99838883C2540D
:106CF000D140C45CDE4F08811981CC53D140B8012A
:106D0000012E000C880B990B0E944BB49B01AC0127
:106D10000E940BB7811103C01016110644F080E5E4
:106D200090E0C45CDE4F99838883CC53D140C45C2F
:106D3000DE4F88819981CC53D14090933F0280935C
:106D40003E0288E2FE01E551FF4FA1E2BAE0019068
:106D50000D928A95E1F7CE5CDE4F88819981AA81F8
:106D6000BB81C253D1408093290290932A02A09301
:106D70002B02B0932C02CA5CDE4F88819981AA81D4
:106D8000BB81C653D1408093250290932602A093E5
:106D90002702B0932802C65CDE4F88819981CA53CE
:106DA000D14090934D0280934C02CC5BDE4F6881C2
:106DB0007981C454D140072E000C880B990B0E9496
:106DC0004BB49B01AC010E940BB7882341F088E3D0
:106DD00090E0CC5BDE4F99838883C454D140CC5B78
:106DE000DE4F88819981C454D140909345028093AD
:106DF000440210924D0AC053DF4F88819981C05DD3
:106E0000D04097FD03C081E080934D0A6091CA1283
:106E100070E090E080E00E9449B49B01AC010E94C8
:106E20000BB781111092CA122C960FB6F894DEBFE0
:106E30000FBECDBFDF91CF911F910F91089580912B
:106E40003B0C90913C0C90933E0C80933D0CC2CD3A
:106E5000CE0107960E94B88D65E774E0D6CD41500B
:106E6000510969EF72E1CE0101960E948A2EBE019E
:106E70006F5F7F4F8BED92E10E94E08CCE01019617
:106E80000E94198D69EF72E1CE0101960E94AF8DCB
:106E900066E874E0CE0101960E941D8CBC0189EF6A
:106EA00092E10E94C98C03CEDF92EF92FF920F9382
:106EB0001F93CF93DF93CDB7DEB762970FB6F894E9
:106EC000DEBF0FBECDBF2091F002222379F12091C9
:106ED000EF02222359F17A018C016F3F7F4FA1F518
:106EE00060E080E00E948B84D12CB80181E593E1C1
:106EF0000E94CD8E6EE776E081E593E10E94ED8EF3
:106F0000F801848160E08D0D0E948B840E94700ED8
:106F10006093430E7093440E8093450E9093460EFB
:106F2000B701FF0C880B990B0E943D0E62960FB6BD
:106F3000F894DEBF0FBECDBFDF91CF911F910F91AF
:106F4000FF90EF90DF90089560E080E00E948B84D6
:106F50000E94700E28EE33E040E050E00E948EB5B3
:106F6000CA01B90120E831E541E050E00E94B0B526
:106F7000AB01BC0120E0CE0101960E94578DBE01FD
:106F80006F5F7F4FCE0107960E94AF8D6DE077E077
:106F9000CE0107960E941D8CBC01CE010D960E9469
:106FA000AF8DCE0107960E94198DCE0101960E94E9
:106FB000198DBE01635F7F4F81E593E10E94CD8E05
:106FC000D98860E08D2D0E948B84CE010D960E94A1
:106FD000198D8BCFCF93DF9300D000D0CDB7DEB724
:106FE0000E94D82CCE0101960E94EC2F4AE050E07E
:106FF0006FEF7FEFCE0101960E945437CE010196CC
:107000000E94198D61E080E00E948B84CE01019680
:107010000E947B2C61E573E1CE0101960E94658E92
:107020006AE974E081E593E10E94C58E0E94700ECA
:107030006093C90B7093CA0B8093CB0B9093CC0BCE
:1070400026960FB6F894DEBF0FBECDBFDF91CF916D
:107050000895EF92FF920F931F93CF93DF9300D089
:107060001F92CDB7DEB78C017B01FB018485883090
:10707000A8F080E394E0F801918380831282138268
:1070800014821582C8010F900F900F900F90DF911E
:10709000CF911F910F91FF90EF90089580E591E0BF
:1070A0000E94878324E030E0AE014F5F5F4F6CE0C9
:1070B00070E0F70184850E948522BE016F5F7F4FDB
:1070C000C8010E94238FDECF3F924F925F926F9252
:1070D0007F928F929F92AF92BF92CF92DF92EF9268
:1070E000FF920F931F93CF93DF93CDB7DEB7EA974D
:1070F0000FB6F894DEBF0FBECDBF7C012A013B0165
:1071000069010E94700E4B015C0187010D5B1F4FEE
:10711000C8010E94FF25181619069CF00E94700EE7
:10712000681979098A099B0946165706680679067F
:1071300008F466C162E370E080E090E00E943D0EDA
:10714000E7CF42E250E0BE016F5F7F4FC8010E946F
:10715000B62589818230D1F0312C832DEA960FB685
:10716000F894DEBF0FBECDBFDF91CF911F910F917D
:10717000FF90EF90DF90CF90BF90AF909F908F9057
:107180007F906F905F904F903F900895F8018489B1
:1071900095898334910501F76D817E818F81988572
:1071A0000E942CB74B015C01F60180829182A28281
:1071B000B38246E050E0B701685F7F4FCE014D9645
:1071C0000E945AB9892B41F6F70180819181A281F1
:1071D000B38188169906AA06BB0608F4BDCF848140
:1071E0009581A681B78188159905AA05BB0508F484
:1071F000B3CF89899A89AB89BC8986879787A08B09
:10720000B18B4EEC50E070E060E0C8010E94B62502
:10721000312CC701829698AB8FA7F701B696FAABCF
:10722000E9AB08969CAB8BAB67019AE1C90ED11C08
:10723000BD96FEABEDABC701429698AF8FABFD9705
:10724000FAAFE9AF4701FEE18F0E911CF801818D85
:10725000928D181619060CF080CFC8010E94D52512
:107260008333910509F4B2C014F58130910509F416
:1072700064C044F4892B51F3C8010E94D525AC01A8
:10728000552775C08330910509F462C00697A1F7B0
:10729000C8010E94D525B82E44E050E0B401C801D1
:1072A0000E94B625EB2DE450FF0BAF0160C08A337E
:1072B000910509F45FC084F585339105B1F1C69756
:1072C000D9F6C8010E94D5255C01B601CE01899688
:1072D0000E94238F8BA59CA5ADA5BEA5892B8A2BCB
:1072E0008B2BB1F0EDA9FEA94080518062807380A4
:1072F000B601CE0183960E94238F8DA19EA1AFA1DE
:10730000B8A5A501481659066A067B0609F0B8CF4C
:1073100044E050E0B60118C08B33910509F440C039
:107320008F3F910509F492CFA7CFC8010E94D525C0
:10733000C8010E94D525382E89CFC8010E94D525C5
:1073400044E050E06FA978ADC8010E94B6257ECF19
:10735000C8010E94D525B82E44E050E069AD7AAD51
:10736000C8010E94B6258B2D8450990BAC0170E0AA
:1073700060E0EACFC8010E94D52544E050E069A949
:107380007AA9C8010E94B625F70166A177A180A558
:1073900091A50E942CB766A377A380A791A756CF8B
:1073A000C8010E94D52544E050E06BA97CA9C80122
:1073B0000E94B625F70162A573A584A595A50E9434
:1073C0002CB762A773A784A795A740CFC8010E94D6
:1073D000D52544E050E06FA578A9C8010E94B625E4
:1073E000F70162A173A184A195A10E942CB762A3A9
:1073F00073A384A395A366A777A780AB91AB26CF91
:1074000033243A94AACE2F923F924F925F926F927A
:107410007F928F929F92AF92BF92CF92DF92EF9224
:10742000FF920F931F93CF93DF9300D000D0CDB77F
:10743000DEB78C010E94AFAB2FEC37E040E050E0AC
:107440000E94B0B5DC01CB010196A11DB11DF80170
:1074500084839583A683B78380839183A283B38338
:107460005801F3E4AF0EB11CC5010E94D72664E4B5
:1074700070E0C5010E94AB29882309F445C10E9430
:10748000700E2B013C01480182E4880E911C48EEED
:10749000C42E43E0D42EE12CF12C52E0252E1E8286
:1074A0001D82D4018C918330B1F1811166C0F80145
:1074B00084819581A681B7810196A11DB11D848328
:1074C0009583A683B7830E94700E64197509860997
:1074D0009709A70196010E948EB5A90161E0C80134
:1074E0000E946B2A81E0D4018C938D819E8101974B
:1074F000C1F20E94700E6419750986099709D801B6
:10750000D6962D913D914D915C91D99726173707CD
:107510004807590720F6C5010E94D726F801848143
:107520009581A681B7810196A11DB11D84839583A4
:10753000A683B7830E94700EF801FE966083718364
:10754000828393838D819E8126960FB6F894DEBF49
:107550000FBECDBFDF91CF911F910F91FF90EF90A4
:10756000DF90CF90BF90AF909F908F907F906F9063
:107570005F904F903F902F9008958430F1F4F80180
:1075800084819581A681B7810196A11DB11D848357
:107590009583A683B7830E94700E641975098609C6
:1075A0009709A70196010E948EB5A90163E0C80161
:1075B0000E946B2AD4012C9298CF813051F5F801AA
:1075C00042AD53AD64AD75AD9E012F5F3F4FC80115
:1075D0000E946438382EF2E08F1390C089819A811E
:1075E000AB81BC81F80184839583A683B7830E9415
:1075F000700E6419750986099709A70196010E9402
:107600008EB5A90163E0C8010E946B2AD4013C92A7
:107610006CCF823009F069CFF80142AD53AD64AD53
:1076200075AD9E012F5F3F4FC8010E946438382E10
:10763000F5E08F135DC0E3E0D401EC93F80182A183
:1076400093A1A4A1B5A1892B8A2B8B2B41F484E8AB
:1076500093E0A0E0B0E082A393A3A4A3B5A3F801B4
:1076600086A197A1A0A5B1A5892B8A2B8B2B61F4AC
:1076700082A193A1A4A1B5A1B695A7959795879549
:1076800086A397A3A0A7B1A7F80182A593A5A4A557
:10769000B5A5892B8A2B8B2BA9F482A193A1A4A138
:1076A000B5A1AC01BD0123E0769567955795479547
:1076B0002A95D1F7841B950BA60BB70B82A793A72E
:1076C000A4A7B5A7F80186A197A1A0A5B1A586A7F3
:1076D00097A7A0ABB1AB82A593A5A4A5B5A582AB96
:1076E00093ABA4ABB5AB81E090E09E838D83FDCEE0
:1076F00096E0891303C0D4011C92F7CEBFEF3B1272
:10770000F4CEF4011082F1CE1E821D821BCF8F9227
:107710009F92AF92BF92EF92FF920F931F93CF93DE
:10772000DF9300D000D0CDB7DEB70091300C1091C0
:10773000310CF12CE12C0115110509F4DAC00E947D
:10774000700E4B015C0178012EE3E20EF11CF70193
:1077500080819181A281B381A5019401281B390BFD
:107760004A0B5B0BCA01B901683E33E07307810520
:107770009105A0F128EE33E040E050E00E948EB584
:10778000861A970AA80AB90AD7018D929D92AD92DE
:10779000BC921397F80186A597A5A0A9B1A94901A4
:1077A0005A01880C991CAA1CBB1C88159905AA05AE
:1077B000BB0508F0B0C016A617A610AA11AAF801BA
:1077C00082A993A9A4A9B5A988159905AA05BB05FD
:1077D00008F0AAC012AA13AA14AA15AAF80186A52D
:1077E00097A5A0A9B1A9892B8A2B8B2B09F0A5C03D
:1077F000EE5BFF4F8081833009F09FC084E080837F
:10780000C8010E94033A01967C01F80182A993A95C
:10781000A4A9B5A9892B8A2B8B2BA1F4EE5BFF4F72
:107820008081833011F081110DC01082F8013E96E5
:1078300084E1DF011D928A95E9F7C8010E94033AAD
:1078400003967C01B2E0EB16F10429F0E4E0EE16B9
:10785000F10409F04EC080E591E00E9487836091B9
:10786000300C7091310C625F7F4FCE0101960E9407
:10787000238FCE0103960E948B236091300C709170
:10788000310C6A5E7F4FCE0101960E94238F44E047
:1078900050E0BE016D5F7F4F81E090E00E942D219E
:1078A0006091300C7091310C6E5E7F4FCE0101966D
:1078B0000E94238F44E050E0BE016D5F7F4F85E062
:1078C00090E00E942D216091300C7091310C625E2D
:1078D0007F4FCE0101960E94238F8B819C81AD81C9
:1078E000BE818093291090932A10A0932B10B093FF
:1078F0002C10C70126960FB6F894DEBF0FBECDBF81
:10790000DF91CF911F910F91FF90EF90BF90AF90BB
:107910009F908F900895821B930BA40BB50B86A7A5
:1079200097A7A0ABB1AB4BCF821B930BA40BB50BAE
:1079300082AB93ABA4ABB5AB51CFF12CE12C65CFAF
:10794000EF92FF920F931F93CF93DF93CDB7DEB7E4
:10795000E8970FB6F894DEBF0FBECDBF6DE574E0BB
:10796000CE0187960E94B88D6DE574E0CE018D96AC
:107970000E94B88D82E0E82EF12C2496FFAEEEAE88
:10798000249786E0EBEFF2E0DE01D39601900D92B2
:107990008A95E1F786E0FE01F396DE01AC5BBF4F0E
:1079A00001900D928A95E1F701E010E02C961FAF4F
:1079B0000EAF2C972E961FAE1EAE2E9788E0E1E0FC
:1079C000F3E0DE01599601900D928A95E1F788E087
:1079D000FE017996DE01A25BBF4F01900D928A9560
:1079E000E1F788E1E9E0F3E0DE01119601900D9204
:1079F0008A95E1F788E1FE013196DE01AA5ABF4F70
:107A000001900D928A95E1F78091210390912203D4
:107A1000A0912303B0912403E2968CAF9DAFAEAF4B
:107A2000BFAFE2976EE974E0CE0187960E94FB8AB1
:107A300060E0CE0187960E94708C4BA55CA5BE01CC
:107A40006E587F4FCE0187960E94DD8967E977E007
:107A5000CE018D960E94A48C64E175E08BED92E1DD
:107A60000E94FB8A60E0CE018D960E94708C49A92D
:107A70005AA9BE0166567F4FCE018D960E94DD89C0
:107A80006DE574E0CE0187960E94FB8A6DE574E097
:107A9000CE018D960E94FB8AC250DF4F1982188258
:107AA000CE5FD04010924D0A8091460290914702DD
:107AB000C050DF4F99838883C050D14080E090E070
:107AC000A0E7B2E4CA5BDE4F88839983AA83BB83B5
:107AD000C654D140C65BDE4FF982E882CA54D14019
:107AE00080E090E0A0E2B2E4C45BDE4F888399833B
:107AF000AA83BB83CC54D14080E090E0A4E3B2E4FD
:107B0000C05BDE4F88839983AA83BB83C055D14075
:107B100084EB90E0CC5ADE4F99838883C455D140E2
:107B200088E790E0CA5ADE4F99838883C655D140D2
:107B30008CE291E0A0E0B0E0C85ADE4F88839983E0
:107B4000AA83BB83C855D140C45ADE4F198308832A
:107B5000CC55D140C25ADE4FF982E882CE55D14091
:107B600060E08DEE92E10E94708C60E087EE92E121
:107B70000E94708C4091F1125091F212BE016E5F22
:107B80007E4F8DEE92E10E94DD894091EB12509183
:107B9000EC12BE01635F7E4F87EE92E10E94DD89A9
:107BA00088E2E1E2FAE0DE01A75EBE4F01900D92AD
:107BB0008A95E1F78CE390E0A0E0B0E0CE5BDE4F89
:107BC00088839983AA83BB83C254D140CF5BDE4FA5
:107BD0001882C154D14084EE98E3AEE8B2E4C05AB2
:107BE000DE4F88839983AA83BB83C056D14084EE3D
:107BF00098E3AEE8B1E4CC59DE4F88839983AA8339
:107C0000BB83C456D140C859DE4F19830883C85678
:107C1000D14080E590E0C659DE4F99838883CA56EB
:107C2000D14083E090E0C059DE4F99838883C057EC
:107C3000D14088E390E0CE58DE4F99838883C257C5
:107C4000D140CC58DE4F1882C457D1408FEF9FEF00
:107C5000CB58DE4F99838883C557D14084EF91E09C
:107C60009093570280935602BE016E5B7F4F0E9435
:107C7000972C64EF71E080E090E00E943D0E60E898
:107C800077E0CE0181960E94A68DCE0181960E945A
:107C90005931CE0181960E94198DCE018D960E9498
:107CA000198DCE0187960E94198DE8960FB6F8942B
:107CB000DEBF0FBECDBFDF91CF911F910F91FF901F
:107CC000EF9008956F927F929F92AF92BF92CF9262
:107CD000DF92EF92FF920F931F93CF93DF93CDB775
:107CE000DEB7C351D1400FB6F894DEBF0FBECDBF93
:107CF0003C016B015A017E0181E8E80EF11C60EF46
:107D000071E1C7010E94B88D66E874E08E010F5FD3
:107D10001F4FC8010E94B88DB701C8010E94338C63
:107D2000BC01CE01885F9E4F0E94AF8DC8010E94AA
:107D3000198DC7010E94198DB301CE01825F9E4F3C
:107D40000E94B88D94E0C916D10409F07FC066EA9C
:107D500074E0CE01885F9E4F0E94938C9924939487
:107D600060E0CE01885F9E4F0E94708CC45FDE4F42
:107D700048815981CC50D140B701CE01885F9E4FD8
:107D80000E94DD898091BC0B8823B9F062EC74E01D
:107D9000C8010E94B88DC8010E94A731C8010E9485
:107DA000198DBE01685F7E4FC8010E94AF8DC8016A
:107DB0000E945931C8010E94198DE6E8F8E080EC74
:107DC000DF011D928A95E9F7992009F44DC0C25F41
:107DD000DE4F68817981CE50D140CF010E949DB99C
:107DE0006DE574E0CE01825F9E4F0E94FB8AA090F9
:107DF0003E02B0903F0281E08093D90B1092C00BFD
:107E00001092BF0BA5016EE47AE087E791E10E9432
:107E100068286C018FE1682E712C91E0C916D1049D
:107E200009F457C1A1E06A1A710809F4AAC16AE00D
:107E300070E080E090E00E943D0EA5016EE47AE0E3
:107E400087E791E10E9468286C01E7CF63EB74E05B
:107E5000C114D10411F066EA74E0CE01885F9E4F30
:107E60000E94938C912C7CCFD5018C9111969C9182
:107E7000C114D10491F49F938F931F921F928BEDA5
:107E800094E09F938F93FF93EF930E94DBB90FB61B
:107E9000F894DEBF0FBECDBFA3CF9F938F93DF9229
:107EA000CF92C15FDE4F8881CF50D1408F93C25FA8
:107EB000DE4F8881CE50D1408F9382ED94E09F9326
:107EC0008F93FF93EF930E94DBB9E1CF81E0809322
:107ED000320C41E066E878E0CE018F519F4F0E945E
:107EE0000092CE018F519F4F0E942820882309F4D1
:107EF000ACC060EC75E087E791E10E94118F6DE600
:107F000075E087E791E10E94118F6CE575E087E7E6
:107F100091E10E94ED8EC650DF4FE881F981CA5F82
:107F2000D04040E050E0BA01309721F043895489B5
:107F3000658976894C535F4F6F4F7F4F2AE087E703
:107F400091E10E94198E87E791E10E94AF8E87E749
:107F500091E10E94AF8E63E375E087E791E10E94B3
:107F6000118F6BEF74E087E791E10E94ED8E66E878
:107F700078E0CE018E5F9E4F0E94B88DBE016E5F8D
:107F80007E4FCE0184509F4F0E94AF8D6EEE74E005
:107F9000CE0184509F4F0E941D8CBC0187E791E168
:107FA0000E94DB8ECE0184509F4F0E94198DCE011E
:107FB0008E5F9E4F0E94198D64ED74E087E791E11A
:107FC0000E94118F87E791E10E94AF8E3801B12C9A
:107FD000A12CCE018F519F4F0E94FD0B892BB9F030
:107FE000CE018F519F4F0E949D1BF30181933F0152
:107FF000FFEFAF1ABF0A80E8A816B10451F740E8B6
:1080000050E0B80187E791E10E940D24DFCFA11471
:10801000B10431F0A501B80187E791E10E940D2478
:1080200087E791E10E94AF8E69EA74E087E791E10A
:108030000E94118F87E791E10E94AF8ECE018F5190
:108040009F4F0E9434201092320C61E070E080E07B
:1080500090E00E943D0E1092320C1092D90B62E318
:1080600070E080E090E00E943D0E87E791E10E9481
:108070001A2887E791E10E945328E6E8F8E080ECAF
:10808000DF011D928A95E9F780E6F70111928A9542
:10809000E9F7CE01825F9E4F0E94198DCE01885F65
:1080A0009E4F0E94198DC601CD5EDE4F0FB6F8942B
:1080B000DEBF0FBECDBFDF91CF911F910F91FF901B
:1080C000EF90DF90CF90BF90AF909F907F906F9098
:1080D0000895FF92EF9285E095E09F938F931F9311
:1080E0000F930E94DBB9B80187E791E10E94B38E3C
:1080F0008EE49AE09F938F9386E195E09F938F9310
:108100001F930F930E94DBB9B80187E791E10E94AA
:10811000B38E0FB6F894DEBF0FBECDBF9110D6CE92
:1081200066E674E087E791E10E94118F86E898E0A7
:10813000DC010D900020E9F7CD01875898409F930E
:108140008F9380EF94E09F938F931F930F930E94E0
:10815000DBB9B80187E791E10E94B38E66E878E069
:1081600087E791E10E94B38E62E574E087E791E1D1
:108170000E94118F0F900F900F900F900F900F9003
:1081800064CF66E474E0C8010E94A68DC8010E9415
:108190005931C8010E94198D1092320C1092D90BDE
:1081A00062ED75E0C8010E94A68DC8010E94A7314A
:1081B000C8010E94198D66E878E0C8010E94B88D58
:1081C000C8010E945931C8010E94198DD12CC12CBF
:1081D00046CFEF92FF920F931F93CF93DF93CDB7CC
:1081E000DEB768970FB6F894DEBF0FBECDBF81E053
:1081F0008093D90B0E94873B8C0160ED77E080E093
:1082000090E00E943D0E8BE0E82EF12C0D7F0130B6
:10821000110571F481E0E81AF10851F00E94873BE2
:108220008C0160ED77E080E090E00E943D0EEECFA3
:108230000E942F8F7C0168EE73E080E090E00E9446
:108240003D0E0BE010E0EF2899F40150110981F088
:1082500060ED77E080E090E00E943D0E0E942F8F5D
:108260007C0168EE73E080E090E00E943D0EEBCF71
:1082700081E390E10E94792B1092D90B0E94EA379A
:108280006DE574E082E391E10E94FB8A66E077E0AD
:10829000CE010D960E94A68DCE0143960E947B2CA6
:1082A000888D1F928F938F891F928F938E891F9233
:1082B0008F938D891F928F938EE894E09F938F9375
:1082C0008CE899E09F938F930E94DBB96CE879E08A
:1082D000CE0101960E94B88DBE016F5F7F4F82E391
:1082E00091E10E94E08CCE0101960E94198D62E31B
:1082F00071E1CE0101960E94AF8DAE014F5F5F4FDD
:1083000063E070E080E092E00E94623E8C01CE016A
:1083100001960E94198D0FB6F894DEBF0FBECDBF37
:108320000130110579F5BE01635F7F4FCE010196E3
:108330000E94AF8D62E371E1CE0101960E94338C01
:10834000BC01CE0107960E94AF8DCE0107960E9418
:108350005931CE0107960E94198DCE0101960E94D7
:10836000198DCE010D960E94198D68960FB6F8945E
:10837000DEBF0FBECDBFDF91CF911F910F91FF9058
:10838000EF9008956CEF76E0CE0101960E94A68DE5
:10839000CE0101960E94A731CE0101960E94198D4F
:1083A000BE01635F7F4FCE0101960E94AF8DCE016B
:1083B00001960E94A731CE0101960E94198D62E3B9
:1083C00071E1CE0101960E94AF8DCE0101960E940F
:1083D0005931CE0101960E94198D64E471E1CE01FC
:1083E00001960E94AF8DCE0101960E945931CE01B7
:1083F00001960E94198DB5CF3F924F925F926F9276
:108400007F928F929F92AF92BF92CF92DF92EF9224
:10841000FF920F931F93CF93DF93CDB7DEB7629791
:108420000FB6F894DEBF0FBECDBF69EE76E0CE0189
:1084300001960E94A68DCE0101960E945931CE016F
:1084400001960E94198D04E010E038E5C32E39E052
:10845000D32E40E3E42E53EE752E66E0662E7CEEBE
:10846000572EE1E3FE2EFEE44F2EA4E33A2E68EBF6
:1084700072E287E191E10E94AB29F6018E2D119203
:108480008A95E9F77092580960925A0950925B09EF
:10849000F092640940926509F0926609309267098A
:1084A00060E472E0CE0101960E94238F4BE750E01A
:1084B000BE016F5F7F4F87E191E10E94342A40E364
:1084C00050E068E579E087E191E10E94C92987E100
:1084D00091E10E94032A68EE73E080E090E00E9440
:1084E0003D0E87E191E10E94FF25892B09F054C0E0
:1084F0000150110909F081C0809188099091890982
:10850000A0918A09B0918B09892B8A2B8B2B09F0BA
:108510008EC06DE574E082E691E10E94FB8A62E61E
:1085200071E1CE0101960E94AF8DAE014F5F5F4FAA
:1085300070E060E083E892E00E94623E8C01CE0130
:1085400001960E94198D0130110571F061ED76E000
:10855000CE0101960E94A68DCE0101960E9459314E
:10856000CE0101960E94198D62960FB6F894DEBF77
:108570000FBECDBFDF91CF911F910F91FF90EF9074
:10858000DF90CF90BF90AF909F908F907F906F9033
:108590005F904F903F90089540E350E068E579E0A8
:1085A00087E191E10E94B62560918009709181096F
:1085B00076276727762790E080E0CB01772766272C
:1085C000009182091091830910270127102730E0BC
:1085D00020E0602B712B822B932B7E508A4A93488C
:1085E0000E947C0E0E942F0F609388097093890966
:1085F00080938A0990938B097FCF8090880990900F
:108600008909A0908A09B0908B0968EE73E080E038
:1086100090E00E943D0E2AE0B501A40185E39FE0B1
:108620000E94198E85E39FE00E94AF8E20CF68EEF6
:1086300073E080E090E00E943D0E0E942F0F609357
:10864000D10B7093D20B8093D30B9093D40B0E94D9
:108650002F0F6093CD0B7093CE0B8093CF0B909325
:10866000D00BCE0101960E946D30CE0101960E9482
:108670005931CE0101960E94198D0E94870FBC01CD
:10868000CE0107960E94962E69E574E0CE0107960A
:108690000E94938C0E947F0FBC01CE0101960E9424
:1086A000962EBE016F5F7F4FCE0107960E949D8C74
:1086B000CE0101960E94198D69E574E0CE010796FE
:1086C0000E94938C0E94750FBC01CE0101960E94FE
:1086D000962EBE016F5F7F4FCE0107960E949D8C44
:1086E000CE0101960E94198D6FE175E0CE010196D1
:1086F0000E94B88DBE01695F7F4FCE0101960E9436
:10870000338CBC01CE010D960E94AF8D4AE050E043
:108710006FEF7FEFCE010D960E945437CE010D967C
:108720000E94198DCE0101960E94198DCE010796E7
:108730000E94198D68EE73E080E090E00E943D0E8B
:108740000E94970FBC01CE010D960E94962E0E94AA
:108750008F0FBC01CE0101960E94962E6FE376E04A
:10876000CE0107960E94B88DBE016F5F7F4FCE018C
:1087700007960E94338CBC01CE010D960E949D8C01
:10878000CE0107960E94198DCE0101960E94198D87
:108790000E942F0F0E94550A60919C0B70E0CE0141
:1087A00001960E94962E6FE376E0CE0107960E9416
:1087B000B88DBE016F5F7F4FCE0107960E94338C4C
:1087C000BC01CE010D960E949D8CCE0107960E94A1
:1087D000198DCE0101960E94198D65E275E0CE01DA
:1087E00001960E94B88DBE01635F7F4FCE01019656
:1087F0000E94338CBC01CE0107960E94AF8D4AE0E7
:1088000050E06FEF7FEFCE0107960E945437CE0104
:1088100007960E94198DCE0101960E94198DCE01F6
:108820000D960E94198D68EE73E080E090E00E9442
:108830003D0ECE0101960E94EC2F4AE050E06FEF12
:108840007FEFCE0101960E9454378ACE0F931F937B
:10885000CF93DF93CDB7DEB762970FB6F894DEBF44
:108860000FBECDBF8C010E942F0F603579468F401F
:10887000910560F1CE0101960E94EC2F4AE050E094
:108880006FEF7FEFCE0101960E945437CE01019623
:108890000E94198DB801CE0101960E94AF8D4AE069
:1088A00050E06FEF7FEFCE0101960E94FC2CCE01CD
:1088B00001960E94198D62960FB6F894DEBF0FBE26
:1088C000CDBFDF91CF911F910F9108950E94700E3F
:1088D00028EE33E040E050E00E948EB5CA01B901B5
:1088E0000E9449B4AB01BC0121E0CE0101960E9477
:1088F000218DBE016F5F7F4FCE0107960E94AF8D25
:108900006DE175E0CE0107960E941D8CBC01CE0181
:108910000D960E94AF8DCE0107960E94198DCE0153
:1089200001960E94198DBE01635F7F4FCE010196B3
:108930000E94AF8D4AE050E06FEF7FEFCE010196CD
:108940000E945437CE0101960E94198DB801CE01C4
:1089500001960E94AF8D4AE050E06FEF7FEFCE01AD
:1089600001960E94FC2CCE0101960E94198DCE0129
:108970000D969FCFCF92DF92EF92FF920F931F93AE
:10898000CF93DF93CDB7DEB768970FB6F894DEBF0D
:108990000FBECDBF6DE574E0CE0143960E94B88D49
:1089A00065EE78E0CE0101960E94A68DCE0101967B
:1089B0000E94A731CE0101960E94198D6CA17DA164
:1089C000CE0101960E94058BCE0101960E9459317D
:1089D000CE0101960E94198D6DEC78E0CE010196D2
:1089E0000E94A68DCE0101960E94A731CE0101966C
:1089F0000E94198DCE5ADE4F68817981C255D140CF
:108A0000CE0101960E94058BCE0101960E9459313C
:108A1000CE0101960E94198D60EC78E0CE0101969E
:108A20000E94A68DCE0101960E94A731CE0101962B
:108A30000E94198D07E31CE0EE24E394F12CCE5A3A
:108A4000DE4F88819981C255D1408E159F050CF467
:108A50004AC0F80182819381C6979CF16BE275E070
:108A6000CE0101960E94B88DCE0101960E94A731D9
:108A7000CE0101960E94198DF801628173816653BF
:108A80007109CE0101960E94058BCE0101960E94CC
:108A9000A731CE0101960E94198D6AEA75E0CE01D8
:108AA00001960E94B88DCE0101960E94A731CE0199
:108AB00001960E94198DFFEFEF1AFF0A0E5F1F4FFC
:108AC000BECF6DE275E0CE0101960E94B88DCE0159
:108AD00001960E94A731CE0101960E94198DF801DE
:108AE00062817381CECF6AEA75E0CE0101960E9461
:108AF000B88DCE0101960E945931CE0101960E9497
:108B0000198D61EB78E0CE0101960E94A68DCE0111
:108B100001960E94A731CE0101960E94198D6091A5
:108B20003F0C7091400CCE0101960E94058BCE0146
:108B300001960E94A731CE0101960E94198D6AEA22
:108B400075E0CE0101960E94B88DCE0101960E947B
:108B5000A731CE0101960E94198D6091410C709150
:108B6000420CCE0101960E94058BCE0101960E9417
:108B70005931CE0101960E94198D6AE978E0CE0143
:108B800001960E94A68DCE0101960E94A731CE01CA
:108B900001960E94198DBE01605D7F4FCE01019646
:108BA0000E94B88DCE0101960E94A731CE01019698
:108BB0000E94198D6AEA75E0CE0101960E94B88D77
:108BC000CE0101960E94A731CE0101960E94198D17
:108BD000BE016C5C7F4FCE0101960E94B88DCE0124
:108BE00001960E945931CE0101960E94198D6AE8C2
:108BF00078E0CE0101960E94A68DCE0101960E94DA
:108C00005931CE0101960E94198D8E010C5D1F4FC6
:108C1000EE24E394F12C680188E0C80ED11C8CA1ED
:108C20009DA18E159F050CF449C0B701CE01079692
:108C30000E94058B65E776E0CE0101960E94B88D13
:108C4000BE01695F7F4FCE0101960E94338CBC014B
:108C5000CE010D960E94AF8DCE010D960E94A731D8
:108C6000CE010D960E94198DCE0101960E94198D9C
:108C7000CE0107960E94198D6FE376E0CE01019632
:108C80000E94B88DCE0101960E94A731CE010196B7
:108C90000E94198DB801645E7F4FCE0101960E943B
:108CA000B88DCE0101960E945931CE0101960E94E5
:108CB000198DEFEFEE1AFE0A8601ADCF69E778E075
:108CC000CE0101960E94A68DCE0101960E94A73189
:108CD000CE0101960E94198D7E01F2EBEF1AFEEF94
:108CE000FF0A10E000E0F70161917F0170E0CE0122
:108CF00001960E94058BCE0101960E94A731CE01FC
:108D000001960E94198D0330110571F06FE275E034
:108D1000CE0101960E94B88DCE0101960E94A73126
:108D2000CE0101960E94198D0F5F1F4F043011056F
:108D3000D1F66AEA75E0CE0101960E94B88DCE01A7
:108D400001960E945931CE0101960E94198DC45B93
:108D5000DE4F68817981CC54D140072E000C880BFE
:108D6000990B0E944BB49B01AC010E940BB7882366
:108D700041F080E590E0C45BDE4F99838883CC545A
:108D8000D140C45BDE4F88819981CC54D14090930F
:108D90003F0280933E026FE578E0CE0101960E948B
:108DA000A68DCE0101960E94A731CE0101960E94A8
:108DB000198D6EE47AE0CE0101960E94B88DCE0145
:108DC00001960E94A731CE0101960E94198D6DE592
:108DD00078E0CE0101960E94A68DCE0101960E94F8
:108DE000A731CE0101960E94198D60913E027091CB
:108DF0003F02CE0101960E94058BCE0101960E9492
:108E00005931CE0101960E94198D6EE478E0CE01B1
:108E100001960E94A68DCE0101960E94A731CE0137
:108E200001960E94198DBE016C5A7F4FCE010196AA
:108E30000E94B88DCE0101960E945931CE01019653
:108E40000E94198D61E375E0CE0101960E94B88DF4
:108E5000CE0101960E94A731CE0101960E94198D84
:108E6000BE0164587F4FCE0101960E94B88DCE019D
:108E700001960E945931CE0101960E94198DC0526F
:108E8000DF4F88819981C05ED040892B71F466E400
:108E900078E0CE0101960E94A68DCE0101960E9437
:108EA0005931CE0101960E94198DC052DF4F888141
:108EB0009981C05ED040019771F46CE378E0CE01F7
:108EC00001960E94A68DCE0101960E945931CE01D5
:108ED00001960E94198DC052DF4F88819981C05E32
:108EE000D040029771F463E378E0CE0101960E94CE
:108EF000A68DCE0101960E945931CE0101960E94A5
:108F0000198D6DE278E0CE0101960E94A68DCE010A
:108F100001960E94A731CE0101960E94198DCE5173
:108F2000DF4F68817981C25ED040CE0101960E94F8
:108F3000058BCE0101960E945931CE0101960E9407
:108F4000198D64E278E0CE0101960E94A68DCE01D3
:108F500001960E94A731CE0101960E94198DCC5A2C
:108F6000DE4F88819981C455D140C6970CF43FC12A
:108F70006BE275E0CE0101960E94B88DCE0101969C
:108F80000E94A731CE0101960E94198DCC5ADE4F66
:108F900068817981C455D14066537109CE0101962B
:108FA0000E94058BCE0101960E945931CE01019697
:108FB0000E94198D4091C50B5091C60B6091C70B53
:108FC0007091C80B21E0CE0107960E94218D6CE3C1
:108FD00075E0CE0101960E94B88DBE01695F7F4F9A
:108FE000CE0101960E94338C68E475E00E941D8CCE
:108FF000BC01CE010D960E94AF8DCE010D960E9450
:109000005931CE010D960E94198DCE0101960E9414
:10901000198DCE0107960E94198D4091C10B509178
:10902000C20B6091C30B7091C40B21E0CE01079677
:109030000E94218D6DE475E0CE0101960E94B88DED
:10904000BE01695F7F4FCE0101960E94338C68E4B8
:1090500075E00E941D8CBC01CE010D960E94AF8D63
:10906000CE010D960E945931CE010D960E94198DA8
:10907000CE0101960E94198DCE0107960E94198D8E
:1090800065E078E0CE0101960E94A68DCE010196A2
:109090000E94A731CE0101960E94198D40912902AC
:1090A00050912A0260912B0270912C0225E0CE0192
:1090B00001960E94218DCE0101960E945931CE0168
:1090C00001960E94198D6AEE77E0CE0101960E940A
:1090D000A68DCE0101960E94A731CE0101960E9475
:1090E000198D4091250250912602609127027091BE
:1090F000280225E0CE0101960E94218DCE01019625
:109100000E945931CE0101960E94198D69ED77E0D8
:10911000CE0101960E94A68DCE0101960E94A73134
:10912000CE0101960E94198D6091700270917102BA
:10913000CE0101960E94058BCE0101960E94593105
:10914000CE0101960E94198D60EC77E0CE01019668
:109150000E94A68DCE0101960E94A731CE010196F4
:109160000E94198DC65BDE4F68817981CA54D14057
:10917000CE0101960E94058BCE0101960E945931C5
:10918000CE0101960E94198D69EA77E0CE01019621
:109190000E94A68DCE0101960E94A731CE010196B4
:1091A0000E94198DC95ADE4F68817981C755D14017
:1091B000CE0101960E94058BCE0101960E94593185
:1091C000CE0101960E94198DCE0143960E94198D01
:1091D00068960FB6F894DEBF0FBECDBFDF91CF917A
:1091E0001F910F91FF90EF90DF90CF9008956DE267
:1091F00075E0CE0101960E94B88DCE0101960E94C5
:10920000A731CE0101960E94198DCC5ADE4F68819C
:109210007981C455D140C2CE2F923F924F925F9236
:109220006F927F928F929F92AF92BF92CF92DF9276
:10923000EF92FF920F931F93CF93DF93CDB7DEB7DB
:10924000EC970FB6F894DEBF0FBECDBF9CA78BA7DF
:109250001B0170E060E00E94D18B182F6DE574E077
:10926000CE0149960E94B88D809170029091710252
:10927000019709F07AC082E090E00E94858988E039
:1092800090E0909324028093230289E090E09093F1
:1092900022028093210280911F0A9091200A9093CC
:1092A0001E0A80931D0A80911D0290911E02A091BA
:1092B0001F02B09120028093190290931A02A0938A
:1092C0001B02B0931C028091350290913602A0914E
:1092D0003702B09138028093390290933A02A093FA
:1092E0003B02B0933C0280911C0A80931B0A809140
:1092F000170A9091180AA091190AB0911A0A80933E
:10930000130A9093140AA093150AB093160A8AE3DD
:1093100090E090931802809317028091C50B909172
:10932000C60BA091C70BB091C80B8093490A9093CC
:109330004A0AA0934B0AB0934C0A8091150290916F
:109340001602909314028093130280912902909147
:109350002A02A0912B02B0912C0280932D029093AF
:109360002E02A0932F02B093300280917002909150
:109370007102029709F07AC083E090E00E9485892B
:109380008AE090E090932402809323028BE090E0A7
:1093900090932202809321028091110A9091120AE7
:1093A00090931E0A80931D0A80910F0290911002E3
:1093B000A0911102B09112028093190290931A02A7
:1093C000A0931B02B0931C02809131029091320253
:1093D000A0913302B09134028093390290933A0203
:1093E000A0933B02B0933C028091100A80931B0A29
:1093F00080910C0A90910D0AA0910E0AB0910F0A6B
:109400008093130A9093140AA093150AB093160A36
:109410008BE390E090931802809317028091C10B28
:109420009091C20BA091C30BB091C40B8093490AD9
:1094300090934A0AA0934B0AB0934C0A80910D0274
:1094400090910E0290931402809313028091250252
:1094500090912602A0912702B091280280932D02BC
:1094600090932E02A0932F02B09330021335C1F4D3
:1094700010921E0A10921D0A8091BC0B882371F075
:1094800065E575E0CE0101960E94B88DCE0101968A
:109490000E945931CE0101960E94198DE12CE1C044
:1094A000C1010197029708F06EC181E090E0A0E051
:1094B000B0E08093190290931A02A0931B02B0931C
:1094C0001C02ABA5BCA514968D919C911597029793
:1094D00050F141E050E0BD01CE0101960E948A2E7C
:1094E000BE016F5F7F4FCE0149960E94E08CCE0196
:1094F00001960E94198DCE014996B1E02B163104D8
:1095000071F50E945E8B20E030E040E251E40E9461
:10951000AAB40E94D0B66093190270931A02809385
:109520001B0290931C0281E090E090931E0A8093AE
:109530001D0A1134F9F48091BC0B882371F06AE59F
:1095400075E0CE0101960E94B88DCE0101960E9471
:109550005931CE0101960E94198DE12C4FC00E9415
:109560005E8B20912D0230912E0240912F0250915E
:109570003002CDCF163409F0F0C08091BC0B8823A7
:1095800071F063E675E0CE0101960E94B88DCE01C0
:1095900001960E94A731CE0101960E94198DEE24FA
:1095A000E394F12CD090210260E08D2D0E94B90D42
:1095B00064E670E080E090E00E943D0E009123029E
:1095C0006E2D802F0E94B90D64EF71E080E090E075
:1095D0000E943D0E60E08D2D0E94B90D64E670E0A2
:1095E00080E090E00E943D0E6E2D802F0E94B90D0C
:1095F00064EF71E080E090E00E943D0E8091BC0B32
:10960000882379F14091190250911A0260911B024E
:1096100070911C022AE0CE0101960E94578DBE0176
:109620006F5F7F4FCE0107960E94AF8D67E775E0B1
:10963000CE0107960E941D8CBC01CE010D960E94A2
:10964000AF8DCE010D960E945931CE010D960E942C
:10965000198DCE0107960E94198DCE0101960E94A8
:10966000198D8090190290901A02A0901B02B09060
:109670001C02181419041A041B040CF046C51634F5
:1096800009F44CC4123509F44DC4109123026E2D17
:10969000812F0E94B90D64EF71E080E090E00E949C
:1096A0003D0E6E2D812F0E94B90D60ED77E080E0B8
:1096B00090E00E943D0E6E2D812F0E94B90D6CED41
:1096C00075E080E090E00E943D0E81E090E0909394
:1096D0001E0A80931D0A1091210261E0812F0E94D1
:1096E000B90D61E070E080E090E00E943D0E60E026
:1096F000812F0E94B90D6AE070E080E090E00E9446
:109700003D0EC12CD12C7601C3948C149D04AE0463
:10971000BF0409F409C461E0812F0E94B90D61E022
:1097200070E080E090E00E943D0E60E0812F0E949A
:10973000B90D6091390270913A0280913B0290918B
:109740003C026F5F7F4F8F4F9F4F0E943D0EFFEF98
:10975000CF1ADF0AEF0AFF0AD8CF123591F48091B1
:10976000BC0B882371F06DE675E0CE0101960E9476
:10977000B88DCE0101960E94A731CE0101960E94BC
:10978000198DE12C0FCF2114310429F0E3E02E16BE
:10979000310409F083CE809170029091710220E132
:1097A00037E240E050E08130910521F420E43CE9CB
:1097B00040E050E02FA738AB49AB5AAB21E030E096
:1097C00030931E0A20931D0A30934D0220934C02C1
:1097D000029761F433E02316310441F48091BE1204
:1097E0009091BF1290934D0280934C0240914C0295
:1097F00050914D025EA74DA7052F001F0027001FA7
:1098000081E090E090934D0280934C02E090210221
:1098100060E08E2D0E94B90D64E670E080E090E07B
:109820000E943D0EF0902302602F8F2D0E94B90DF3
:1098300064EF71E080E090E00E943D0E602F8F2D7C
:109840000E94B90D68EE73E080E090E00E943D0E4A
:1098500060E08E2D0E94B90D64E670E080E090E03B
:109860000E943D0E602F8F2D0E94B90D64EF71E0B4
:1098700080E090E00E943D0E8FEF9FEF90931402E6
:1098800080931302812C912C54011FA218A619A6B3
:109890001AA61BA21CA21DA21EA21F8E18A219A2EC
:1098A0001AA2412C512C32011FAA18AE19AE1AAEC1
:1098B0001BAA1CAA1DAA1EAAF090210261E08F2DEE
:1098C0000E94B90D61E070E080E090E00E943D0EE2
:1098D00060E08F2D0E94B90D61E070E080E090E0C3
:1098E0000E943D0EC501B40126E030E040E050E0AA
:1098F0000E94B0B5672B682B692B09F0F8C0A2E075
:10990000B0E0BCAFABAFC12CD12C76018091170277
:10991000863308F0865320917B00982F9870277F1C
:10992000922B90937B008770806480937C00809161
:109930007A00806480937A0080917A0086FDFCCF63
:109940008091780060917900762F682F072E000CA7
:10995000880B990B0E944BB49B01AC01C701B60167
:109960000E94F2B56B017C0162E070E080E090E063
:109970000E943D0E2BAD3CAD2130310509F0ADC04C
:1099800020E030EC4FEF54E4C701B6010E945EB610
:109990006B017C018091BC0B882399F12DEC3CEC90
:1099A0004CE45EE3C701B6010E9406B787FD29C0FB
:1099B00022E0B701A601CE0107960E94218D6EE735
:1099C00075E0CE0101960E94B88DBE01695F7F4FA0
:1099D000CE0101960E94338CBC01CE010D960E94EF
:1099E000AF8DCE010D960E945931CE010D960E9489
:1099F000198DCE0101960E94198DCE0107960E9405
:109A0000198D2AE939E949E95EE3C701B6010E94E7
:109A100006B787FD13C0411451046104710411F4A9
:109A2000240135018BA19CA1ADA1BEA1892B8A2B5C
:109A30008B2B21F48BA29CA2ADA2BEA22DEC3CEC00
:109A40004CE45EE3C701B6010E9444B418160CF45E
:109A500049C0411451046104710409F448C02F8DB8
:109A600038A149A15AA1232B242B252B69F48FA1BE
:109A700098A5A9A5BAA5892B8A2B8B2B09F403C11C
:109A80008F8E98A2A9A2BAA22F8D38A149A15AA15E
:109A9000421653066406750654F5809113029091A0
:109AA000140297FFF5C01092140210921302420E96
:109AB000531E641E751ED301C201B595A7959795D7
:109AC00087958FAB98AFA9AFBAAF1F8E18A219A216
:109AD0001AA2412C512C32010AC0E1E0F0E0FCAFA7
:109AE000EBAF14CF411451046104710469F6E090A6
:109AF0001302F090140292E0E916F1043CF4F7FC32
:109B0000E3C0A3E02A16310409F0DEC08FA498A8B0
:109B1000A9A8BAA8BAE08B0E911CA11CB11C8FA5F4
:109B200098A9A9A9BAA988169906AA06BB060CF491
:109B3000C3CEF2E0EF16F1040CF479C06BA97CA956
:109B40008DA99EA92FA938AD49AD5AAD621B730BE3
:109B5000840B950B0E944BB44B015C01B701FF0CC9
:109B6000880B990B0E944BB49B01AC01C501B40159
:109B70000E945EB620E030E044EB53E40E945EB603
:109B80006B017C01C0922D02D0922E02E0922F0236
:109B9000F092300220E030E040E85FE30E9406B738
:109BA00087FDACC080917002909171028130910567
:109BB00009F090C0C092B612D092B712E092B812DB
:109BC000F092B912C0922902D0922A02E0922B029E
:109BD000F0922C026FE277E0CE0101960E94A68DF2
:109BE000CE0101960E94A731CE0101960E94198DE7
:109BF00040912D0250912E0260912F0270913002FF
:109C000025E0CE0101960E94218DCE0101960E9491
:109C10005931CE0101960E94198D84EF91E0909305
:109C200057028093560268E971E10E94972C33E055
:109C30002316310429F0E02E2114310409F011CD4E
:109C40008BA59CA50E945E8B6B017C01C092490A8A
:109C5000D0924A0AE0924B0AF0924C0A20E030E09F
:109C600044EB53E4C701B6010E9406B787FD6AC002
:109C700020E030E044EB53E4C701B6010E94F1B5A7
:109C80006B017C01EBCF8FA298A6A9A6BAA6F8CE4D
:109C90002114310409F02BCF019690931402809384
:109CA00013022F8D38A149A15AA1420E531E641EE2
:109CB000751ED301C201B595A795979587958BAB76
:109CC0009CABADABBEAB01CFEFEF8E1A9E0AAE0AD6
:109CD000BE0A25CF029709F07DCFC092BA12D0926A
:109CE000BB12E092BC12F092BD12C0922502D0923B
:109CF0002602E0922702F09228026CCF63E177E01F
:109D0000CE0101960E94A68DCE0101960E94A73138
:109D1000CE0101960E94198D40912D0250912E0284
:109D200060912F027091300225E0CE0101960E94D1
:109D3000218DCE0101960E945931CE0101960E94DB
:109D4000198D75CF20E030E0A901C701B6010E944E
:109D500044B487FF0BC020E030E044EB53E4C7017C
:109D6000B6010E94F2B56B017C01ECCFC092130AE0
:109D7000D092140AE092150AF092160A4FA058A445
:109D800069A47AA48BA19CA1ADA1BEA1481A590ACD
:109D90006A0A7B0A21143104D9F41092130A109232
:109DA000140A1092150A1092160AADA5BEA5C12C70
:109DB000D12C7601C394812C912C5401B7FF1CC087
:109DC000812C912C5401CC24CA94DC2C760114C033
:109DD000EDA5FEA5C12CD12C7601C394F7FF04C0DC
:109DE000CC24CA94DC2C76018090130A9090140A3B
:109DF000A090150AB090160A20912D0230912E02E3
:109E000040912F0250913002C501B4010E94AAB4C2
:109E10004B015C01A3019201C701B6010E947EB50E
:109E20000E944BB420E030E040E05FE30E94AAB41F
:109E30009B01AC01C501B4010E94F1B50E94D0B6EE
:109E40006093190270931A0280931B0290931C0274
:109E50008091BC0B882309F441C02AE04FA158A58A
:109E600069A57AA5CE010D960E94578D2AE04BA1D7
:109E70005CA16DA17EA1CE0107960E94578D65E879
:109E800075E0CE0101960E94B88DBE01695F7F4FDB
:109E9000CE0101960E94338C6AEA75E00E941D8C07
:109EA000BE01635F7F4F0E94338CBC01CE0143969D
:109EB0000E94AF8DCE0143960E945931CE01439648
:109EC0000E94198DCE0101960E94198DCE01079630
:109ED0000E94198DCE010D960E94198D8091190254
:109EE00090911A02A0911B02B0911C02E12C12E584
:109EF000B7FFB7CBB095A095909581959F4FAF4F89
:109F0000BF4F8093190290931A02A0931B02B09343
:109F10001C02EE24E394F12C16E4A3CBEE24E3948C
:109F2000F12CB3CBE12CB1CB22E02216310424F486
:109F30002114310409F0E1C061E080E00E948B84CB
:109F400032E02316310424F42114310409F09CC0BA
:109F5000C090490AD0904A0AE0904B0AF0904C0A0F
:109F600020E030E044EB53E4C701B6010E9406B79D
:109F700087FD0BC020E030E044EB53E4C701B6019D
:109F80000E94F1B56B017C01EBCF20E030E0A9012C
:109F9000C701B6010E9444B487FF0BC020E030E047
:109FA00044EB53E4C701B6010E94F2B56B017C019A
:109FB000ECCFC092490AD0924A0AE0924B0AF09242
:109FC0004C0A80917002909171020197B1F46DE397
:109FD00075E083EF90E10E94FB8A8091490A90919D
:109FE0004A0AA0914B0AB0914C0A8093C50B9093FA
:109FF000C60BA093C70BB093C80B809170029091D1
:10A0000071020297B1F46EE475E083EF90E10E9473
:10A01000FB8A8091490A90914A0AA0914B0AB0911B
:10A020004C0A8093C10B9093C20BA093C30BB093C7
:10A03000C40B4091490A50914A0A60914B0A7091B1
:10A040004C0A20E0CE0107960E94218D63EF70E15B
:10A05000CE0101960E94AF8DBE01695F7F4FCE0198
:10A0600001960E94338C69E475E00E941D8CBC014E
:10A0700083EF90E10E94C98CCE0101960E94198D58
:10A08000CE0107960E94198D41E02416310439F55E
:10A090004091190250911A0260911B0270911C02AA
:10A0A00021E0CE0107960E94578D6DE875E0CE0144
:10A0B00001960E94B88DBE01695F7F4FCE01019667
:10A0C0000E94338CBC0183EF90E10E94C98CCE01C9
:10A0D00001960E94198DCE0107960E94198D63EF9B
:10A0E00070E1CE0101960E94AF8DCE0101960E94D3
:10A0F0002644CE0101960E94198D109219021092E9
:10A100001A0210921B0210921C0280917002909110
:10A1100071028130910509F083C080911D0A9091F0
:10A120001E0A9093200A80931F0A80911902909131
:10A130001A02A0911B02B0911C0280931D02909301
:10A140001E02A0931F02B0932002809139029091C9
:10A150003A02A0913B02B0913C0280933502909369
:10A160003602A0933702B093380280911B0A809385
:10A170001C0A8091130A9091140AA091150AB091BB
:10A18000160A8093170A9093180AA093190AB0939D
:10A190001A0A8091490A90914A0AA0914B0AB091FB
:10A1A0004C0A8093C50B9093C60BA093C70BB0933A
:10A1B000C80B809113029091140290931602809321
:10A1C0001502232881F480912D0290912E02A091F6
:10A1D0002F02B09130028093290290932A02A0931B
:10A1E0002B02B0932C02CE0149960E94198DEC9659
:10A1F0000FB6F894DEBF0FBECDBFDF91CF911F9198
:10A200000F91FF90EF90DF90CF90BF90AF909F9015
:10A210008F907F906F905F904F903F902F90089518
:10A22000029709F780911D0A90911E0A9093120AD5
:10A230008093110A8091190290911A02A0911B0239
:10A24000B0911C0280930F0290931002A093110210
:10A25000B09312028091390290913A02A0913B0290
:10A26000B0913C028093310290933202A09333026A
:10A27000B093340280911B0A8093100A8091130AD4
:10A280009091140AA091150AB091160A80930C0AB5
:10A2900090930D0AA0930E0AB0930F0A8091490A79
:10A2A00090914A0AA0914B0AB0914C0A8093C10B3D
:10A2B0009093C20BA093C30BB093C40B8091130275
:10A2C0009091140290930E0280930D02232809F0BE
:10A2D0008ACF80912D0290912E02A0912F02B091F1
:10A2E00030028093250290932602A0932702B09318
:10A2F000280279CF2F923F924F925F926F927F9276
:10A300008F929F92AF92BF92CF92DF92EF92FF9285
:10A310000F931F93CF93DF93CDB7DEB7E5970FB6BB
:10A32000F894DEBF0FBECDBF61E171E1CE018E9624
:10A330000E94AF8D0EA51FA50115110571F0D80162
:10A340008D918D01882349F0082E000C990B0E94F5
:10A3500052B9F80131978083F2CF65E97DE0CE01F3
:10A3600001960E94A68DBE016F5F7F4FCE018E9633
:10A370000E94028C182FCE0101960E94198D112384
:10A3800009F401C145E050E061E171E1CE010196BF
:10A390000E948A2EBE016F5F7F4F8DEE90E10E947A
:10A3A000E08CCE0101960E94198D8DEE90E10E9405
:10A3B000748B60E08DEE90E10E94708C4091F11002
:10A3C0005091F21060EF71E18DEE90E10E94DD8915
:10A3D00066E874E0CE0101960E94B88DBE016F5F01
:10A3E0007F4F8DEE90E10E94028C182FCE010196D6
:10A3F0000E94198D60E774E0111102C065E774E0F6
:10A40000CE0101960E94B88D6DEE70E1CE010196ED
:10A410000E94338CBC0189EF92E10E94C98CCE016D
:10A4200001960E94198D89EF92E10E94748B4091F0
:10A43000FD125091FE124150510969EF72E1CE01B7
:10A4400001960E948A2EBE016F5F7F4F8BED92E1D5
:10A450000E94E08CCE0101960E94198D8BED92E155
:10A460000E94698B0E944BB49B01AC010E940BB708
:10A47000882309F448C06091FD127091FE12625069
:10A48000710989EF92E10E94D18B682FCE0101966C
:10A490000E94848DBE016F5F7F4F8BED92E10E9421
:10A4A000E08CCE0101960E94198D66E874E0CE0121
:10A4B00001960E94B88DBE016F5F7F4F8BED92E1D8
:10A4C0000E94028C182FCE0101960E94198D112333
:10A4D000D1F06091FD127091FE126350710989EF05
:10A4E00092E10E94D18B682FCE0101960E94848D4B
:10A4F000BE016F5F7F4F8BED92E10E94E08CCE0139
:10A5000001960E94198D84EF91E0909357028093F9
:10A51000560268E971E10E94972C64E670E080E0E1
:10A5200090E00E943D0E80913D02882371F061E130
:10A5300071E1CE0101960E94AF8DCE0101960E947D
:10A54000C02FCE0101960E94198DCE018E960E94D9
:10A55000198D81E0E5960FB6F894DEBF0FBECDBF32
:10A56000DF91CF911F910F91FF90EF90DF90CF90EF
:10A57000BF90AF909F908F907F906F905F904F9023
:10A580003F902F9008956FE87DE0CE0101960E94E4
:10A59000A68DBE016F5F7F4FCE018E960E94028C0A
:10A5A000182FCE0101960E94198D112309F447C07E
:10A5B00045E050E061E171E1CE0101960E948A2EF2
:10A5C000BE016F5F7F4F8DEE90E10E94E08CCE0167
:10A5D00001960E94198D8DEE90E10E94748B60E0CF
:10A5E0008DEE90E10E94708C4091F1105091F2102C
:10A5F00068EC71E18DEE90E10E94DD8968EC71E11B
:10A60000CE014C960E94B88D68E874E0CE010196A8
:10A610000E94B88DBE01645E7F4FCE0101960E94FC
:10A62000338CBC0183EF92E10E94C98CCE0101966C
:10A630000E94198DCE014C960E94198D64CF6BE853
:10A640007DE0CE0101960E94A68DBE016F5F7F4F17
:10A65000CE018E960E94028C182FCE0101960E9488
:10A66000198D1123E1F043E050E061E171E1CE0189
:10A6700001960E948A2EBE016F5F7F4F8DEE90E1A2
:10A680000E94E08CCE0101960E94198D6DEE70E162
:10A69000CE0101960E94AF8DCE010196CDCF66E826
:10A6A0007DE0CE0101960E94A68DBE016F5F7F4FB7
:10A6B000CE018E960E94028C182FCE0101960E9428
:10A6C000198D112301F144E050E061E171E1CE0107
:10A6D00001960E948A2EBE016F5F7F4F8DEE90E142
:10A6E0000E94E08CCE0101960E94198D8DEE90E1C2
:10A6F0000E94698B709357126093561270934702B1
:10A700006093460200CF60E87DE0CE0101960E9492
:10A71000A68DBE016F5F7F4FCE018E960E94028C88
:10A72000182FCE0101960E94198D112309F449C0FA
:10A7300045E050E061E171E1CE0101960E948A2E70
:10A74000BE016F5F7F4F8DEE90E10E94E08CCE01E5
:10A7500001960E94198D8DEE90E10E94698B709395
:10A76000B3126093B21284EF91E0909357028093FA
:10A77000560268E971E10E94972C64E670E080E07F
:10A7800090E00E943D0E65E776E0CE0101960E94C2
:10A79000B88D61E171E1CE0101960E94338CBC015C
:10A7A000CE014C960E94AF8DCE014C960E9459313D
:10A7B000CE014C960E94198DCE0101960E94198DF2
:10A7C000B2CE6BE77DE0CE0101960E94A68DBE0160
:10A7D0006F5F7F4FCE018E960E94028C182FCE01A4
:10A7E00001960E94198D1123E1F044E050E061E1EF
:10A7F00071E1CE0101960E948A2EBE016F5F7F4FEC
:10A800008DEE90E10E94E08CCE0101960E94198DA0
:10A810008DEE90E10E94698B7093B5126093B41233
:10A82000A2CF62E77DE0CE0101960E94A68DBE0117
:10A830006F5F7F4FCE018E960E94028C182FCE0143
:10A8400001960E94198D1123E1F048E050E061E18A
:10A8500071E1CE0101960E948A2EBE016F5F7F4F8B
:10A860008DEE90E10E94E08CCE0101960E94198D40
:10A870008DEE90E10E94698B7093CC126093CB12A5
:10A8800072CF6DE67DE0CE0101960E94A68DBE01DD
:10A890006F5F7F4FCE018E960E94028C182FCE01E3
:10A8A00001960E94198D1123A1F044E050E061E16E
:10A8B00071E1CE0101960E948A2EBE016F5F7F4F2B
:10A8C0008DEE90E10E94E08CCE0101960E94198DE0
:10A8D00054CF65E67DE0CE0101960E94A68DBE01B3
:10A8E0006F5F7F4FCE018E960E94028C182FCE0193
:10A8F00001960E94198D1123A1F047E050E061E11B
:10A9000071E1CE0101960E948A2EBE016F5F7F4FDA
:10A910008DEE90E10E94E08CCE0101960E94198D8F
:10A92000FCCD6DE57DE0CE0101960E94A68DBE01B5
:10A930006F5F7F4FCE018E960E94028C182FCE0142
:10A9400001960E94198D1111D8CF63E57DE0CE01EB
:10A9500001960E94A68DBE016F5F7F4FCE018E963D
:10A960000E94028C182FCE0101960E94198D11238E
:10A9700021F081E00E94972DD0CD6CE47DE0CE01E6
:10A9800001960E94A68DBE016F5F7F4FCE018E960D
:10A990000E94028C182FCE0101960E94198D11235E
:10A9A00019F00E94E940B9CD62E47DE0CE01019644
:10A9B0000E94A68DBE016F5F7F4FCE018E960E94D2
:10A9C000028C182FCE0101960E94198D112309F4D3
:10A9D00083C067E37DE0CE0101960E94A68DBE0193
:10A9E0006F5F7F4FCE018E960E94028C182FCE0192
:10A9F00001960E94198D112309F452C04AE050E0DB
:10AA000061E171E1CE0101960E948A2EBE016F5F65
:10AA10007F4F8DEE90E10E94E08CCE0101960E9466
:10AA2000198D8DEE90E10E94698B0E947C0E0E9430
:10AA30002F0F6093D10B7093D20B8093D30B909315
:10AA4000D40B0E942F0F6093CD0B7093CE0B80938D
:10AA5000CF0B9093D00BCE014C960E946D3064E9E1
:10AA600075E0CE0101960E94B88DBE01645E7F4FF5
:10AA7000CE0101960E94338CBC01CE0182960E94C9
:10AA8000AF8DCE0182960E945931CE0182960E94EE
:10AA9000198DCE0101960E94198DCE014C9678C277
:10AAA0004BE050E061E171E1CE0101960E948A2EF7
:10AAB000BE016F5F7F4F8DEE90E10E94E08CCE0172
:10AAC00001960E94198D8DEE90E10E94698B60586D
:10AAD0007F488F4F9F4FA9CF61E37DE0CE01019664
:10AAE0000E94A68DBE016F5F7F4FCE018E960E94A1
:10AAF000028C182FCE0101960E94198D112309F4A2
:10AB00006AC045E050E061E171E1CE0101960E942A
:10AB10008A2EBE016F5F7F4F8DEE90E10E94E08C28
:10AB2000CE0101960E94198D0E942F0F6093D10BC8
:10AB30007093D20B8093D30B9093D40B8DEE90E156
:10AB40000E94698B60937202709373028093740207
:10AB500090937502609398127093991280939A1251
:10AB600090939B12209197122093340C672B682BA3
:10AB7000692B11F41092340C84EF91E090935702FA
:10AB80008093560268E971E10E94972C64E670E0B8
:10AB900080E090E00E943D0E62E27DE0CE010196F1
:10ABA0000E94A68DCE0101960E94A731CE0101968A
:10ABB0000E94198D4091720250917302609174024B
:10ABC00070917502CE0101960E94318BCE010196E3
:10ABD0000E945931DBC167E17DE0CE0101960E9400
:10ABE000A68DBE016F5F7F4FCE018E960E94028CB4
:10ABF000182FCE0101960E94198D1123D9F14AE038
:10AC000050E061E171E1CE0101960E948A2EBE0101
:10AC10006F5F7F4F8DEE90E10E94E08CCE01019638
:10AC20000E94198D8DEE90E10E94698B6130710553
:10AC30008105910519F481E0809397128DEE90E1E2
:10AC40000E94698B672B682B692B11F41092971265
:10AC5000809197128093340C882309F484CD0E944C
:10AC60002F0F6093D10B7093D20B8093D30B9093E3
:10AC7000D40B79CD6EE07DE0CE0101960E94A68DC9
:10AC8000BE016F5F7F4FCE018E960E94028C182FFF
:10AC9000CE0101960E94198D1123A1F048E050E0E9
:10ACA00061E171E1CE0101960E948A2EBE016F5FC3
:10ACB0007F4F8DEE90E10E94E08CCE0101960E94C4
:10ACC000198D61CD68E07DE0CE0101960E94A68DD0
:10ACD000BE016F5F7F4FCE018E960E94028C182FAF
:10ACE000CE0101960E94198D112321F145E050E01B
:10ACF00061E171E1CE0101960E948A2EBE016F5F73
:10AD00007F4F8DEE90E10E94E08CCE0101960E9473
:10AD1000198D8DEE90E10E94698B6130710521F4EF
:10AD200081E08093350CFFCB672B09F0FCCB1092B0
:10AD3000350CF9CB64E07DE0CE0101960E94A68D32
:10AD4000BE016F5F7F4FCE018E960E94028C182F3E
:10AD5000CE0101960E94198D112351F163E070E03C
:10AD600081E191E10E94D18B682FCE0101960E9472
:10AD7000848DBE016F5F7F4F8DEE90E10E94E08C6D
:10AD8000CE0101960E94198D8DEE90E10E94748B88
:10AD90008DEE90E10E94698B9B0121503109233097
:10ADA000310508F0C0CB7093C7126093C612ABCBCD
:10ADB0006DEF7CE0CE0101960E94A68DBE016F5F13
:10ADC0007F4FCE018E960E94028C182FCE010196E5
:10ADD0000E94198D112309F46AC066E070E081E1D8
:10ADE00091E10E94D18B682FCE0101960E94848D43
:10ADF000BE016F5F7F4F8DEE90E10E94E08CCE012F
:10AE000001960E94198D8DEE90E10E94748B60E096
:10AE10008DEE90E10E94708C8DEE90E10E94698B26
:10AE20006B01CB010197039708F07DCB48E050E020
:10AE300061E171E1CE0101960E948A2EBE016F5F31
:10AE40007F4F8DEE90E10E94E08CCE0101960E9432
:10AE5000198D8DEE90E10E94748B8091F11090918C
:10AE6000F2100997A8F028E030E050E040E06DEEE5
:10AE700070E1CE0101960E94CD8DBE016F5F7F4FC4
:10AE80008DEE90E10E94E08CCE0101960E94198D1A
:10AE9000B601B3E0660F771FBA95E1F764557E4EB1
:10AEA00048E050E08DEE90E10E94DD892CCB65EF0B
:10AEB0007CE0CE0101960E94A68DBE016F5F7F4FA0
:10AEC000CE018E960E94028C182FCE0101960E9410
:10AED000198D112309F488C06DE574E0CE01019647
:10AEE0000E94B88D47E050E0BE01625D7F4FCE0109
:10AEF0004C960E948A2EBE01645E7F4FCE01019661
:10AF00000E94E08CCE014C960E94198D6BE275E098
:10AF1000CE014C960E94B88DBE01645E7F4FCE017B
:10AF200001960E94028C182FCE014C960E94198D1A
:10AF3000112389F141E050E0BE016F5F7F4FCE01E8
:10AF40004C960E948A2ECE014C960E94698B8B01F2
:10AF50000A5C1F4FCE014C960E94198D1093C912A6
:10AF60000093C812109345020093440284EF91E0CD
:10AF7000909357028093560268E971E10E94972CE2
:10AF800064E670E080E090E00E943D0ECE01019604
:10AF90000E94198DC8CA6DE275E0CE014C960E94E0
:10AFA000B88DBE01645E7F4FCE0101960E94028C77
:10AFB000182FCE014C960E94198D112379F041E093
:10AFC00050E0BE016F5F7F4FCE014C960E948A2EEB
:10AFD000CE014C960E94698B8B01BCCFCE010196AD
:10AFE0000E94698B8B01BACF6EEE7CE0CE01019698
:10AFF0000E94A68DBE016F5F7F4FCE018E960E948C
:10B00000028C182FCE0101960E94198D112309F48C
:10B01000AAC06DEA75E0CE0101960E94B88D46E0A7
:10B0200050E0BE016F5F7F4FCE018E960E941DAA39
:10B030008C01CE0101960E94198D980146E050E0E6
:10B04000BE01625D7F4FCE0101960E94CD8DCE0183
:10B0500001960E94698B6B01CE0101960E94198DA9
:10B060006DE574E0CE0101960E94B88DA8014F5F96
:10B070005F4FBE01625D7F4FCE014C960E948A2ECB
:10B08000BE01645E7F4FCE0101960E94E08CCE012E
:10B090004C960E94198D6BE275E0CE014C960E9491
:10B0A000B88DBE01645E7F4FCE0101960E94028C76
:10B0B000182FCE014C960E94198D112321F141E0E9
:10B0C00050E0BE016F5F7F4FCE014C960E948A2EEA
:10B0D000CE014C960E94698B8B010A5C1F4FCE01FA
:10B0E0004C960E94198DF6013196EE0FFF1FE8561F
:10B0F000FE4E11830083F601EE0FFF1FE95CF34F54
:10B100001183008333CF6DE275E0CE014C960E942F
:10B11000B88DBE01645E7F4FCE0101960E94028C05
:10B12000182FCE014C960E94198D112379F041E021
:10B1300050E0BE016F5F7F4FCE014C960E948A2E79
:10B14000CE014C960E94698B8B01C9CFCE0101962E
:10B150000E94698B0091390C10913A0C0150110931
:10B16000060F171FC0CF67EE7CE0CE014C960E9401
:10B17000A68DBE01645E7F4FCE018E960E94028C2A
:10B1800011E0811115C060EE7CE0CE0101960E94B5
:10B19000A68DBE016F5F7F4FCE018E960E94028CFE
:10B1A00011E0811101C010E0CE0101960E94198DBD
:10B1B000CE014C960E94198D112309F4F0C16AEA60
:10B1C00075E0CE014C960E94B88D65EA75E0CE011F
:10B1D00001960E94B88DAE01445E5F4FBE016F5F65
:10B1E0007F4FCE018E960E9424A9CE0101960E9427
:10B1F000198DCE014C960E94198D6AEA75E0CE0138
:10B200004C960E94B88D67EA75E0CE0101960E94C7
:10B21000B88DAE01445E5F4FBE016F5F7F4FCE01C0
:10B220008E960E9424A9CE0101960E94198DCE010E
:10B230004C960E94198D6AEA75E0CE014C960E94E8
:10B24000B88D69EA75E0CE0101960E94B88DAE0115
:10B25000445E5F4FBE016F5F7F4FCE018E960E94AE
:10B2600024A9CE0101960E94198DCE014C960E9410
:10B27000198D6DEA75E0CE014C960E94B88D6CEA8E
:10B2800075E0CE0101960E94B88DAE01445E5F4F1D
:10B29000BE016F5F7F4FCE018E960E9424A9CE0122
:10B2A00001960E94198DCE014C960E94198D6DEA6F
:10B2B00075E0CE014C960E94B88D67EC76E0CE0129
:10B2C00001960E94B88DAE01445E5F4FBE016F5F74
:10B2D0007F4FCE018E960E9424A9CE0101960E9436
:10B2E000198DCE014C960E94198DCE018E960E942A
:10B2F000748B0E942F0F6093D50B7093D60B8093A5
:10B30000D70B9093D80B06E010E054E6852E912CD5
:10B31000A12CB12C22242394312C6801B3E0CB0E54
:10B32000D11C8AA99BA90197C816D9060CF0FBC8A5
:10B33000B801CE018E960E94D18B682FCE014C961B
:10B340000E94848D7801E2E0EE0EF11C0F5F1F4F2A
:10B350009701A801BE01625D7F4FCE0101960E9458
:10B36000CD8DCE0101960E94698B2B01CE010196F5
:10B370000E94198D6AEA75E0CE0101960E94B88D8F
:10B38000A701BE016F5F7F4FCE018E960E941DAA5E
:10B390007C01CE0101960E94198D6DE574E0CE010D
:10B3A00001960E94B88DC20101979DAB8CAB1E1413
:10B3B0001F0424F59701A601BE01625D7F4FCE01F7
:10B3C00082960E94CD8DBE016E5D7F4FCE010196AB
:10B3D0000E94E08CCE0182960E94198DACA9BDA975
:10B3E000139718F187010F5F1F4FCE0101960E943E
:10B3F000198DCE014C960E94198D8FCFA601BE01EA
:10B40000625D7F4FCE0182960E948A2EBE016E5DE4
:10B410007F4FCE0101960E94E08CCE0182960E9461
:10B42000198DECA9FDA9339700F770E060E0CE011B
:10B430004C960E94D18B823509F050C0CE01019606
:10B440000E94698B672B682B692BB1F4F201EE0F18
:10B45000FF1FE952FD4F11821082F201EE0FFF1F14
:10B46000EE0FFF1FE154FD4F82E090E0A0E0B0E05E
:10B4700080839183A283B383CE0101960E94698B5E
:10B48000613071058105910509F067C0F201EE0F89
:10B49000FF1FE952FD4F31822082440C551C440CA1
:10B4A000551CF201E154FD4F80819181A281B3814D
:10B4B000181619061A061B0624F080829182A282B1
:10B4C000B382CE0101960E94698B623071058105BD
:10B4D0009105D4F1F201E154FD4F51C0863409F0D9
:10B4E00041C0CE0101960E94698B672B682B692BA6
:10B4F00039F4F201EE0FFF1FE85AFD4F118210825E
:10B50000CE0101960E94698B61307105810591051C
:10B5100039F4F201EE0FFF1FE85AFD4F318220820D
:10B52000440C551C440C551CF201E154FD4F808124
:10B530009181A281B381181619061A061B0624F000
:10B5400080829182A282B3820E942F0FF201E15287
:10B55000FD4F60837183828393831E141F040CF458
:10B5600041CF43CF843481F4CE0101960E94698B90
:10B57000440C551C440C551CF201E05AFD4F6083ED
:10B58000718382839383E0CF843539F7CE010196AE
:10B590000E94698B440C551C440C551C9BCF6AEDD2
:10B5A0007CE0CE0101960E94A68DBE016F5F7F4FA9
:10B5B000CE018E960E94028C082FCE0101960E9429
:10B5C000198D002309F49DC045E050E061E171E16F
:10B5D000CE0101960E948A2EBE016F5F7F4F8DEED5
:10B5E00090E10E94E08CCE0101960E94198D8DEEB3
:10B5F00090E10E94748B60E08DEE90E10E94708C6F
:10B600006FE275E0CE014C960E94B88D6DEE70E150
:10B61000CE0101960E94AF8DAE014E5D5F4FBE011F
:10B62000645E7F4FCE0101960E9439AA182FCE0189
:10B6300001960E94198DCE014C960E94198D1123FE
:10B6400011F40C9493528E010E5D1F4F52ECC52ED7
:10B6500052E1D52E60E4A62E62E0B62EF12CE12C4C
:10B66000D8016D918D01F60161936F01D5016D9344
:10B670005D01CE0101960E94ACA8CE0101960E9408
:10B68000A731CE0101960E94198DB3E0EB16F104AB
:10B6900071F06FE275E0CE0101960E94B88DCE0187
:10B6A00001960E94A731CE0101960E94198DEFEFFD
:10B6B000EE1AFE0AF4E0EF16F10491F66DE574E07F
:10B6C000CE0101960E94B88DCE0101960E9459319B
:10B6D000CE0101960E94198D68E971E180915602B0
:10B6E000909157020E94972C64E670E080E090E011
:10B6F0000E943D0E62EC7CE0CE0101960E94A68D78
:10B7000065CA6DEB7CE0CE0101960E94A68DBE015C
:10B710006F5F7F4FCE018E960E94028C082FCE0164
:10B7200001960E94198D002309F47CC044E050E08A
:10B7300061E171E1CE0101960E948A2EBE016F5F28
:10B740007F4F8DEE90E10E94E08CCE0101960E9429
:10B75000198D8DEE90E10E94748B60E08DEE90E18A
:10B760000E94708C4091F1105091F2106EE47AE0DA
:10B770008DEE90E10E94DD896FE275E0CE014C967E
:10B780000E94B88D6DEE70E1CE0101960E94AF8DE2
:10B79000AE014E5D5F4FBE01645E7F4FCE010196EC
:10B7A0000E9439AA182FCE0101960E94198DCE0150
:10B7B0004C960E94198D112311F40C9493528E0112
:10B7C0000E5D1F4F44ECE42E41E1F42E6E0186E243
:10B7D000C80ED11CD8016D918D01F70161937F01D5
:10B7E000CE0101960E94ACA8CE0101960E9459316B
:10B7F000CE0101960E94198D0C151D0559F784EF95
:10B8000091E0909357028093560268E971E10E949B
:10B81000972C64E670E080E090E00E943D0E62EBC1
:10B820007CE06ACF6BEA7CE0CE0101960E94A68D97
:10B83000BE016F5F7F4FCE018E960E94028C082F53
:10B84000CE0101960E94198D0023F1F146E050E0EF
:10B8500061E171E1CE0101960E948A2EBE016F5F07
:10B860007F4F8DEE90E10E94E08CCE0101960E9408
:10B87000198D8DEE90E10E94748B8091F110909162
:10B88000F210892B11F40C9493528DEE90E10E94EA
:10B89000698B7093C1126093C01270933F026093E2
:10B8A0003E0284EF91E0909357028093560268E93C
:10B8B00071E10E94972C64E670E080E090E00E94C5
:10B8C0003D0E67E97CE018CF60E97CE0CE0101968F
:10B8D0000E94A68DBE016F5F7F4FCE018E960E94A3
:10B8E000028C082FCE0101960E94198D002321F1B0
:10B8F00063E87CE0CE0101960E94A68D44E650E00C
:10B900006FEF7FEFCE0101960E94FC2CCE010196D5
:10B910000E94198D81E08093CA1284EF91E0909388
:10B9200057028093560268E971E10E94972CF0E07B
:10B93000E0E019950C9493526BE77CE0CE01019600
:10B940000E94A68DBE016F5F7F4FCE018E960E9432
:10B95000028C082FCE0101960E94198D002381F0E0
:10B960000E94B09461E47CE0882309F4C5CE64E6CB
:10B9700070E080E090E00E943D0E62E67CE0BCCE8C
:10B9800069E37CE0CE0101960E94A68DBE016F5F47
:10B990007F4FCE018E960E94028C082FCE01019619
:10B9A0000E94198D002301F16FEA75E0CE01019626
:10B9B0000E94B88D61EE72E1CE0101960E94338C37
:10B9C000BC0183EF90E10E94C98CCE0101960E94D8
:10B9D000198D63EF70E1CE0101960E94AF8DCE010B
:10B9E00001960E94593180C462E37CE0CE01019649
:10B9F0000E94A68DBE016F5F7F4FCE018E960E9482
:10BA0000028C082FCE0101960E94198D002349F166
:10BA100063E27CE083EF90E10E94A48C6DEE72E122
:10BA200087EE92E10E94C98C67EE72E1CE01019629
:10BA30000E94AF8DBE016F5F7F4F83EF90E10E9448
:10BA40009D8CCE0101960E94198D63EF70E1CE01AD
:10BA500001960E94AF8DCE0101960E9459310C943F
:10BA60008C546AE17CE0CE0101960E94A68DBE0155
:10BA70006F5F7F4FCE018E960E94028C082FCE0101
:10BA800001960E94198D002331F00E94FC41109212
:10BA90003D020C94935265E17CE0CE0101960E9438
:10BAA000A68DBE016F5F7F4FCE018E960E94028CE5
:10BAB000082FCE0101960E94198D002309F441C080
:10BAC0006DEA75E0CE0101960E94B88D4091151186
:10BAD000509116118D819E81481B590BBE016F5FDD
:10BAE0007F4F81E191E10E94D6A8AC014F5F5F4F8B
:10BAF00061E171E1CE014C960E948A2EBE01645E26
:10BB00007F4F8DEE90E10E94E08CCE014C960E941A
:10BB1000198DCE0101960E94198D8DEE90E10E9443
:10BB2000698B6115710531F481E08093F0020E9408
:10BB30000C96ADCF6130710509F0A9CF1092F002DB
:10BB4000F6CF61E17CE0CE0101960E94A68DBE0198
:10BB50006F5F7F4FCE018E960E94028C082FCE0120
:10BB600001960E94198D002309F438C143E050E08A
:10BB700061E171E1CE0101960E948A2EBE016F5FE4
:10BB80007F4F8DEE90E10E94E08CCE0101960E94E5
:10BB9000198D6DEE70E1CE0101960E94AF8DCE0140
:10BBA00001960E94C02FCE0101960E94198D84EF4C
:10BBB00091E090935702809356026DEE70E1CE01B2
:10BBC00001960E94AF8DCE0101960E94848CBC012B
:10BBD0008DEE92E10E94C98CCE0101960E94198DD2
:10BBE0006DEE70E1CE0101960E94AF8DCE010196FF
:10BBF0000E94848CBC0187EE92E10E94C98CCE0128
:10BC000001960E94198D4091F1125091F21268E54F
:10BC100072E18DEE92E10E94DD894091EB1250912C
:10BC2000EC1263E672E187EE92E10E94DD8968E939
:10BC300071E180915602909157020E94972C6AEB15
:10BC400075E0CE0101960E94B88D6DEE70E1CE01D7
:10BC500001960E94338CBC01CE0182960E94AF8D6A
:10BC6000CE0101960E94198D809154129091551227
:10BC7000892B39F4BE016E5D7F4F88E99EE00E94FA
:10BC8000CD8E68EB7BE080E090E00E943D0E8091DD
:10BC9000541290915512029709F087C06DEE70E131
:10BCA000CE0188960E94AF8D62EC75E0CE010196C0
:10BCB0000E94B88DCE0101960E943896CE01019661
:10BCC0000E94198D64EF71E080E090E00E943D0ECB
:10BCD00065EC75E0CE0101960E94B88DCE0101960B
:10BCE0000E943896CE0101960E94198D6CED75E088
:10BCF00080E090E00E943D0E6EEC75E0CE01019672
:10BD00000E94B88DCE0101960E943896CE01019610
:10BD10000E94198D64EF71E080E090E00E943D0E7A
:10BD20006CED75E0CE0101960E94B88DCE010196B2
:10BD30000E943896CE0101960E94198D64EF71E041
:10BD400080E090E00E943D0E6AEB75E0CE01019626
:10BD50000E94B88DBE01685D7F4FCE0101960E94A2
:10BD6000338CBC01CE014C960E94AF8DCE01019662
:10BD70000E94198DCE014C960E94748BBE01645EA8
:10BD80007F4FCE0101960E94AF8DCE0101960E9499
:10BD90003896CE0101960E94198DCE014C960E94D4
:10BDA000198DCE0188960E94198D68EB7BE080E0AA
:10BDB00090E00E943D0E68E572E1CE0101960E947E
:10BDC000B88DCE0101960E94C02FCE0101960E942F
:10BDD000198D10923D02CE018296DAC86CE07CE0AB
:10BDE000CE0101960E94A68DBE016F5F7F4FCE01EE
:10BDF0008E960E94028C811110914D0ACE010196FF
:10BE00000E94198D112309F486C044E050E061E1DD
:10BE100071E1CE0101960E948A2EBE016F5F7F4FB5
:10BE20008DEE90E10E94E08CCE0101960E94198D6A
:10BE30006AEE75E0CE0101960E94B88D6DEE70E15C
:10BE4000CE0101960E94338CBC01CE014C960E941B
:10BE5000AF8DCE0101960E94198D80915412909160
:10BE60005512892B39F4BE01645E7F4F88E99EE04C
:10BE70000E94CD8E68E873E180E090E00E943D0E64
:10BE80008091541290915512029759F561EF75E027
:10BE9000CE0101960E94B88D8091F1109091F21020
:10BEA000892B19F56AEF75E0CE0101960E94FB8A95
:10BEB000BE01645E7F4FCE0182960E94AF8DCE019F
:10BEC00082960E943896CE0182960E94198D68E86B
:10BED00073E180E090E00E943D0ECE0101960E9449
:10BEE000198D10923D020C944D55BE016F5F7F4F2E
:10BEF000CE0182960E94AF8DCE0182960E94389626
:10BF0000CE0182960E94198D60E777E180E090E093
:10BF10000E943D0ECDCF68E07CE0CE0101960E94EC
:10BF2000A68DBE016F5F7F4FCE018E960E94028C60
:10BF3000811110914D0ACE0101960E94198D112395
:10BF400009F462C061E171E18DEE90E10E94C98C5B
:10BF500081E080933D0261E171E1CE0101960E9492
:10BF6000AF8DCE0101960E94C02FCE0101960E9496
:10BF7000198D8091541290915512029709F16DEE2E
:10BF800070E188E99EE00E94CD8E68EB7BE080E066
:10BF900090E00E943D0ECE0101960E94D196BE0116
:10BFA0006F5F7F4F81E191E10E94E08CCE010196AD
:10BFB0000E94198D60ED77E080E090E00E943D0ED8
:10BFC0008091541290915512029771F46DEE70E1C8
:10BFD000CE0101960E94AF8DCE0101960E94389647
:10BFE000CE0101960E94198D809115119091161124
:10BFF000892B09F44CCD65E776E0CE0101960E94CD
:10C00000B88D61E171E1A2C462E07CE0CE010196ED
:10C010000E94A68DBE016F5F7F4FCE018E960E945B
:10C02000028C182FCE0101960E94198D112309F45C
:10C0300095C18091541290915512019709F027CD26
:10C0400063E076E0CE0188960E94B88DBE01685DFF
:10C050007F4F88E99EE00E94CD8E6CE271E080E027
:10C0600090E00E943D0ECE0182960E94D19664E639
:10C0700070E080E090E00E943D0E10E000E025E0DE
:10C08000C22ED12C3AE0A32EB12C6EE076E0CE0188
:10C0900001960E94B88D50E040E0BE016F5F7F4F77
:10C0A000CE0182960E941DAA7C01CE0101960E94BB
:10C0B000198DA7014F5F5F4FBE016E5D7F4FCE01AF
:10C0C00001960E948A2EBE016F5F7F4FCE01889637
:10C0D0000E94E08CCE0101960E94198D8CA59DA531
:10C0E000892B09F170E060E0CE0188960E94D18B27
:10C0F000082E000C990BC0970A97A8F460E176E02F
:10C10000CE0101960E94B88DBE016F5F7F4FCE01B8
:10C1100088960E94028CE82ECE0101960E94198D0D
:10C12000FF24F394E110F12C65EF78E0CE01019645
:10C130000E94A68D64E170E0CE0101960E94F3AAF0
:10C14000CE0101960E94198D0F5F1F4F62E370E0D0
:10C1500080E090E00E943D0EC801B6010E9410B739
:10C160000197C1F4CE0101960E9468338D819E81B2
:10C17000892B09F4BEC0BE016F5F7F4F81E191E161
:10C180000E94C98C0E947A51FF24F394CE0101963B
:10C190000E94198DCE0101960E94D196BE016F5F5B
:10C1A0007F4FCE0182960E94E08CCE0101960E94C4
:10C1B000198D62E370E080E090E00E943D0E04364D
:10C1C000110519F0FF2009F460CF8091BC0B882382
:10C1D000F1F065E776E0CE014C960E94B88DBE0185
:10C1E000685D7F4FCE014C960E94338CBC01CE011E
:10C1F00001960E94AF8DCE0101960E945931CE0169
:10C2000001960E94198DCE014C960E94198D8CA525
:10C210009DA5892B69F070E060E0CE0188960E94B0
:10C22000D18B082E000C990BC0970A9708F47AC09E
:10C2300068E176E0CE0101960E94B88DCE0182962B
:10C240000E94198DCE0188960E94198D8D819E8144
:10C25000009709F449C0E981FA812081222309F479
:10C2600043C0079708F440C069EF7BE0CE014C96CD
:10C270000E94A68D68EC70E0CE014C960E94F3AA55
:10C28000CE014C960E94198DBE016F5F7F4FCE018B
:10C290004C960E94AF8D40ED57E06FEF7FEFCE01DF
:10C2A0004C960E94FC2CCE014C960E94198D64E2A3
:10C2B00076E0CE014C960E94B88D61E171E1CE012D
:10C2C0004C960E94338CBC01CE0182960E94AF8DA9
:10C2D000CE0182960E945931CE0182960E94198D1C
:10C2E000CE014C960E94198DCE0101960E94198DA7
:10C2F000CECB043111050CF449CFC801B5010E9421
:10C3000010B7892B09F042CFBE01685D7F4F88E9E5
:10C310009EE00E94CD8E68EC70E080E090E00E948C
:10C320003D0E34CF60E176E0CE0101960E94B88DDB
:10C33000BE016F5F7F4FCE0188960E94028C182F3E
:10C34000CE0101960E94198D111172CFBE01685D58
:10C350007F4FCE0101960E949D8D70CF64EF7BE0F0
:10C36000CE0101960E94A68DBE016F5F7F4FCE0168
:10C370008E960E94028C182FCE0101960E94198D74
:10C38000112309F4F7C025E030E044E050E061E11A
:10C3900071E1CE0101960E94CD8DBE016F5F7F4F8E
:10C3A0008DEE90E10E94E08CCE0101960E94198DE5
:10C3B00061E171E1CE0101960E94AF8DCE0101963F
:10C3C0000E94C02FCE0101960E94198D8DEE90E142
:10C3D0000E94698B6130710509F06EC0709355122F
:10C3E0006093541264E279E0CE0101960E94A68D1A
:10C3F000CE0101960E94C02FCE0101960E94198D98
:10C4000062E376E0CE014C960E94B88D67EE72E151
:10C41000CE014C960E94338CBC01CE0101960E9445
:10C42000AF8D48EC50E06FEF7FEFCE0101960E9498
:10C430005437CE0101960E94198DCE014C960E9470
:10C44000198D0E948FA840E052EC61E070E088E90D
:10C450009EE00E94B88484EF91E09093570280930D
:10C46000560281E080934D0A68E971E184EF91E022
:10C470000E94972C61E476E0CE014C960E94B88D24
:10C4800061EE72E1CE014C960E94338CBC01CE016C
:10C4900001960E94AF8D40ED57E06FEF7FEFCE0128
:10C4A00001960E94FC2CCE0101960E94198DCE01AE
:10C4B0004C960E94198DEBCA61157105D1F5109249
:10C4C00055121092541266E179E0CE0101960E9455
:10C4D000A68DCE0101960E94C02FCE0101960E942A
:10C4E000198D68E376E0CE014C960E94B88D67EE18
:10C4F00072E1CE014C960E94338CBC01CE010196B4
:10C500000E94AF8D48EC50E06FEF7FEFCE010196B7
:10C510000E945437CE0101960E94198DCE014C968F
:10C520000E94198D0E948FA840E855E260E070E0FB
:10C530008ECF62307105A9F4709355126093541236
:10C5400065E079E0CE0101960E94A68DCE010196AC
:10C550000E94C02FCE0101960E94198D6CE376E0F7
:10C56000C2CF77FF94CA10924D0A70935512609310
:10C5700054128DCA6CEE7BE0CE0101960E94A68D0E
:10C58000BE016F5F7F4FCE018E960E94028C182FE6
:10C59000CE0101960E94198D112309F441C047E094
:10C5A00050E061E171E1CE0101960E948A2EBE0148
:10C5B0006F5F7F4F8DEE90E10E94E08CCE0101967F
:10C5C0000E94198D66E176E0CE0101960E94B88D39
:10C5D000BE016F5F7F4F8DEE90E10E94028C182F9D
:10C5E000CE0101960E94198D11111092330C64E155
:10C5F00075E0CE0101960E94B88DBE016F5F7F4F3E
:10C600008DEE90E10E94028C182FCE0101960E94BF
:10C61000198D112309F4EFCC81E08093330CEBCC1E
:10C6200065EE7BE0CE0101960E94A68DBE016F5F94
:10C630007F4FCE018E960E94028C182FCE0101965C
:10C640000E94198D112381F146E050E061E171E112
:10C65000CE0101960E948A2EBE016F5F7F4F8DEE44
:10C6600090E10E94E08CCE0101960E94198D8DEE22
:10C6700090E10E945E8B60939C1270939D12809358
:10C680009E1290939F1284EF91E0909357028093B3
:10C69000560268E971E10E94972C64E670E080E040
:10C6A00090E00E943D0EA7CC6CED7BE0CE010196A0
:10C6B0000E94A68DBE016F5F7F4FCE018E960E94B5
:10C6C000028C182FCE0101960E94198D112301F1C1
:10C6D00048E050E061E171E1CE0101960E948A2EAE
:10C6E000BE016F5F7F4F8DEE90E10E94E08CCE0126
:10C6F00001960E94198D8DEE90E10E945E8B6093F1
:10C70000A2127093A3128093A4129093A512BBCF90
:10C7100062ED7BE0CE0101960E94A68DBE016F5FA7
:10C720007F4FCE018E960E94028C182FCE0101966B
:10C730000E94198D112301F149E050E061E171E19E
:10C74000CE0101960E948A2EBE016F5F7F4F8DEE53
:10C7500090E10E94E08CCE0101960E94198D8DEE31
:10C7600090E10E945E8B6093A6127093A712809353
:10C77000A8129093A91287CF68EC7BE0CE010196B6
:10C780000E94A68DBE016F5F7F4FCE018E960E94E4
:10C79000028C182FCE0101960E94198D1123F1F001
:10C7A00049E050E061E171E1CE0101960E948A2EDC
:10C7B000BE016F5F7F4F8DEE90E10E94E08CCE0155
:10C7C00001960E94198D8DEE90E10E945E8B0E9471
:10C7D000D0B67093AD126093AC1255CF6DEB7BE089
:10C7E000CE0101960E94A68DBE016F5F7F4FCE01E4
:10C7F0008E960E94028C182FCE0101960E94198DF0
:10C800001123F1F04AE050E061E171E1CE010196BF
:10C810000E948A2EBE016F5F7F4F8DEE90E10E94D5
:10C82000E08CCE0101960E94198D8DEE90E10E9460
:10C830005E8B0E94D0B67093AB126093AA1223CF86
:10C8400061EB7BE0CE0101960E94A68DBE016F5F79
:10C850007F4FCE018E960E94028C182FCE0101963A
:10C860000E94198D112311F14BE050E061E171E15B
:10C87000CE0101960E948A2EBE016F5F7F4F8DEE22
:10C8800090E10E94E08CCE0101960E94198D8DEE00
:10C8900090E10E945E8B0E94D0B66093AE127093BE
:10C8A000AF128093B0129093B112EDCE6AEA7BE0A2
:10C8B000CE0101960E94A68DBE016F5F7F4FCE0113
:10C8C0008E960E94028C182FCE0101960E94198D1F
:10C8D000112309F44FC046E050E061E171E1CE015F
:10C8E00001960E948A2EBE016F5F7F4F8DEE90E110
:10C8F0000E94E08CCE0101960E94198D8DEE90E190
:10C900000E94698B7093A1116093A0118DEE90E14C
:10C910000E94698B7093400C60933F0C84EF91E010
:10C92000909357028093560268E971E10E94972C18
:10C9300064E670E080E090E00E943D0E66E476E000
:10C94000CE0101960E94B88D6DEE70E1CE01019688
:10C950000E94338CBC01CE014C960E94AF8DCE015B
:10C960004C960E945931CE014C960E94198DCE01F1
:10C9700001969FCD62EA7BE0CE0101960E94A68DD2
:10C98000BE016F5F7F4FCE018E960E94028C182FE2
:10C99000CE0101960E94198D1123B1F147E050E0BC
:10C9A00061E171E1CE0101960E948A2EBE016F5FA6
:10C9B0007F4F8DEE90E10E94E08CCE0101960E94A7
:10C9C000198D8DEE90E10E94698B7093A311609395
:10C9D000A2118DEE90E10E94698B7093420C6093DE
:10C9E000410C84EF91E0909357028093560268E9DE
:10C9F00071E10E94972C64E670E080E090E00E9474
:10CA00003D0E62E576E09CCF6CE97BE0CE010196BD
:10CA10000E94A68DBE016F5F7F4FCE018E960E9451
:10CA2000028C182FCE0101960E94198D1123E1F07E
:10CA300045E050E061E171E1CE0101960E948A2E4D
:10CA4000BE016F5F7F4F8DEE90E10E94E08CCE01C2
:10CA500001960E94198D8DEE90E10E94698B709372
:10CA6000A1126093A0120FCE66E97BE0CE01019681
:10CA70000E94A68DBE016F5F7F4FCE018E960E94F1
:10CA8000028C182FCE0101960E94198D112361F09E
:10CA90000E942F0F6093D50B7093D60B8093D70B0A
:10CAA0009093D80B0C94475D62E97BE0CE01019630
:10CAB0000E94A68DBE016F5F7F4FCE018E960E94B1
:10CAC000028C182FCE0101960E94198D112389F135
:10CAD00043E050E0BE01625D7F4FCE0101960E94AF
:10CAE0008A2EBE016F5F7F4F8DEE90E10E94E08C39
:10CAF000CE0101960E94198D8091F1109091F21053
:10CB0000892B41F08DEE90E10E94698B7093710248
:10CB10006093700280917002909171020197029768
:10CB200008F469CA81E090E09093710280937002EA
:10CB300062CA6BE87BE0CE014C960E94A68DBE01D6
:10CB4000645E7F4FCE018E960E94028C11E08111AF
:10CB500015C068E87BE0CE0101960E94A68DBE015B
:10CB60006F5F7F4FCE018E960E94028C11E0811183
:10CB700001C010E0CE0101960E94198DCE014C96A5
:10CB80000E94198D112309F468C061E87BE0CE0191
:10CB900001960E94A68DBE016F5F7F4FCE018E96DB
:10CBA0000E94028C182FCE0101960E94198D11232C
:10CBB000A1F046E050E0BE01625D7F4FCE010196DC
:10CBC0000E948A2EBE016F5F7F4F8DEE90E10E9422
:10CBD000E08CCE0101960E94198D6EE77BE0CE01BC
:10CBE00001960E94A68DBE016F5F7F4FCE018E968B
:10CBF0000E94028C182FCE0101960E94198D1123DC
:10CC0000A1F042E050E0BE01625D7F4FCE0101968F
:10CC10000E948A2EBE016F5F7F4F8DEE90E10E94D1
:10CC2000E08CCE0101960E94198D8091F1109091B7
:10CC3000F210892B09F4DFC96DEE70E1CE01019687
:10CC40000E94AF8D61E070E0CE0101960E940C4918
:10CC5000CE0101960E94198DCEC967E77BE0CE0117
:10CC600082960E94A68DBE016E5D7F4FCE018E968C
:10CC70000E94028C11E0811129C06FE67BE0CE0199
:10CC80004C960E94A68DBE01645E7F4FCE018E96AB
:10CC90000E94028C11E0811115C067E67BE0CE0195
:10CCA00001960E94A68DBE016F5F7F4FCE018E96CA
:10CCB0000E94028C11E0811101C010E0CE010196AA
:10CCC0000E94198DCE014C960E94198DCE0182963C
:10CCD0000E94198D112309F4E6C060E67BE0CE01C5
:10CCE00001960E94A68DBE016F5F7F4FCE018E968A
:10CCF0000E94028C182FCE0101960E94198D1123DB
:10CD000009F466C046E050E0BE01625D7F4FCE018F
:10CD100001960E948A2EBE016F5F7F4F8DEE90E1DB
:10CD20000E94E08CCE0101960E94198D8DEE90E15B
:10CD30000E945E8B6B017C0120E030E0A9010E9423
:10CD400006B718160CF08EC0A701960160E070E0DF
:10CD50008AE794E40E945EB60E94D0B660933902DE
:10CD600070933A0280933B0290933C028091390287
:10CD700090913A02A0913B02B0913C02181619061C
:10CD80001A061B0664F081E090E0A0E0B0E080931A
:10CD9000390290933A02A0933B02B0933C028091F7
:10CDA0007002909171028130910509F068C0809104
:10CDB000390290913A02A0913B02B0913C028093DB
:10CDC000350290933602A0933702B093380213C90C
:10CDD00047E050E0BE01625D7F4FCE0101960E94A8
:10CDE0008A2EBE016F5F7F4F8DEE90E10E94E08C36
:10CDF000CE0101960E94198D6CE974E0CE01019676
:10CE00000E94B88DBE016F5F7F4FCE018E960E944B
:10CE1000028C182FCE0101960E94198D112331F03A
:10CE200081E090E0909371028093700263EC75E072
:10CE3000CE0101960E94B88DBE016F5F7F4FCE017B
:10CE40008E960E94028C182FCE0101960E94198D99
:10CE5000112309F46BCF82E090E0909371028093EC
:10CE6000700264CF81E090E0A0E0B0E080933902EE
:10CE700090933A02A0933B02B0933C0277CF029783
:10CE800009F0B9C88091390290913A02A0913B0211
:10CE9000B0913C028093310290933202A09333020E
:10CEA000B0933402A8C86BE57BE0CE014C960E949B
:10CEB000A68DBE01645E7F4FCE018E960E94E28BEE
:10CEC00011E0811115C064E57BE0CE0101960E945E
:10CED000A68DBE016F5F7F4FCE018E960E94028CA1
:10CEE00011E0811101C010E0CE0101960E94198D60
:10CEF000CE014C960E94198D112309F48EC260E573
:10CF00007BE0CE0101960E94A68DBE016F5F7F4F30
:10CF1000CE018E960E94028C182FCE0101960E949F
:10CF2000198D112309F4FCC001E010E01093710287
:10CF30000093700210934D0200934C026FE576E06F
:10CF40008DEE90E10E94FB8A10934D0200934C02FB
:10CF500081E090E0A0E0B0E08093390290933A0243
:10CF6000A0933B02B0933C0280933502909336022B
:10CF7000A0933702B09338026DEE70E1CE010196B6
:10CF80000E94AF8D62E070E0CE0101960E940C49D4
:10CF9000CE0101960E94198D6FE37BE0CE010196D0
:10CFA0000E94A68DCE0101960E945931CE010196B4
:10CFB0000E94198D6FE27BE0CE0101960E94A68D42
:10CFC000CE0101960E942644CE0101960E94198D41
:10CFD00066E176E08DEE90E10E94FB8A6DEE70E1F5
:10CFE000CE0101960E94AF8D63E070E0CE01019604
:10CFF0000E940C49CE0101960E94198D82E090E0BA
:10D0000090937102809370026EE17BE0CE010196F5
:10D010000E94A68DCE0101960E945931CE01019643
:10D020000E94198D62E17BE0CE0101960E94A68DDF
:10D03000CE0101960E942644CE0101960E94198DD0
:10D040006FE576E08DEE90E10E94FB8A8091BE1242
:10D050009091BF1297FF06C063E676E08DEE90E1F7
:10D060000E94FB8A6DEE70E1CE0101960E94AF8DA9
:10D0700062E070E0CE0101960E940C49CE0101965B
:10D080000E94198D66E176E08DEE90E10E94FB8AA8
:10D0900082E090E090937102809370026DEE70E1F7
:10D0A000CE0101960E94AF8D63E070E0CE01019643
:10D0B0000E940C49CE0101960E94198D84EF91E0E7
:10D0C000909357028093560268E971E10E94972C71
:10D0D00064E670E080E090E00E943D0E81E090E028
:10D0E00090937102809370021092DA021092D9022A
:10D0F00082E090E0A0E0B0E08093C3029093C4028D
:10D10000A093C502B093C6020E942F0F6093E30262
:10D110007093E4028093E5029093E6020C94FB5F27
:10D120006DE07BE0CE0101960E94A68DBE016F5F8F
:10D130007F4FCE018E960E94028C182FCE01019651
:10D140000E94198D11110C94FB5F6BE07BE0CE0106
:10D1500001960E94A68DBE016F5F7F4FCE018E9615
:10D160000E94028C182FCE0101960E94198D112366
:10D1700031F081E090E0909371028093700269E059
:10D180007BE0CE0101960E94A68DBE016F5F7F4FAE
:10D19000CE018E960E94028C182FCE0101960E941D
:10D1A000198D112331F082E090E090937102809309
:10D1B000700281E090E0A0E0B0E0809339029093AB
:10D1C0003A02A0933B02B0933C028091700290918E
:10D1D00071028130910509F099C090934D028093BE
:10D1E0004C0262E07BE0CE0101960E94A68DBE015A
:10D1F0006F5F7F4FCE018E960E94028C182FCE015A
:10D2000001960E94198D112319F146E050E0BE01EC
:10D21000625D7F4FCE014C960E948A2E67E676E0D3
:10D22000CE0101960E94B88DBE01645E7F4FCE0193
:10D2300001960E94338CBC018DEE90E10E94C98C56
:10D24000CE0101960E94198DCE014C960E94198D37
:10D250008091390290913A02A0913B02B0913C0238
:10D260008093350290933602A0933702B093380230
:10D270006FE576E08DEE90E10E94FB8A6DEE70E145
:10D28000CE0101960E94AF8D62E070E0CE01019662
:10D290000E940C49CE0101960E94198D61EF7AE03F
:10D2A000CE0101960E94A68DCE0101960E945931B1
:10D2B000CE0101960E94198D81E090E090934D027D
:10D2C00080934C0266E176E08DEE90E10E94FB8A4D
:10D2D0006DEE70E1CE0101960E94AF8D63E070E0CB
:10D2E000CE0101960E940C49CE0101960E94198D33
:10D2F00061EE7AE0CE0101960E94A68DCE010196E4
:10D300000E942644CE0101960E94198D80917002E0
:10D3100090917102029711F00C94FB5F6DED7AE031
:10D320008DEE90E10E94A48C8091BE129091BF126C
:10D3300097FF06C069ED7AE08DEE90E10E94A48C23
:10D3400001E010E010934D0200934C026DEE70E18D
:10D35000CE0101960E94AF8D62E070E0CE01019691
:10D360000E940C49CE0101960E94198D66E176E07B
:10D370008DEE90E10E94FB8A68EC7AE0CE01019686
:10D380000E94A68DCE0101960E945931CE010196D0
:10D390000E94198D6DEE70E1CE0101960E94AF8D55
:10D3A00063E070E0CE0101960E940C49CE01019627
:10D3B0000E94198D6CEB7AE0CE0101960E94A68D39
:10D3C000CE0101960E942644CE0101960E94198D3D
:10D3D0008091BE129091BF12919581959109909381
:10D3E000BF128093BE1210934D0200934C0284EF43
:10D3F00091E0909357028093560268E971E10E9490
:10D40000972C64E670E080E090E00E943D0E10935F
:10D410007102009370020C94FB5F65EB7AE0CE0121
:10D4200088960E94A68DBE01685D7F4FCE018E96C4
:10D430000E94028C01E081113DC062EB7AE0CE01D6
:10D4400082960E94A68DBE016E5D7F4FCE018E96A4
:10D450000E94028C01E0811129C06EEA7AE0CE01BF
:10D460004C960E94A68DBE01645E7F4FCE018E96C3
:10D470000E94028C01E0811115C06AEA7AE0CE01B7
:10D4800001960E94A68DBE016F5F7F4FCE018E96E2
:10D490000E94028C01E0811101C000E0CE010196E2
:10D4A0000E94198DCE014C960E94198DCE01829654
:10D4B0000E94198DCE0188960E94198D002309F4CF
:10D4C0001FC263EA7AE0CE0101960E94A68DBE01DA
:10D4D0006F5F7F4FCE018E960E94028C082FCE0187
:10D4E00001960E94198D46E050E0011117C069E6CF
:10D4F00076E0CE0101960E94B88DBE016F5F7F4F2E
:10D50000CE018E960E94028C082FCE0101960E94B9
:10D51000198D002309F48BC042E050E0BE01625D2A
:10D520007F4FCE0101960E948A2EBE016F5F7F4F12
:10D530008DEE90E10E94E08CCE0101960E94198D43
:10D540008091F1109091F210892B11F40C94FB5FF3
:10D5500067E676E0CE014C960E94B88DBE01645E0F
:10D560007F4F8DEE90E10E94028C811114C061EA20
:10D570007AE0CE0101960E94A68DBE016F5F7F4FBB
:10D580008DEE90E10E94028C11E0811110E0CE013D
:10D5900001960E94198DCE014C960E94198DC12CC6
:10D5A000D12C7601112309F46AC18DEE90E10E941D
:10D5B0005E8B6B017C0180917002909171020197EA
:10D5C00009F09FC08DEE90E10E945E8B9B01AC0143
:10D5D0006091490A70914A0A80914B0A90914C0AD5
:10D5E0000E94F2B56093490A70934A0A80934B0AED
:10D5F00090934C0A8090490A90904A0AA0904B0A56
:10D60000B0904C0A20E030E044EB53E4C501B40193
:10D610000E9406B787FD86C020E030E044EB53E46B
:10D62000C501B4010E94F1B54B015C01EBCF43E0B1
:10D6300050E0BE01625D7F4FCE0101960E948A2EAE
:10D64000BE016F5F7F4F8DEE90E10E94E08CCE01B6
:10D6500001960E94198D6CE974E0CE0101960E943A
:10D66000B88DBE016F5F7F4FCE018E960E94028CF7
:10D67000082FCE0101960E94198D0023B1F081E0A0
:10D6800090E090937102809370028091C50B90910D
:10D69000C60BA091C70BB091C80B8093490A909319
:10D6A0004A0AA0934B0AB0934C0A63EC75E0CE0192
:10D6B00001960E94B88DBE016F5F7F4FCE018E969E
:10D6C0000E94028C082FCE0101960E94198D002322
:10D6D00009F436CF82E090E090937102809370025B
:10D6E0008091C10B9091C20BA091C30BB091C40B60
:10D6F0008093490A90934A0AA0934B0AB0934C0A2C
:10D700001FCF8DEE90E10E945E8B9B01AC0160917A
:10D71000490A70914A0A80914B0A90914C0A0E94E2
:10D72000F1B560CF20E030E0A901C501B4010E944D
:10D7300044B487FF0BC020E030E044EB53E4C50164
:10D74000B4010E94F2B54B015C01ECCF8092490A12
:10D7500090924A0AA0924B0AB0924C0A20E030E024
:10D76000A901C701B6010E9406B787FD15C067E190
:10D7700077E0CE0101960E94B88D6DEE70E1CE018A
:10D7800001960E94338CBC018DEE90E10E94C98C01
:10D79000CE0101960E94198D20E030E0A901C70159
:10D7A000B6010E9444B487FF6AC0809170029091D4
:10D7B0007102019799F520E030E0A901C701B60197
:10D7C0000E9406B718160CF092C020E030E040E24C
:10D7D00051E4C701B6010E94F2B522E0AB01BC01E1
:10D7E000CE014C960E94218D67E676E0CE0101962F
:10D7F0000E94B88DBE01645E7F4FCE0101960E94EB
:10D80000338CBC018DEE90E10E94C98CCE01019653
:10D810000E94198DCE014C960E94198D8091700244
:10D8200090917102019759F120E030E0A901C70100
:10D83000B6010E9406B7B701A60118160CF0705881
:10D8400022E0CE014C960E94218D67E676E0CE0163
:10D8500001960E94B88DBE01645E7F4FCE01019695
:10D860000E94338CBC018DEE90E10E94C98CCE01E8
:10D8700001960E94198DCE014C960E94198D81E06F
:10D8800090E090934D0280934C026DEE70E1CE01DA
:10D8900001960E94AF8D62E070E0CE0101960E9479
:10D8A0000C49CE0101960E94198D20E030E0A901BB
:10D8B000C701B6010E9444B487FD02C00C94FB5F0F
:10D8C0008091700290917102019711F00C94FB5FAE
:10D8D0006CE676E08DEE90E10E94FB8A6DEE70E1E1
:10D8E000CE0101960E94AF8D62E070E0ADC9A70144
:10D8F000960160E070E080E291E40E94F1B56DCFA6
:10D900006BE97AE0CE0182960E94A68DBE016E5D23
:10D910007F4FCE018E960E94028C11E0811129C0AA
:10D9200064E97AE0CE014C960E94A68DBE01645E49
:10D930007F4FCE018E960E94028C11E0811115C09E
:10D940006DE87AE0CE0101960E94A68DBE016F5F60
:10D950007F4FCE018E960E94028C11E0811101C092
:10D9600010E0CE0101960E94198DCE014C960E94C6
:10D97000198DCE0182960E94198D112309F49BC046
:10D98000CE018E960E94748B6FE576E08DEE90E16D
:10D990000E94FB8A6CE974E0CE0101960E94B88D6A
:10D9A000BE016F5F7F4FCE018E960E94028C182FB2
:10D9B000CE0101960E94198D112331F081E090E093
:10D9C000909371028093700263EC75E0CE01019632
:10D9D0000E94B88DBE016F5F7F4FCE018E960E9470
:10D9E000028C182FCE0101960E94198D112391F0FF
:10D9F00082E090E090937102809370028091BE1259
:10DA00009091BF1297FF06C069E87AE08DEE90E131
:10DA10000E94A48C81E090E090934D0280934C0290
:10DA20006DEE70E1CE0101960E94AF8D62E070E074
:10DA3000CE0101960E940C49CE0101960E94198DDB
:10DA400063E87AE0CE0101960E94A68DBE016F5F69
:10DA50007F4FCE018E960E94028C182FCE01019628
:10DA60000E94198D45E050E0111102C046E050E0DF
:10DA7000BE01625D7F4FCE0101960E948A2EBE01DB
:10DA80006F5F7F4F8DEE90E10E94E08CCE0101969A
:10DA90000E94198D8091F1109091F210892B11F450
:10DAA0000C94FB5F6DEE70E1CE0101960E94AF8D8C
:10DAB00063E070E0C9C86DE77AE0CE0182960E940B
:10DAC000A68DBE016E5D7F4FCE018E960E94028CA8
:10DAD00011E0811129C066E77AE0CE014C960E94E0
:10DAE000A68DBE01645E7F4FCE018E960E94028C91
:10DAF00011E0811115C06FE67AE0CE0101960E9417
:10DB0000A68DBE016F5F7F4FCE018E960E94028C64
:10DB100011E0811101C010E0CE0101960E94198D23
:10DB2000CE014C960E94198DCE0182960E94198DCD
:10DB3000112309F426C169E67AE0CE0101960E941C
:10DB4000A68DBE016F5F7F4FCE018E960E94028C24
:10DB5000182FCE0101960E94198D112309F443C09C
:10DB600045E050E0BE01625D7F4FCE0101960E940C
:10DB70008A2EBE016F5F7F4F8DEE90E10E94E08C98
:10DB8000CE0101960E94198D8091F1109091F210B2
:10DB9000892B61F08DEE90E10E945E8B6093490AC3
:10DBA00070934A0A80934B0A90934C0AC090490A9A
:10DBB000D0904A0AE0904B0AF0904C0A20E030E006
:10DBC00044EB53E4C701B6010E9406B787FD55C078
:10DBD00020E030E044EB53E4C701B6010E94F1B508
:10DBE0006B017C01EBCF46E050E0BE01625D7F4FF0
:10DBF000CE0101960E948A2EBE016F5F7F4F8DEE8F
:10DC000090E10E94E08CCE0101960E94198D6CE992
:10DC100074E0CE0101960E94B88DBE016F5F7F4F08
:10DC2000CE018E960E94028C182FCE0101960E9482
:10DC3000198D112331F081E090E09093710280936F
:10DC4000700263EC75E0CE0101960E94B88DBE01B2
:10DC50006F5F7F4FCE018E960E94028C182FCE01EF
:10DC600001960E94198D112309F48ECF82E090E075
:10DC7000909371028093700287CF20E030E0A90179
:10DC8000C701B6010E9444B487FF0BC020E030E01A
:10DC900044EB53E4C701B6010E94F2B56B017C016D
:10DCA000ECCFC092490AD0924A0AE0924B0AF09215
:10DCB0004C0A8091700290917102019771F4C092A8
:10DCC000C50BD092C60BE092C70BF092C80B6EE565
:10DCD0007AE083EF90E10E94A48C8091490A9091B0
:10DCE0004A0AA0914B0AB0914C0A209170023091DF
:10DCF00071022230310571F48093C10B9093C20BF5
:10DD0000A093C30BB093C40B67E57AE083EF90E177
:10DD10000E94A48C4091490A50914A0A60914B0A92
:10DD200070914C0A21E0CE014C960E94218D63EF48
:10DD300070E1CE0101960E94AF8DBE01645E7F4FFF
:10DD4000CE0101960E94338C68E475E00E941D8C20
:10DD5000BC0183EF90E10E94C98CCE0101960E9424
:10DD6000198DCE014C960E94198D63EF70E1CE01A2
:10DD700001960E94AF8DCE0101960E9426440C941C
:10DD8000286662E57AE0CE0182960E94A68DBE01E9
:10DD90006E5D7F4FCE018E960E94028C11E0811144
:10DDA00029C06CE47AE0CE014C960E94A68DBE019B
:10DDB000645E7F4FCE018E960E94028C11E081112D
:10DDC00015C066E47AE0CE0101960E94A68DBE01E0
:10DDD0006F5F7F4FCE018E960E94028C11E0811101
:10DDE00001C010E0CE0101960E94198DCE014C9623
:10DDF0000E94198DCE0182960E94198D112309F47B
:10DE000012C2C0903902D0903A02E0903B02F090EA
:10DE10003C0261E47AE0CE0101960E94A68DBE012B
:10DE20006F5F7F4FCE018E960E94028C182FCE011D
:10DE300001960E94198D112309F465C044E050E059
:10DE4000BE01625D7F4FCE0101960E948A2EBE0107
:10DE50006F5F7F4F8DEE90E10E94E08CCE010196C6
:10DE60000E94198D8091700290917102813091050C
:10DE700009F093C0C0903502D0903602E09037028E
:10DE8000F090380281E090E0A0E0B0E080933502AD
:10DE900090933602A0933702B09338028091F1102C
:10DEA0009091F210892B09F090C06BE37AE08DEE2F
:10DEB00090E10E94A48C8091F1109091F210892B36
:10DEC00081F06DEE70E1CE0101960E94AF8D70E0A1
:10DED00060E0CE0101960E940C49CE0101960E949D
:10DEE000198D80917002909171028130910509F035
:10DEF0008CC1C0923502D0923602E0923702F09285
:10DF000038020C94FB5F45E050E0BE01625D7F4F3C
:10DF1000CE0101960E948A2EBE016F5F7F4F8DEE6B
:10DF200090E10E94E08CCE0101960E94198D6CE96F
:10DF300074E0CE0101960E94B88DBE016F5F7F4FE5
:10DF4000CE018E960E94028C182FCE0101960E945F
:10DF5000198D112331F081E090E09093710280934C
:10DF6000700263EC75E0CE0101960E94B88DBE018F
:10DF70006F5F7F4FCE018E960E94028C182FCE01CC
:10DF800001960E94198D112309F46CCF82E090E074
:10DF9000909371028093700265CF029709F07ECF53
:10DFA000C0903102D0903202E0903302F0903402FF
:10DFB00081E090E0A0E0B0E08093310290933202E3
:10DFC000A0933302B093340269CF60E776E0CE01CC
:10DFD00001960E94B88DBE016F5F7F4F8DEE90E17C
:10DFE0000E94E28B182FCE0101960E94198D1123F9
:10DFF00009F477CF8DEE90E10E945E8B20E030E057
:10E00000A9010E9444B4811128C0809170029091AE
:10E010007102019731F466E37AE08DEE90E10E949F
:10E02000A48C8091700290917102029731F460E3A8
:10E030007AE08DEE90E10E94A48C8091F110909195
:10E04000F210892B09F44DCF6DEE70E1CE010196EF
:10E050000E94AF8D61E070E03CCF6DEA75E0CE01CB
:10E0600001960E94B88DBE016F5F7F4F8DEE90E1EB
:10E070000E94E28B182FCE0101960E94198D112368
:10E0800009F42FCF41E050E06DEE70E1CE01019632
:10E090000E948A2ECE0101960E945E8B4B015C018C
:10E0A000CE0101960E94198D20E030E0A901C50142
:10E0B000B4010E9444B4181634F0812C912C90E8DD
:10E0C000A92E9FE3B92E00917002109171020130C8
:10E0D000110509F075C0A501940160E070E48CE9B8
:10E0E00095E40E945EB660932D0270932E02809399
:10E0F0002F02909330026093B6127093B712809300
:10E10000B8129093B9126093290270932A028093F7
:10E110002B0290932C02B801CE014C960E94058BE5
:10E1200063E776E0CE0101960E94B88DBE01645E81
:10E130007F4FCE0101960E94338CBC01CE018296A6
:10E140000E94AF8DCE0182960E94A731CE018296A9
:10E150000E94198DCE0101960E94198DCE014C9618
:10E160000E94198D6EE17AE0CE0101960E94A68D83
:10E17000CE0101960E94A731CE0101960E94198D11
:10E1800040912D0250912E0260912F027091300229
:10E1900025E0CE0101960E94218DCE0101960E94BC
:10E1A0005931CE0101960E94198D84EF91E0909330
:10E1B00057028093560268E971E10E94972C91CE34
:10E1C0000230110509F0A7CFA501940160E070E4C9
:10E1D0008CE196E40E945EB660932D0270932E024D
:10E1E00080932F02909330026093BA127093BB1207
:10E1F0008093BC129093BD12609325027093260207
:10E20000809327029093280286CF029711F00C94F6
:10E21000FB5FC0923102D0923202E0923302F09260
:10E2200034020C94FB5F69E17AE0CE0182960E9491
:10E23000A68DBE016E5D7F4FCE018E960E94028C30
:10E2400011E0811129C063E17AE0CE014C960E9471
:10E25000A68DBE01645E7F4FCE018E960E94028C19
:10E2600011E0811115C06DE07AE0CE0101960E94A7
:10E27000A68DBE016F5F7F4FCE018E960E94028CED
:10E2800011E0811101C010E0CE0101960E94198DAC
:10E29000CE014C960E94198DCE0182960E94198D56
:10E2A000112309F429C18AA99BA9059710F40C949C
:10E2B000FB5F44E050E0BE01625D7F4FCE010196FE
:10E2C0000E948A2EBE016F5F7F4F8DEE90E10E940B
:10E2D000E08CCE0101960E94198D68E07AE0CE01B3
:10E2E00001960E94A68DBE016F5F7F4FCE018E9674
:10E2F0000E94028C182FCE0101960E94198D1123C5
:10E3000009F49BC044E050E0BE01625D7F4FCE0146
:10E3100001960E948A2EBE016F5F7F4F8DEE90E1C5
:10E320000E94E08CCE0101960E94198D8DEE90E145
:10E330000E945E8B20E030E0A9010E9406B718160B
:10E3400014F00C94FB5F8DEE90E10E945E8B609365
:10E350002D0270932E0280932F0290933002209111
:10E360007002309171022130310509F0B0C0609324
:10E37000B6127093B7128093B8129093B91260934B
:10E38000290270932A0280932B0290932C02B901E8
:10E39000CE014C960E94058B63E776E0CE01019694
:10E3A0000E94B88DBE01645E7F4FCE0101960E942F
:10E3B000338CBC01CE0182960E94AF8DCE01829635
:10E3C0000E94A731CE0182960E94198DCE0101963E
:10E3D0000E94198DCE014C960E94198D66EF79E04E
:10E3E000CE0101960E94A68DCE0101960E94A73112
:10E3F000CE0101960E94198D40912D0250912E025E
:10E4000060912F027091300225E0CE0101960E94AA
:10E41000218DCE0101960E945931CE0101960E94B4
:10E42000198D84EF91E0909357028093560268E92A
:10E4300071E10E94972C0C94FB5F45E050E0BE0117
:10E44000625D7F4FCE0101960E948A2EBE016F5FF2
:10E450007F4F8DEE90E10E94E08CCE0101960E94EC
:10E46000198D6CE974E0CE0101960E94B88DBE0151
:10E470006F5F7F4FCE018E960E94028C182FCE01C7
:10E4800001960E94198D112331F081E090E0909364
:10E4900071028093700263EC75E0CE0101960E94D8
:10E4A000B88DBE016F5F7F4FCE018E960E94028CA9
:10E4B000182FCE0101960E94198D112309F436CF31
:10E4C00082E090E090937102809370022FCF22300F
:10E4D000310509F05CCF6093BA127093BB12809340
:10E4E000BC129093BD126093250270932602809314
:10E4F0002702909328024BCF63EF79E0CE014C9630
:10E500000E94A68DBE01645E7F4FCE018E960E9452
:10E51000028C11E0811115C06FEE79E0CE010196F9
:10E520000E94A68DBE016F5F7F4FCE018E960E9426
:10E53000028C11E0811101C010E0CE0101960E9411
:10E54000198DCE014C960E94198D112309F463C0D8
:10E550006CEE79E0CE0101960E94A68DBE016F5F40
:10E560007F4FCE018E960E94028C182FCE0101960D
:10E570000E94198D112399F042E050E061E171E1B0
:10E58000CE0101960E948A2EBE016F5F7F4F8DEEF5
:10E5900090E10E94E08CCE0101960E94198D68EEF8
:10E5A00079E0CE0101960E94A68DBE016F5F7F4F7C
:10E5B000CE018E960E94028C182FCE0101960E94E9
:10E5C000198D112399F043E050E061E171E1CE0132
:10E5D00001960E948A2EBE016F5F7F4F8DEE90E103
:10E5E0000E94E08CCE0101960E94198D8DEE90E183
:10E5F0000E94698B653B710510F40C94FB5F65ED1F
:10E6000079E0CE0101960E94A68DCE0101960E946E
:10E61000A7310C94286661ED79E0CE0101960E9445
:10E62000A68DBE016F5F7F4FCE018E960E94028C39
:10E63000182FCE0101960E94198D112309F474C080
:10E6400026E030E044E050E061E171E1CE01019666
:10E650000E94CD8DBE016F5F7F4F8DEE90E10E94D5
:10E66000E08CCE0101960E94198D6DEA75E0CE0115
:10E6700001960E94B88D40911511509116118D810F
:10E680009E81481B590BBE016F5F7F4F81E191E175
:10E690000E94D6A8AC014F5F5F4F61E171E1CE01EE
:10E6A0004C960E948A2EBE01645E7F4F8DEE90E1F3
:10E6B0000E94E08CCE014C960E94198DCE010196ED
:10E6C0000E94198D8DEE90E10E945E8B88E2E1E25E
:10E6D000FAE0AFE6B2E101900D928A95E1F784EF9E
:10E6E00091E0909357028093560268E971E10E948D
:10E6F000972C60EB79E083EF90E10E94A48C44E0DA
:10E7000050E061E171E1CE0101960E948A2EBE01C6
:10E710006F5F7F4F83EF90E10E949D8CCE01019649
:10E720000E94198D0C94E95C68EA79E0CE010196AB
:10E730000E94A68DBE016F5F7F4FCE018E960E9414
:10E74000028C182FCE0101960E94198D11110C9484
:10E75000CF6261EA79E0CE0101960E94A68DBE01EA
:10E760006F5F7F4FCE018E960E94028C182FCE01D4
:10E7700001960E94198D112371F141E068E972E060
:10E78000CE0101960E940092BE016F5F7F4F8FEF16
:10E7900092E10E94662D8FEF92E10E9428206DE2A7
:10E7A00079E0882311F40C947C5B8FEF92E10E9456
:10E7B000FD0B892B51F08FEF92E10E949D1B682F7A
:10E7C00085E39FE00E941A83F0CF8FEF92E10E94D1
:10E7D00034200C94935268E979E0CE0101960E94AE
:10E7E000A68DBE016F5F7F4FCE018E960E94028C78
:10E7F000182FCE0101960E94198D1123E9F08DB7D3
:10E800009EB7855391400FB6F8949EBF0FBE8DBF43
:10E81000ADB7BEB7119685E391E0E8E9F1E101906B
:10E820000D920197E1F70E94BA440FB6F894DEBF4B
:10E830000FBECDBF0C94935262E979E0CE010196F0
:10E840000E94A68DBE016F5F7F4FCE018E960E9403
:10E85000028C182FCE0101960E94198D112309F404
:10E8600057C0EDB7FEB7E553F1400FB6F894FEBFC1
:10E870000FBEEDBFADB7BEB7119685E391E0E8E9F5
:10E88000F1E101900D920197E1F70E94A03C0FB6D3
:10E89000F894DEBF0FBECDBF61E879E0CE010196EE
:10E8A0000E94A68DADB7BEB7A553B1400FB6F89480
:10E8B000BEBF0FBEADBF119685E391E0E8E9F1E17F
:10E8C00001900D920197E1F70E94B3340FB6F894CE
:10E8D000DEBF0FBECDBF8DB79EB7855391400FB63B
:10E8E000F8949EBF0FBE8DBFADB7BEB7119685E33E
:10E8F00091E0E8E9F1E101900D920197E1F70E94C2
:10E90000BA440FB6F894DEBF0FBECDBF0C94C65705
:10E910006DE779E0CE0101960E94A68DBE016F5F82
:10E920007F4FCE018E960E94028C182FCE01019649
:10E930000E94198D1123F9F06AE679E0CE01019663
:10E940000E94A68DBE016F5F7F4FCE014C960E9444
:10E95000AF8DCE014C960E945931CE014C960E944B
:10E96000198DEDB7FEB7E553F1400FB6F894FEBF31
:10E970000FBEEDBFB9CF66E679E0CE0101960E94E9
:10E98000A68DBE016F5F7F4FCE018E960E94028CD6
:10E99000182FCE0101960E94198D112309F4F0C0A1
:10E9A0006AE379E0CE0182960E94A68DBE016E5D7B
:10E9B0007F4FCE0101960E94AF8DAE014F5F5F4F3A
:10E9C00062E070E086E792E00E94623E8C01CE0138
:10E9D00001960E94198D0130110511F1BE016E5D85
:10E9E0007F4FCE014C960E94AF8D67E776E0CE0157
:10E9F0004C960E941D8C64E471E10E94338CBC0132
:10EA0000CE0101960E94AF8DCE0101960E94593130
:10EA1000CE0101960E94198DCE014C960E94198D4F
:10EA200068EE73E080E090E00E943D0EBE016E5DF6
:10EA30007F4FCE0101960E94AF8DAE014F5F5F4FB9
:10EA400062E070E083E892E00E94623E8C01CE01B9
:10EA500001960E94198D01301105F1F0BE016E5D25
:10EA60007F4FCE014C960E94AF8D64E471E1CE01E0
:10EA70004C960E94338CBC01CE0101960E94AF8D52
:10EA8000CE0101960E945931CE0101960E94198D46
:10EA9000CE014C960E94198D68EE73E080E090E004
:10EAA0000E943D0E68E371E1CE0101960E94AF8D98
:10EAB000AE014F5F5F4F61E070E082EB92E00E9439
:10EAC000623E8C01CE0101960E94198D0130110524
:10EAD000E9F068E371E1CE014C960E94AF8D64E4E9
:10EAE00071E1CE014C960E94338CBC01CE0101969F
:10EAF0000E94AF8DCE0101960E945931CE01019640
:10EB00000E94198DCE014C960E94198D68EE73E01B
:10EB100080E090E00E943D0E8091330C882311F438
:10EB20000C94EB5E43E162EB72E0CE0101960E9431
:10EB30000092BE016F5F7F4F85E393E10E94662DD7
:10EB400085E393E10E942820882311F40C94EB5E66
:10EB500068E371E185E393E10E94DB8E66E970E092
:10EB600080E090E00E943D0E85E393E10E94342016
:10EB700062E370E080E090E00E943D0E0C94EB5E5A
:10EB800062E679E0CE0101960E94A68DBE016F5F1C
:10EB90007F4FCE018E960E94028C182FCE010196D7
:10EBA0000E94198D1123C1F009E31CE08FE3E82EC8
:10EBB0008CE0F82ED8018C910E5F1F4F60E00E9410
:10EBC000B90D6CE271E080E090E00E943D0EE0162D
:10EBD000F10681F70C9493526DE579E0CE01019630
:10EBE0000E94A68DBE016F5F7F4FCE018E960E9460
:10EBF000028C182FCE0101960E94198D1123A9F0C5
:10EC000009E31CE0F80180810E5F1F4F61E00E9464
:10EC1000B90D6CE271E080E090E00E943D0EFCE0F6
:10EC20000F331F0779F70C94935266E579E0CE0114
:10EC300001960E94A68DBE016F5F7F4FCE018E961A
:10EC40000E94028C182FCE0101960E94198D11236B
:10EC500011F40C94935227E030E046E050E061E17B
:10EC600071E1CE0101960E94CD8DBE016F5F7F4F95
:10EC70008DEE90E10E94E08CCE0101960E94198DEC
:10EC80008DEE90E10E94698B672B71F41092BC0BA2
:10EC900061E171E1CE0101960E94AF8DCE01019636
:10ECA0000E94C02F0C94746181E08093BC0BF0CF64
:10ECB0002F923F924F925F926F927F928F929F928C
:10ECC000AF92BF92CF92DF92EF92FF920F931F937A
:10ECD000CF93DF93CDB7DEB72C970FB6F894DEBF96
:10ECE0000FBECDBF2090440230904502E090460216
:10ECF000F0904702B101C7010E94E61184E1482E5D
:10ED0000512C612C712CD12CC12CAFEFCA1ADA0A0C
:10ED1000C301B2010E943D0EB101C7010E94E6117C
:10ED20008C01B3E0CB16D10434F08EE1C816D104C7
:10ED300044F4012B51F094E1490E511C611C711CEB
:10ED4000E4CF0115110509F0B0C08BE0E816F1041D
:10ED500009F090C08090D1129090D212A090D3125E
:10ED6000B090D4128091CD129091CE12A091CF127A
:10ED7000B091D01289879A87AB87BC8764E670E030
:10ED800080E090E00E943D0E6BE776E0CE010196B8
:10ED90000E94A68DCE0101960E942644CE010196C6
:10EDA0000E94198D61E082E00E948B8421E0B50110
:10EDB000A401CE0101960E94218DBE016F5F7F4F9D
:10EDC00081E593E10E94CD8ECE0101960E94198DBE
:10EDD0006FED81E593E10E94180F66E776E081E52B
:10EDE00093E10E94ED8E20E049855A856B857C85F4
:10EDF000CE0101960E94218DBE016F5F7F4F81E59C
:10EE000093E10E94CD8ECE0101960E94198D67E894
:10EE100076E081E593E10E94C58E89829A82AB8279
:10EE2000BC8289859A85AB85BC858D839E83AF83A3
:10EE3000B88729813A814B815C816D817E818F8188
:10EE400098852C960FB6F894DEBF0FBECDBFDF912C
:10EE5000CF911F910F91FF90EF90DF90CF90BF90D7
:10EE6000AF909F908F907F906F905F904F903F906A
:10EE70002F90089596E1E916F10409F46BCFACE008
:10EE8000EA16F10409F07ACF80904A0990904B0974
:10EE9000A0904C09B0904D09809146099091470986
:10EEA000A0914809B091490965CF0F3F9FEF19071D
:10EEB000CCF068E676E0CE0101960E94A68D4AE08D
:10EEC00050E070E060E0CE0101960E945437CE0120
:10EED00001960E94198D65E476E083EF90E10E942F
:10EEE000A48C32C00E3FAFEF1A07B9F167E376E0AA
:10EEF000CE0101960E94A68D4AE050E070E060E0ED
:10EF0000CE0101960E945437CE0101960E94198DC0
:10EF100068E276E083EF90E10E94A48CB801CE0114
:10EF200001960E94058BBE016F5F7F4F83EF90E1DA
:10EF30000E949D8CCE0101960E94198D62E176E0BF
:10EF400083EF90E10E94468C19821A821B821C82F8
:10EF50001D821E821F8218866CCF67E076E0CE018C
:10EF600001960E94A68D4AE050E070E060E0CE017C
:10EF700001960E945437CE0101960E94198D67EECA
:10EF800075E0ABCF2F923F924F925F926F927F923C
:10EF90008F929F92AF92BF92CF92DF92EF92FF92A9
:10EFA0000F931F93CF93DF93CDB7DEB7A6970FB61E
:10EFB000F894DEBF0FBECDBF8C017B018091BF0BEB
:10EFC0009091C00B01969093C00B8093BF0B209142
:10EFD000D90B222341F06AE070E00E9410B71816A6
:10EFE00019060CF4D2C281E08093D90B1092C00BA9
:10EFF0001092BF0B50E040E069E374E0C8010E944A
:10F00000452E82E0E816F10409F4D8C26DE574E0FB
:10F0100082E391E10E94FB8A609144027091450273
:10F0200080914602909147020E94E6111C0163E321
:10F030007EE0C8010E942C2E69E876E0C8010E949B
:10F04000C58E6BED72E1CE0101960E94AF8DBE01BF
:10F050006F5F7F4FC8010E94CD8ECE0101960E9446
:10F06000198D62E976E0C8010E94C58E6BE677E0F3
:10F07000C8010E94ED8E61EE72E1CE0101960E9400
:10F08000AF8DBE016F5F7F4FC8010E94CD8E61E6DC
:10F0900077E0C8010E94ED8E60EF71E1CE01099624
:10F0A0000E94B88DBE01675F7F4FC8010E94CD8E60
:10F0B00064E577E0C8010E94ED8E68E572E1CE015B
:10F0C0000F960E94B88DBE01615F7F4FC8010E94FC
:10F0D000CD8E6DE477E0C8010E94ED8ECE010F96D3
:10F0E0000E94198DCE0109960E94198DCE010196BC
:10F0F0000E94198D0E94700E28EE33E040E050E02F
:10F100000E948EB529013A0163E477E0C8010E94AC
:10F11000ED8ECE0101960E946D30BE016F5F7F4F74
:10F12000C8010E94CD8ECE0101960E94198DC301A7
:10F13000B20120E13EE040E050E00E94B0B54B015A
:10F140005C01B901CE0181960E94962E4CE3C42E3B
:10F15000D12CE12CF12CC501B401A70196010E942C
:10F16000B0B5B901CE0101960E94962E6FE376E00C
:10F17000CE0109960E94B88DBE016F5F7F4FCE0110
:10F1800009960E94338CBC01CE0181960E949D8C11
:10F19000CE0109960E94198DCE0101960E94198D0B
:10F1A000C301B201A70196010E94B0B5CE0101963C
:10F1B0000E94962E6FE376E0CE0109960E94B88DEC
:10F1C000BE016F5F7F4FCE0109960E94338CBC0158
:10F1D000CE0181960E949D8CCE0109960E94198DC8
:10F1E000CE0101960E94198D68E976E0CE0109965C
:10F1F0000E94B88DBE016F5D7F4FCE0109960E94BF
:10F20000338C6BE976E00E941D8CBC01CE01019627
:10F210000E94AF8DBE016F5F7F4FC8010E94CD8EEF
:10F22000CE0101960E94198DCE0109960E94198D7A
:10F2300069EA76E0C8010E94C58ECE0101960E945F
:10F240007B2CB801CE0101960E94658E64EA76E0BF
:10F25000C8010E94B38E2114310479F060914402F8
:10F260007091450280914602909147020E94E611FA
:10F270001C018C3F9F4F0CF483C00E945876298359
:10F280003A834B835C836D837E838F839887498128
:10F290005A816B817C8121E0CE010F960E94218DE5
:10F2A000BE01615F7F4FCE0109960E94AF8D61EB79
:10F2B00076E0CE0109960E941D8CBC0182E391E1AB
:10F2C0000E94C98CCE0109960E94198DCE010F961D
:10F2D0000E94198D68EB76E0CE010F960E94B88DE2
:10F2E00062E371E1CE010F960E94338CBC01CE0126
:10F2F00009960E94AF8DBE01675F7F4FC8010E94D3
:10F30000CD8ECE0109960E94198DCE010F960E94D6
:10F31000198D4D815E816F81788521E0CE0109963E
:10F320000E94218DBE01675F7F4F82E391E10E94C1
:10F33000E08CCE0109960E94198D6AEC76E0CE0130
:10F340000F960E94B88D62E371E1CE010F960E9484
:10F35000338C6BED76E00E941D8CBC01CE010996CA
:10F360000E94AF8DBE01675F7F4FC8010E94CD8EA6
:10F37000CE0109960E94198DCE010F960E94198D1B
:10F380004091C50B5091C60B6091C70B7091C80B93
:10F3900022E0CE0109960E94218D62EE76E0CE0138
:10F3A0000F960E94B88DBE01675F7F4FCE010F960A
:10F3B0000E94338C64EF76E00E941D8CBC01CE016C
:10F3C00001960E94AF8DBE016F5F7F4FC8010E9402
:10F3D000CD8ECE0101960E94198DCE010F960E940E
:10F3E000198DCE0109960E94198D4091C10B509143
:10F3F000C20B6091C30B7091C40B22E0CE01099641
:10F400000E94218D6DEF76E0CE010F960E94B88D9F
:10F41000BE01675F7F4FCE010F960E94338C64EF71
:10F4200076E00E941D8CBC01CE0101960E94AF8D3A
:10F43000BE016F5F7F4FC8010E94CD8ECE01019645
:10F440000E94198DCE010F960E94198DCE0109964A
:10F450000E94198DF6EF2F16FFEF3F062CF46EE297
:10F460007FE0C8010E942C2E6BE07EE0C8010E9464
:10F470002C2E98E9E92E91E1F92E27EDA22E22E01B
:10F48000B22ECC24C394D12C470188E0880E911C65
:10F49000E2E0AE0EB11C80919811909199118C15FB
:10F4A0009D050CF464C0B601CE0109960E94058B3F
:10F4B00065E776E0CE010F960E94B88DBE01675FCA
:10F4C0007F4FCE010F960E94338C6AEA75E00E944E
:10F4D0001D8CBC01CE0101960E94AF8DBE016F5FF5
:10F4E0007F4FC8010E94CD8EB701645E7F4FCE0171
:10F4F00045960E94B88DBE016B5E7F4FC8010E9489
:10F50000CD8E6BE077E0C8010E94C58EF501608169
:10F510007181660F771F660F771F6C557E4ECE0187
:10F520004B960E94B88DBE01655E7F4FC8010E9458
:10F53000CD8E60E177E0C8010E94C58ECE014B966A
:10F540000E94198DCE0145960E94198DCE0101961B
:10F550000E94198DCE010F960E94198DCE01099639
:10F560000E94198DFFEFCF1ADF0A74018DCFCE01F3
:10F5700081960E94198D81E08093360C6CEE7EE0BE
:10F58000C8010E942C2E1092D90BA6960FB6F894A3
:10F59000DEBF0FBECDBFDF91CF911F910F91FF90C6
:10F5A000EF90DF90CF90BF90AF909F908F907F9023
:10F5B0006F905F904F903F902F9008956EE27FE0A4
:10F5C000C8010E942C2EDACF8F929F92AF92BF92E9
:10F5D000CF92DF92EF92FF920F931F93CF93DF931F
:10F5E000CDB7DEB7A0970FB6F894DEBF0FBECDBF84
:10F5F0006DE574E08CE591E10E94FB8A6DE574E0B5
:10F6000080E591E10E94FB8A44E6842E42E0942E3C
:10F6100058E9C52E51E1D52E61EDA62E62E0B62E39
:10F6200077EDE72E72E0F72E01E010E0F401819112
:10F630009191A191B1914F01892B8A2B8B2B89F547
:10F64000F70182819381F50120813181821793072F
:10F6500041F10130110559F42091CB123091CC12B7
:10F6600037FF05C0823091050CF405C30197880F60
:10F67000991FFC01E15CF34FD801AA0FBB1FA95CE5
:10F68000B34F60818C910E94B90DF7018281938103
:10F69000F5019183808364E670E080E090E00E9451
:10F6A0003D0EF501619171915F01809198119091EA
:10F6B0009911801791070CF4E3C2CE0145960E9480
:10F6C000058BB801CE010F960E94058BB601645ED2
:10F6D0007F4FCE0109960E94B88D6AEA75E0CE018F
:10F6E00001960E94B88DBE01675F7F4FCE010196E3
:10F6F0000E94338C66E177E00E941D8CBE01615F41
:10F700007F4F0E94338C6DEA75E00E941D8CBE0114
:10F710006B5E7F4F0E94338CBC018CE591E10E94AF
:10F720009D8CCE0101960E94198DCE0109960E94F2
:10F73000198DCE010F960E94198DCE0145960E941B
:10F74000198D0F5F1F4FF8E0CF0ED11C22E0E20EA3
:10F75000F11C0430110509F069CFE091B212F0916B
:10F76000B312EE0FFF1FE153FD4F60817181CE0197
:10F7700001960E94058B46E050E0BE016F5F7F4F0F
:10F78000CE0109960E941231BE01675F7F4F80E56E
:10F7900091E10E949D8CCE0109960E94198DCE01A7
:10F7A00001960E94198DE091B412F091B512EE0FFE
:10F7B000FF1FE153FD4F60817181CE0101960E94D0
:10F7C000058B46E050E0BE016F5F7F4FCE0109968A
:10F7D0000E941231BE01675F7F4F80E591E10E9478
:10F7E0009D8CCE0109960E94198DCE0101960E9432
:10F7F000198D6AEA75E0CE0145960E94B88D0E9487
:10F80000700E28EE33E040E050E00E948EB56901B2
:10F810007A016DE574E0CE014B960E94B88D6DE5DE
:10F8200074E082E691E10E94FB8ACE0101960E947B
:10F830006D3044E150E0BE016F5F7F4FCE0109960D
:10F840000E941231BE01675F7F4F82E691E10E9404
:10F85000E08CCE0109960E94198DCE0101960E947E
:10F86000198D2AE0B701A601CE0109960E94578D95
:10F8700048E050E0BE01675F7F4FCE010F960E94C7
:10F88000123162E671E1CE0101960E94AF8DBE0198
:10F89000615F7F4FCE0101960E94338CBC0186E5EB
:10F8A00091E10E94C98CCE0101960E94198DCE0172
:10F8B0000F960E94198DCE0109960E94198D2AE09B
:10F8C000B701A601CE0109960E94578D69E177E044
:10F8D000CE0101960E94B88DBE01675F7F4FCE01B9
:10F8E00001960E94338CBE016B5E7F4F0E94338C69
:10F8F000BC0182E691E10E949D8CCE0101960E949E
:10F90000198DCE0109960E94198D4091C50B509119
:10F91000C60B6091C70B7091C80B21E0CE01019618
:10F920000E94218DBE016F5F7F4FCE014B960E94DA
:10F93000E08CCE0101960E94198D60E277E0CE0145
:10F9400001960E94B88DBE01655E7F4FCE01019683
:10F950000E94338CBE016B5E7F4F0E94338CBC01D2
:10F9600082E691E10E949D8CCE0101960E94198D44
:10F97000BE01655E7F4FCE0101960E94AF8D46E0CD
:10F9800050E0BE016F5F7F4FCE0109960E94123199
:10F99000BE01675F7F4F86E591E10E949D8CCE019D
:10F9A00009960E94198DCE0101960E94198D4091F1
:10F9B000C10B5091C20B6091C30B7091C40B21E03D
:10F9C000CE0101960E94218DBE016F5F7F4FCE0157
:10F9D0004B960E94E08CCE0101960E94198D6EE23A
:10F9E00077E0CE0101960E94B88DBE01655E7F4F23
:10F9F000CE0101960E94338CBE016B5E7F4F0E9448
:10FA0000338CBC0182E691E10E949D8CCE0101966F
:10FA10000E94198DBE01655E7F4FCE0101960E9446
:10FA2000AF8D46E050E0BE016F5F7F4FCE0109967B
:10FA30000E941231BE01675F7F4F86E591E10E940F
:10FA40009D8CCE0109960E94198DCE0101960E94CF
:10FA5000198DE0904402F090450200914602109109
:10FA60004702B701C8010E94E61190938508809370
:10FA70008408892B41F0B701C8010E94E6119093D8
:10FA800085088093840880918408909185088C3F34
:10FA90009F4F0CF415C10E94587629833A834B83FB
:10FAA0005C836D837E838F83988749815A816B81C4
:10FAB0007C8121E0CE0109960E94218DBE01675F05
:10FAC0007F4FCE014B960E94E08CCE0109960E949A
:10FAD000198D68E377E0CE0109960E94B88DBE01CA
:10FAE000655E7F4FCE0109960E94338CBE016B5E2E
:10FAF0007F4F0E94338CBC0182E691E10E949D8C75
:10FB0000CE0109960E94198DBE01655E7F4FCE0120
:10FB100009960E94AF8D46E050E0BE01675F7F4FBF
:10FB2000CE010F960E941231BE01615F7F4F86E5C4
:10FB300091E10E949D8CCE010F960E94198DCE01FD
:10FB400009960E94198D4D815E816F81788521E033
:10FB5000CE0109960E94218DBE01675F7F4FCE01C5
:10FB60004B960E94E08CCE0109960E94198D63E4A9
:10FB700077E0CE0109960E94B88DBE01655E7F4F89
:10FB8000CE0109960E94338CBE016B5E7F4F0E94AE
:10FB9000338CBC0182E691E10E949D8CCE010996D6
:10FBA0000E94198DBE01655E7F4FCE0109960E94AD
:10FBB000AF8D46E050E0BE01675F7F4FCE010F96EC
:10FBC0000E941231BE01615F7F4F86E591E10E9484
:10FBD0009D8CCE010F960E94198DCE0109960E9430
:10FBE000198D6CE571E182E691E10E949D8C6AEAD3
:10FBF00075E0CE0101960E94B88D60E571E1CE01FD
:10FC000001960E94338CBC0186E591E10E949D8C97
:10FC1000CE0101960E94198D66E571E1CE01019633
:10FC20000E94AF8DCE0101960E945931CE010196FE
:10FC30000E94198D6AE070E080E090E00E943D0E25
:10FC4000CE014B960E94198DCE0145960E94198DCA
:10FC5000A0960FB6F894DEBF0FBECDBFDF91CF9157
:10FC60001F910F91FF90EF90DF90CF90BF90AF90DA
:10FC70009F908F9008959801281B390BC901F7CCEC
:10FC8000CE0145960E94058BB801CE010F960E94C9
:10FC9000058BB6016C5E7F4FCE0109960E94B88D30
:10FCA0006AEA75E0CE0101960E94B88DBE01675FD9
:10FCB0007F4FCE0101960E94338C65E177E01CCD29
:10FCC00069E477E082E691E10E94938C68E577E051
:10FCD00086E591E10E94938C6FE577E082E691E101
:10FCE0000E94938C68E577E086E591E10E94938C11
:10FCF00078CFBF92CF92DF92EF92FF920F931F9334
:10FD0000CF93DF93CDB7DEB7C455D1090FB6F894C2
:10FD1000DEBF0FBECDBF6C018B0165965FAF4EAFEE
:10FD200065978091BF0B9091C00B01969093C00B8B
:10FD30008093BF0B8091D90B81113CC0BB24B3943D
:10FD4000B092D90B1092C00B1092BF0B6DE574E00E
:10FD5000CE01895B9F4F0E94B88D6DE574E0CE01A6
:10FD6000835B9F4F0E94B88D50E040E069E374E0F0
:10FD7000C6010E94452E0130110509F0A6C06DE5AF
:10FD800074E082E691E10E94FB8A6596EEADFFADDC
:10FD900065978081811124C00E94E47AB092360C6C
:10FDA000CE01835B9F4F0E94198DCE01895B9F4FCF
:10FDB0000E94198D0FB6F894DEBF0FBECDBFCC5A8E
:10FDC000DF4F0FB6F894DEBF0FBECDBFDF91CF91EE
:10FDD0001F910F91FF90EF90DF90CF90BF9008950B
:10FDE0006596EEADFFAD65978081882309F467C005
:10FDF00000E210E09E012F5F3F4F40E250E0BE0165
:10FE00006F5D7F4FCE018D5A9F4F0E94FC840497F7
:10FE100039F3BE016F5D7F4FCE018F5B9F4F0E9414
:10FE2000B88DBE016F5B7F4FCE01895B9F4F0E94F3
:10FE3000E08CCE018F5B9F4F0E94198DBE016F5FDA
:10FE40007F4FCE018F5B9F4F0E94B88DBE016F5BCD
:10FE50007F4FCE01835B9F4F0E94E08CCE018F5B72
:10FE60009F4F0E94198DBE01695B7F4F82E691E131
:10FE70000E949D8C63968EAD9FAD6397892B09F48C
:10FE8000AFCF6DEA75E0CE018F5B9F4F0E94B88DBA
:10FE9000BE01635B7F4FCE018F5B9F4F0E94338C0F
:10FEA0006AEA75E00E941D8CBC0182E691E10E9425
:10FEB0009D8CCE018F5B9F4F0E94198D91CF62E682
:10FEC00071E18EE391E10E94C98C1092D90B68CF49
:10FED0000895AF92BF92CF92DF92EF92FF920F936D
:10FEE0001F93CF93DF936C017B018B01040F151FD0
:10FEF000EB015E01AE18BF08C017D10759F0699138
:10FF0000D601ED91FC910190F081E02DC60119958B
:10FF1000892B79F7C501DF91CF911F910F91FF9048
:10FF2000EF90DF90CF90BF90AF900895FC01538D7C
:10FF3000448D252F30E0842F90E0821B930B5417C3
:10FF400010F0CF96089501970895FC01918D828D50
:10FF5000981761F0A28DAE0FBF2FB11D5D968C91E9
:10FF6000928D9F5F9F73928F90E008958FEF9FEF28
:10FF70000895FC01918D828D981731F0828DE80FE4
:10FF8000F11D858D90E008958FEF9FEF0895FC019E
:10FF9000918D228D892F90E0805C9F4F821B91096B
:10FFA0008F739927089588E99EE00E94C77F21E01A
:10FFB000892B09F420E0822F089585E39FE00E94B9
:10FFC000C77F21E0892B09F420E0822F0895CF928A
:10FFD000DF92EF92FF92CF93DF93809143108830AE
:10FFE00050F0CFEFDFEFCE01DF91CF91FF90EF9098
:10FFF000DF90CF900895E0916810E11142C00E9417
:020000021000EC
:10000000700E6B017C0128EEC20E23E0D21EE11CB3
:10001000F11C87E390E10E94F827882311F3809177
:100020009E10882331F08091691090916A10892B7D
:10003000C1F287E390E10E945B26EC01CF3FDC0731
:1000400071F080919E10882371F2809169109091D7
:100050006A10019790936A1080936910C4CF0E9430
:10006000700EC616D706E806F90698F610926810C4
:1000700087E390E10E94532887E390E10E941A28C9
:10008000B2CFE150E0936810F0E0E35DFF4EC38D26
:10009000D0E0A9CF0F931F93CF93DF93EC018C0196
:1000A000F80181918F018823A1F10E94E77FF80177
:1000B0002291022E000C330B8217930789F38F3F96
:1000C000980781F0A091681091E09A0F90936810C2
:1000D000B0E0A35DBF4E5B968C93903219F48FE134
:1000E000809368102FE1EC17FD07C9F092919F3FB4
:1000F000D1F3A091681081E08A0F80936810B0E07E
:10010000A35DBF4E5B969C93803269F72093681085
:10011000EACF81E0DF91CF911F910F91089580E0A8
:10012000F9CF8F929F92AF92BF92CF92DF92EF92D0
:10013000FF92CF932EED3FE03093290C2093280CB3
:10014000882309F46DC040E060E070E0CB010E94BC
:10015000AE1681110BC080E0CF91FF90EF90DF9041
:10016000CF90BF90AF909F908F9008958091010E97
:100170008F7789F780910D0E90910E0EA0910F0E42
:10018000B091100E84369105A105B10520F3C09001
:10019000090ED0900A0EE0900B0EF0900C0EC114D8
:1001A000D104E104F104B9F240E0C701B6010E94B4
:1001B000AE16882381F280914E0C90914F0C8115E0
:1001C000924049F6A091530CAA2329F26091510C58
:1001D0007091520C6115710509F4BDCF2091500C3E
:1001E000222309F4B8CFA093FC0F2093EE0F90E0E8
:1001F00080E030E0E1E0F0E0C82FAF01082E02C05F
:10020000440F551F0A94E2F72417350769F041E0BF
:10021000480F01968930910579F74093F70F9BCFEE
:10022000C12CD12C7601C0CF8093F70F2091590CAF
:1002300030915A0C50E040E02115310541F42091F5
:10024000670C3091680C4091690C50916A0C2093B6
:10025000EF0F3093F00F4093F10F5093F20F4601E0
:100260005701860E971EA11CB11C8092FD0F909223
:10027000FE0FA092FF0FB0920010E091540CF0918D
:10028000550CF0930310E0930210B0E00E94CFB53C
:10029000DC01CB01880D991DAA1DBB1D80930410A4
:1002A00090930510A0930610B093071025E0EE0F71
:1002B000FF1F2A95E1F7E150FE4FEF2FFF27E6954C
:1002C0008E0F9F1FA11DB11D8093F80F9093F90F02
:1002D000A093FA0FB093FB0F8090560C9090570CA0
:1002E000B12CA12C8114910441F48090630C909066
:1002F000640CA090650CB090660CC81AD90AEA0A82
:10030000FB0AC80CD91CEA1CFB1C04C0F694E79439
:10031000D794C794CA95D2F7C092F30FD092F40F36
:10032000E092F50FF092F60F85EFC8168FE0D80631
:10033000E104F10428F48CE08093011081E00CCFFB
:1003400080E125EFC2162FEFD206E104F104A0F3FD
:1003500080916F0C9091700CA091710CB091720C07
:100360008093041090930510A0930610B09307108B
:1003700080E2E2CF5F926F927F928F929F92AF92D4
:10038000BF92CF92DF92EF92FF920F931F93CF9382
:10039000DF93CDB7DEB7C754D1090FB6F894DEBFEF
:1003A0000FBECDBF5C013B0119A218A282E993E008
:1003B0009F8F8E8F1BA21C821B829A8389831E8231
:1003C00010E000E06E018EE1C80ED11C88E0E82E3E
:1003D00080E1F82EF501E00FF11F80818F3211F4DA
:1003E0000F5F1F4FD501A00FB11FFE01FB9690E0DC
:1003F00080E04F012D912F3249F0222339F00F5F19
:100400001F4F019621938C309105A1F7880D991DFE
:10041000FC011082F501E00FF11F80818F3211F491
:100420000F5F1F4FF501E00FF11F508041E05110A9
:1004300040E030E020E0B401C701F30119958111DB
:1004400021C0F8E0EF16F0E1FF06C1F480E0C95BDF
:10045000DF4F0FB6F894DEBF0FBECDBFDF91CF9157
:100460001F910F91FF90EF90DF90CF90BF90AF90D2
:100470009F908F907F906F905F900895C7010E942A
:10048000FA1BE4CF552091F021E0A401B701C60189
:100490000E940E1C982E88E0E81680E1F80681F094
:1004A000C7010E94FA1B911010C0D0CF98E0E91646
:1004B00090E1F90619F0C7010E94FA1B81E0C7CF4D
:1004C000992021F2FE0131967F019E2D8F2D76011C
:1004D000C92ED82E7FCF1092270C1092260C109286
:1004E000740E1092960E0E944B1085E79BE090933D
:1004F000250C8093240C86E79BE09093230C80933B
:10050000220C0895FB0101900020E9F73197AF011B
:10051000461B570BDC01ED91FC910280F381E02D2D
:1005200019940E944DB90F931F93CF93DF93EC0161
:1005300088819981009759F02A813B8126173707D6
:1005400030F081E0DF91CF911F910F9108958B01E1
:100550006F5F7F4F0E946CB8009759F09983888332
:100560001B830A832C813D81232B59F7FC011082C8
:10057000E8CF80E0E7CFEF92FF920F931F93CF93E6
:10058000DF936115710541F480E0DF91CF911F91F8
:100590000F91FF90EF90089541155105B1F07B0147
:1005A000EC010C811D81040F151FB8010E9493827C
:1005B000882351F3288139818C819D81B701820F75
:1005C000931F0E949DB91D830C8381E0DECFCF93E2
:1005D000DF93EC0188819981009711F00E94E3B7C5
:1005E000198218821D821C821B821A82DF91CF9190
:1005F0000895EF92FF920F931F93CF93DF93EC0137
:100600007B018A01BA010E94938281110BC0CE0145
:100610000E94E782CE01DF91CF911F910F91FF9051
:10062000EF9008951D830C83B701888199810E9402
:100630009DB9F0CFEF92FF920F931F93CF93DF936B
:10064000EC0181E0888F9B8D8C8D98131AC0E8890E
:10065000F989808185FF15C09FB7F894EE89FF89DD
:100660006083E889F98980818370806480839FBF7B
:1006700081E090E0DF91CF911F910F91FF90EF907B
:100680000895F62E0B8D10E00F5F1F4F0F7311278B
:10069000E02E8C8D8E110CC00FB607FCFACFE889C6
:1006A000F989808185FFF5CFCE010E946E0DF1CFD3
:1006B000EB8DEC0FFD2FF11DE35AFF4FF0829FB73A
:1006C000F8940B8FEA89FB8980818062CFCFCF932A
:1006D000DF93EC01888D8823B9F0AA89BB89E8896A
:1006E000F9898C9185FD03C0808186FD0DC00FB610
:1006F00007FCF7CF8C9185FFF2CF808185FFEDCF8E
:10070000CE010E946E0DE9CFDF91CF9108958CBD8F
:100710009DBD08958F929F92AF92BF92CF92DF922C
:10072000EF92FF920F931F93CF93DF93D091960E8A
:10073000D13208F0D7C0182FC091950E0E94180E24
:100740006B017C0180916D0E81116BC082E0809302
:100750006D0E10936C0E8FEF80936B0E10926A0EDD
:10076000D093690EA5E7BEE0E9E4FEE080E0D8138F
:1007700091C01092480E8091480ECC0FC82BC093A8
:10078000480E8091470E813009F088C01092470EC4
:100790000E94180E6B017C018091480E8093BB0073
:1007A00080916F0E9091700EA091710EB091720EAB
:1007B000892B8A2B8B2BA1F00E94180E00916F0EB3
:1007C0001091700E2091710E3091720E6C197D098E
:1007D0008E099F09061717072807390708F442C032
:1007E0008091BC0083FDD8CF85EC8093BC000E9433
:1007F000180E6B017C0180916D0E823009F450C09F
:1008000080916B0E8F3F09F46FC080916B0E803228
:1008100009F46CC080916B0E803309F469C084E0E8
:1008200026C080916F0E9091700EA091710EB091C4
:10083000720E892B8A2B8B2B09F484CF0E94180E01
:1008400080906F0E9090700EA090710EB090720E0E
:100850006C197D098E099F0986169706A806B906A8
:1008600008F070CF80916E0E0E94691085E01092A2
:10087000740E1092960E1092730EDF91CF911F910D
:100880000F91FF90EF90DF90CF90BF90AF909F902F
:100890008F9008959D9191938F5F69CF85EEA5CF3D
:1008A00080916F0E9091700EA091710EB091720EAA
:1008B000892B8A2B8B2B09F49ECF0E94180E009156
:1008C0006F0E1091700E2091710E3091720E6C1996
:1008D0007D098E099F09061717072807390708F0B1
:1008E0008ACFC0CF81E0C3CF80E0C1CF82E0BFCF4D
:1008F00083E0BDCFCF93C82F682F607F81E593E160
:100900000E94FF0E80E1C89FB001112481E593E1B0
:10091000CF910C94FF0ECF93DF9300D000D01F92A5
:100920001F92CDB7DEB798E0E1E3F3E0DE01119668
:1009300001900D929A95E1F790915A13961708F449
:100940006FEF70E0660F771F21E030E02C0F3D1F46
:10095000620F731FFB019081890F806828960FB684
:10096000F894DEBF0FBECDBFDF91CF910C947A8497
:10097000CF93DF93EC019A01AB01E889F98982E01A
:100980008083211581EE38074105510581F160E032
:1009900079E08DE390E00E948EB521503109410944
:1009A00051095695479537952795EC85FD85108219
:1009B000EE85FF852083188EEC89FD8986E0808393
:1009C000EA89FB89808180618083EA89FB89808153
:1009D00088608083EA89FB89808180688083EA89D6
:1009E000FB8980818F7D8083DF91CF910895E88995
:1009F000F989108220E1D9CF2F923F924F925F92D6
:100A00006F927F928F929F92AF92BF92CF92DF921E
:100A1000EF92FF920F931F93CF93DF9300D0CDB748
:100A2000DEB71C013B014A0129015801FC01C080CD
:100A3000D18070E060E0C3010E9482B9A80170E03B
:100A400060E0C2010E9482B9F601808110E000E0FE
:100A5000811162C004E010E004C07601F101F1826E
:100A6000E082C8010F900F900F90DF91CF911F91FE
:100A70000F91FF90EF90DF90CF90BF90AF909F903D
:100A80008F907F906F905F904F903F902F90089540
:100A90006B3209F482C06D3309F04EC08181882326
:100AA000E9F2F7018FEFE81AF80A6081653209F47C
:100AB00052C00CF048C0662309F456C082E0A81664
:100AC000B1040CF061C0012B09F46BC003E010E02D
:100AD000E8CF81818983882309F282818A83760124
:100AE000811104C0F2E0EF0EF11CB8CF83E0E80EF4
:100AF000F11C1B8240E150E070E060E0CE01019605
:100B00000E9407AC19C0F3016083F1E08F1A9108CD
:100B1000C30101963C0167017601FFEFEF1AFF0A5E
:100B2000F6016081663209F499CF0CF0B1CF6623EB
:100B300009F493CF653269F2F2E08F1691041CF745
:100B400001E010E0E8CF663209F488CF6B3209F09B
:100B5000B5CF60E2B3CF81818983882301F182819F
:100B60008A83811103C032967F0178CF7F0193E0A1
:100B7000E90EF11C1B8240E150E070E060E0CE0124
:100B800001960E9407AC9ACFF2016083F1E0AF1AA0
:100B9000B108C20101962C0184CF60E2CDCFF701EC
:100BA000E3CF02E010E07DCFAF92BF92CF92DF9211
:100BB000EF92FF920F931F93CF93DF93C82FD62FFF
:100BC0001092D5121092D6121092D7121092D812FB
:100BD0001092D91261E00E94E70D60E08C2F0E9414
:100BE000B90D6D2F70E090E080E00E943D0E60E056
:100BF0008C2F0E94E70D8BE990E00197F1F700E957
:100C000011E08C2F0E94900D892B81F40150110965
:100C1000C1F78EEF9FEFDF91CF911F910F91FF9062
:100C2000EF90DF90CF90BF90AF90089500E911E072
:100C30008C2F0E94900D019721F401501109C1F7EA
:100C4000E8CF18E2D0E800E090E9E92EFF24F39421
:100C50008C2F0E94900D892B29F481E0E81AF1086D
:100C6000B9F7D7CF0E94180E6B017C0180E9A82E3E
:100C7000BB24B3948C2F0E94900D019729F481E03E
:100C8000A81AB108B9F7C5CF0E94180E6C197D09D2
:100C90008E099F09693271058105910538F0E02FB1
:100CA000F0E0E353FD4E80858D2B8087D69511F4BF
:100CB0000F5FD0E8115041F690E080E0ACCF0F9389
:100CC0001F93CF93DF93EC010E94700E8B010E9463
:100CD00008158F3F69F00E94700E601B710B6C1736
:100CE0007D07A8F380E0DF91CF911F910F910895C8
:100CF00081E0F9CFCF93DF93EC016E857F85888902
:100D0000998941E00E94AE16882351F08A8920E239
:100D1000829FC00111248D5B934FDF91CF91089585
:100D200090E080E0FACF8F929F92AF92BF92CF92E5
:100D3000DF92EF92FF920F931F93CF93DF9300D038
:100D40001F92CDB7DEB7FC018581813091F080E044
:100D50000F900F900F900F90DF91CF911F910F91F7
:100D6000FF90EF90DF90CF90BF90AF909F908F90CB
:100D70000895848181FFEBCF83899489A589B68901
:100D8000892B8A2B8B2B09F45EC07F0140E050E059
:100D9000BA01CF010E94F1188823C9F2F701C38C70
:100DA000D48C8788908CA18CB28C82E090E0A0E0FB
:100DB000B0E0F60180839183A283B3839E012F5F0D
:100DC0003F4FB501A401C6010E949917882309F479
:100DD000BECF00E010E09801B501A401C6010E9459
:100DE000F716882309F4B3CF89809A80AB80BC8042
:100DF000F6018789803111F188EF9FEFAFEFBFE0F7
:100E000088169906AA06BB06C8F2F701178A108E43
:100E1000118E128E138A148A158A168A848180682C
:100E20008483C7010E94CB1B882309F490CF40E044
:100E300050E0BA01C7010E94F1188ACF88EF9FEFF6
:100E4000A0E0B0E0DDCF81E083CF4F925F926F9260
:100E50007F928F929F92AF92BF92CF92DF92EF924A
:100E6000FF920F931F93CF93DF93CDB7DEB76397B6
:100E70000FB6F894DEBF0FBECDBF7C016B013A0107
:100E8000FB0120E090E080E06AE03191332309F437
:100E900061C040ED430F4A3008F04DC0689FA0018B
:100EA000699F500D1124CA01C097830F911D37FD12
:100EB0009A958F3F910549F340F3F70142815381A1
:100EC000648175818091001490910114A0910214A5
:100ED000B0910314481759076A077B0709F40DC23C
:100EE0008701085F1F4F0E94700E6F7077277C5F2D
:100EF000C8010E94AB29813009F004C280E394E06C
:100F00009A838983F70182819381A481B5818B8340
:100F10009C83AD83BE8345E350E0BE016F5F7F4F8E
:100F2000C8010E94342A892BA9F5D12CC12CC801F3
:100F30000E94D72617C03E3209F0BFCF233009F4F4
:100F4000BCCFD301A20FB11D12968C932F5F90E0FE
:100F500080E09BCF233009F0B0CFF3018583CC2410
:100F6000C394D12CC60163960FB6F894DEBF0FBEB2
:100F7000CDBFDF91CF911F910F91FF90EF90DF9048
:100F8000CF90BF90AF909F908F907F906F905F9029
:100F90004F9008950E94700EF7017783668342E0B8
:100FA00050E0B7016A5F7F4FC8010E94C92981E004
:100FB00090E09A83898342E050E0BE016F5F7F4FEB
:100FC000C8010E94C92980E091E09A83898342E0A8
:100FD00050E0BE016F5F7F4FC8010E94C9291A828D
:100FE000198242E050E0BE016F5F7F4FC8010E944E
:100FF000C92942E050E0BE016F5F7F4FC8010E94E7
:10100000C92942E050E0BE016F5F7F4FC8010E94D6
:10101000C9295601F6018081882301F16501F60195
:1010200081912F01882311F08E32B1F446018A1884
:101030009B081814190474F48D8641E050E0BE0139
:10104000635F7F4FC8010E94C929A401B501C8018F
:101050000E94C9295201DECF6201E1CF1D8641E025
:1010600050E0BE01635F7F4FC8010E94C929C12CB7
:10107000DD24D394DA82C98242E050E0BE016F5F82
:101080007F4FC8010E94C929DA82C98242E050E03C
:10109000BE016F5F7F4FC8010E94C929C8010E942D
:1010A000032A892B09F441CFF3E0AF2EB12C2301A1
:1010B00022E0420E511CD4C0F70142815381648169
:1010C0007581808D918DA28DB38D481759076A0760
:1010D0007B0709F008C1848D958DC59709F003C180
:1010E00081A192A15DEFC52EDD24DA940C970CF45A
:1010F000ADC04CE050E0BE016F5F7F4FC8010E9461
:10110000B6258B819C819827892798279A8B898B74
:10111000F7014681578129813A814217530709F027
:10112000E7C097FFE5C08F7092703BEFC32EDD24C0
:10113000DA94892B09F08AC06F807884762467243A
:1011400076242AEFC22EDD24DA946114710409F4A6
:101150007DC0D12CC12C8D819E819827892798270D
:10116000C816D906F8F441E050E0BE01635F7F4F36
:10117000C8010E94B6254D85442331F050E070E04F
:1011800060E0C8010E94B6258D858111ECCF44E056
:1011900050E070E060E0C8010E94B625FFEFCF1A72
:1011A000DF0AD9CF912C812C41E050E0BE016D5E69
:1011B0007F4FC8010E94B6254B89842F807C09F09F
:1011C0006CC0442331F050E070E060E0C8010E9440
:1011D000B6258B898111E8CF42E050E0BE01615F06
:1011E0007F4FC8010E94B62542E050E0BE01635F18
:1011F0007F4FC8010E94B62544E050E070E060E0F7
:10120000C8010E94B62542E050E0BE016F5E7F4FEC
:10121000C8010E94B6258F85988949895A89811508
:10122000914009F043C0CD84DE84DC24CD24DC244D
:1012300081E0C816D104D1F54115544009F04AC0E7
:1012400044E050E0B201C8010E94B62521E0A21A94
:10125000B10809F46CCEFFEFCF16DF0609F067CEB8
:101260000E94700E3B014C01C8010E94FF25181618
:1012700019060CF421CF0E94700E661977098809AF
:101280009909693873418105910548F562E370E079
:1012900080E090E00E943D0EE7CF41E050E070E03A
:1012A00060E0C8010E94B6251B8A93CF54274527CA
:1012B000542770E060E0C8010E94B625FFEF8F1A46
:1012C0009F0A6814790409F06FCF96EFC92EDD24C8
:1012D000DA94BCCFE7EFCE2EDD24DA94B7CFCC245E
:1012E000CA94DC2CB3CF6EEFC62EDD24DA94AECFD9
:1012F0004CEFC42EDD24DA94A9CF8EEFC82EDD2466
:10130000DA9430CED12CC12C2DCEEF92FF920F93D8
:101310001F93CF93DF93EC010E942F0F7E01EE0C01
:10132000FF1CEE0CFF1CF701E152FD4F608371833F
:1013300082839383CC0FDD1FFE01E952FD4F808134
:1013400091811816190644F4FE01E153FD4F808186
:1013500091811816190654F1FE01E952FD4F01E082
:1013600010E011830083FE01E95CF34F6091410CB2
:1013700080810E94B90DC153DD4F19830883F701A5
:10138000E154FD4F88E097E0A0E0B0E080839183D6
:10139000A283B38364EF71E080E090E0DF91CF91AE
:1013A0001F910F91FF90EF900C943D0EDF91CF9124
:1013B0001F910F91FF90EF9008950F931F93CF937C
:1013C000DF934115510541F0FC01048115810115A0
:1013D000110539F4FB011082DF91CF911F910F911C
:1013E0000895415051094017510708F48A01EB0153
:1013F000FC0160817181A801CE010E94B2B9C00FC9
:10140000D11F1882E9CF20E3FC0120833296862F7A
:1014100082958F706F706A3030F4605D6293682FD0
:101420008111F5CF0895695CF9CF8F929F92AF92A9
:10143000BF92CF92DF92EF92FF920F931F93CF93C1
:10144000DF93CDB7DEB760970FB6F894DEBF0FBE5F
:10145000CDBF7C0190912E0C992351F108E093337C
:1014600009F404E06B0180E591E00E9487839E010E
:101470002F5F3F4F5901490110E0812F0E94172231
:10148000F40181934F018823D9F01F5F0113F5CF39
:1014900000E0F50181915F018D3161F0883151F0FB
:1014A0008A51823038F00F5F1013F3CF0E949223DD
:1014B00018E08AC060E170E0802F0E947522102F32
:1014C000A12EB12CF501EE0FFF1FEE5EF34F11823E
:1014D000108283EE93E00197F1F742E870E060E05C
:1014E000812F0E9458224FEF62E070E0812F0E940E
:1014F0005822B601C114D10491F4809190029091C8
:10150000910201968115F0EC9F0708F471C0909349
:101510009102809390026091900270919102812FCC
:101520000E94422286E0E9E3F3E0DE011996019091
:101530000D928A95E1F7F70183818F778C878481FB
:101540008D8785818E87A7014E5F5F4F24E030E055
:101550006CE070E0812F0E941B22B601812F0E9457
:101560002C2226E030E0AE01475F5F4F66E070E07E
:10157000812F0E941B2261E070E0812F0E94752262
:1015800027E02A9DC0012B9D900D11249C0126521D
:10159000344F7901F9011182108222E030E0AE016E
:1015A000415F5F4F68E270E0812F0E9485228F8546
:1015B0009889982789279827F70193838283168231
:1015C000158214820E949223812F60960FB6F894A0
:1015D000DEBF0FBECDBFDF91CF911F910F91FF9066
:1015E000EF90DF90CF90BF90AF909F908F90089535
:1015F00080E090EC8CCFFB0101900020E9F731975F
:10160000AF01461B570B0C94F9820F931F93CF9396
:10161000DF93CDB7DEB762970FB6F894DEBF0FBE8B
:10162000CDBF8C01CB01F80111821082138212828E
:10163000158214824AE0BE016F5F7F4F0E944EAD5B
:10164000BE016F5F7F4FC8010E94FB8A62960FB692
:10165000F894DEBF0FBECDBFDF91CF911F910F91E8
:1016600008950F931F93CF93DF93CDB7DEB7A19764
:101670000FB6F894DEBF0FBECDBF8C01CB01BA010F
:10168000F8011182108213821282158214822AE0DC
:10169000AE014F5F5F4F0E9488ADBE016F5F7F4F0D
:1016A000C8010E94FB8AA1960FB6F894DEBF0FBE58
:1016B000CDBFDF91CF911F910F910895FC018081E3
:1016C0009181009711F00C940AAD60E070E0CB01BD
:1016D0000895FC0180819181009711F00C940EAD6A
:1016E00060E070E0CB010895AF92BF92CF92DF929D
:1016F000EF92FF920F931F93CF93DF93DC01CD9076
:10170000DC901197C114D10439F01496CD91DC917D
:101710008C017601209761F4DF91CF911F910F9199
:10172000FF90EF90DF90CF90BF90AF90089575013C
:101730005701BFEFAB1ABB0AF7018081082E000CDE
:10174000990B0E9435AD892B91F72197CC0DDD1DAA
:101750008881082E000C990B0E9435AD892B29F049
:10176000CE15DF0510F02197F3CFAE014F5F5F4F2D
:101770004E195F09D80115965C934E931497CE14B9
:10178000DF0420F4B701C6010E9467B9D801ED91CA
:10179000FC91119714968D919C91E80FF91F10827E
:1017A000BBCFFC01248135816217730748F4808127
:1017B0009181009729F0860F971FFC018081089581
:1017C00080E00895FC0124813581FB01448155812D
:1017D00024173507A0F0FC0180819181009779F0F2
:1017E000FB01608171816115710549F0241B350B86
:1017F000820F931F0E9494B921E0892B09F020E009
:10180000822F0895FB0144815581FC01248135819B
:101810002417350778F080819181009759F0FB01FA
:10182000608171816115710529F00E94A4B921E0E0
:10183000892B09F020E0822F0895CF93DF93EC01EC
:10184000FB0101900020E9F73197AF01461B570BD0
:101850000E94BB82811103C0CE010E94E782CE01AB
:10186000DF91CF910895CF93DF93EC01FB01448189
:101870005581608171810E94BB82811103C0CE01BC
:101880000E94E782CE01DF91CF910895EF92FF92FF
:101890000F931F93CF93DF93EC017B01CB010E9449
:1018A00045AD0097A9F00C811D81080F191FB801E3
:1018B000CE010E949382882361F0288139818C8136
:1018C0009D81B701820F931F0E943EAD1D830C8343
:1018D00081E0DF91CF911F910F91FF90EF900895DC
:1018E000CF93DF931F921F92CDB7DEB769831A8221
:1018F00041E050E0BE016F5F7F4F0E94BB820F90BE
:101900000F90DF91CF910895CF93DF93EC0160E0CA
:101910000E94708C811103C0CE010E94E782CE012B
:10192000DF91CF910895FB0101900020E9F73197F5
:10193000AF01461B570B0C94BB82FB0144815581C0
:10194000608171810C94BB82EF92FF920F931F9381
:10195000CF93DF93EC018B01CB010E9445AD7C015D
:10196000BC01CE010E94938281110BC0CE010E9466
:10197000E782CE01DF91CF911F910F91FF90EF9001
:101980000895FD82EC82B801888199810E943EAD64
:10199000F0CFCF93DF93EC01FB018617970749F057
:1019A000608171816115710541F0448155810E940A
:1019B000F982CE01DF91CF9108950E94E782F9CF9D
:1019C0000F931F93CF93DF938C01EB01FC01808178
:1019D00091810097E1F06881798161157105A9F025
:1019E000428153812C813D814217530770F00E9440
:1019F0009DB98C819D81F801958384831D821C8211
:101A0000DF91CF911F910F9108950E94E3B78881D4
:101A10009981F801918380838A819B81938382835A
:101A20008C819D8195838483198218821B821A82FE
:101A3000E5CFFC0180819181009711F00C94E3B710
:101A40000895EF92FF920F931F93CF93DF93CDB73B
:101A5000DEB7A1970FB6F894DEBF0FBECDBF7C01F5
:101A6000CB01BA01F7011182108213821282158212
:101A7000148242E0420F8E010F5F1F4F0E9445AB60
:101A8000009789F0BC01C7010E94FB8AA1960FB69E
:101A9000F894DEBF0FBECDBFDF91CF911F910F91A4
:101AA000FF90EF900895C7010E94E782EFCF0F9358
:101AB0001F93CF93DF93CDB7DEB7A2970FB6F894FD
:101AC000DEBF0FBECDBF8C01CB01BA01F801118280
:101AD0001082138212821582148230E0AE014F5FB1
:101AE0005F4F0E9459ADBE016F5F7F4FC8010E94DA
:101AF000FB8AA2960FB6F894DEBF0FBECDBFDF9172
:101B0000CF911F910F910895CF93DF931F921F9252
:101B1000CDB7DEB7FC0111821082138212821582CA
:101B2000148269831A82BE016F5F7F4F0E94FB8A15
:101B30000F900F90DF91CF910895FC0111821082D8
:101B400013821282158214820C94E08CFC011182A3
:101B5000108213821282158214820C94A48CFC01D0
:101B60001182108213821282158214820C94C98C05
:101B7000FC01118210821382128215821482611577
:101B8000710551F0FB0101900020E9F73197AF0199
:101B9000461B570B0C94F9820895AF92BF92CF92D7
:101BA000DF92EF92FF920F931F93CF93DF936C011D
:101BB0005B017A0189012417350720F48F2D790103
:101BC000042F182F6DE574E0C6010E94B88DD50171
:101BD0001496CD91DC91EC16FD06E0F40C171D0770
:101BE00008F4E801D501ED91FC911197EC0FFD1F70
:101BF000108110826D917C916E0D7F1DC601611563
:101C00007105A1F00E94FB8AF50180819181C80FC6
